:020000040000FA
:107800005469616E59696E673130300000000000C4
:1078100054593230302E303830303030625F747925
:10782000424154333247313339474B3634464200B4
:1078300043414E5F5354440000000000000000002C
:1078400043414E5F43485F300000000000000000ED
:1078500043414E5F3530304B6270730000000000D2
:107860009407000014070000DF070000000000007C
:020000040000FA
:1080000078330020DD800000E5800000E78000007C
:108010000000000000000000000000000000000060
:10802000000000000000000000000000EF800000E1
:108030000000000000000000F3800000F9C901000A
:10804000A1130100E51301001514010045140100FE
:1080500075140100A5140100D514010005150100D7
:10806000351501006515010099150100AD150100D8
:10807000BD150100F11501000116010011160100E6
:108080004516010089160100D116010019170100DB
:1080900061170100A9170100B9170100ED170100D0
:1080A000211801005118010085180100B9180100BC
:1080B000C9180100D91801000D190100411901006A
:1080C000EF3FE8FF0448854600F02CFA00480047DF
:1080D000A50E0200C046C0467833002016488047EF
:1080E00016480047FEE7FEE7FEE7FEE7FEE7FEE78D
:1080F000FEE7FEE7FEE7FEE7FEE7FEE7FEE7FEE758
:10810000FEE7FEE7FEE7FEE7FEE7FEE7FEE7FEE747
:10811000FEE7FEE7FEE7FEE7FEE7FEE7FEE7FEE737
:10812000FEE7FEE7FEE7FEE7FEE7FEE7FEE7FEE727
:10813000FEE7FEE7FEE70000FDCF0100C58000007E
:1081400030B50B46014600202022012409E00D46EF
:10815000D5409D4205D31D469540491B2546954077
:1081600040191546521E002DF1DC30BD70B50024BB
:108170002546002801DA01244042002901DA0125C0
:108180004942FFF7DDFFAC4200D04042002C00D056
:10819000494270BDF0B51FB40646002082B00546C6
:1081A0004024019100901BE0019922460F46304681
:1081B00000F066F9049A059B801A994110D3104685
:1081C0001946224600F04CF9361A8F410197224693
:1081D00001200021009F00F043F938184D41009024
:1081E0002046641E0028DFDC019B009829463246A9
:1081F00007B0F0BDF0B51FB486B00020009001902C
:1082000002900698069980B204900798090C02041F
:108210000014114307900027089D099806913E46D7
:108220003C4603900398A9B20204000C0390049802
:108230002D0C154348430021224600F011F9C719BF
:10824000714110340E46402CECDB3846029A00F0A7
:1082500007F9009A019B80180090594102980191FA
:10826000103002904028CCDB00980BB0F0BD0346E4
:108270000B439B0703D009E008C9121F08C0042A5A
:10828000FAD203E00B780370401C491C521EF9D24D
:108290007047D2B201E00270401C491EFBD2704709
:1082A0000022F6E710B513460A4604461946FFF7C2
:1082B000F0FF204610BD30B504460020034600E024
:1082C0005B1C934203D2E05CCD5C401BF8D030BD18
:1082D0000321001D401E037812021A43491EF9D5DE
:1082E00010467047034603220870000A491C521EBC
:1082F000FAD518467047024670B54A40D30FDB07DF
:1083000040002DD04A002AD0010E140E00021202A5
:108310000919400A520A8418E50104465443000A28
:10832000120A2E045043A4194219200CC543AA185E
:10833000120C0125AD03521C521912047F3924047A
:1083400000D0521C104301D44000491EC2B20C069A
:10835000C0092018401C4008802A02D003E00020F9
:1083600070BD40084000002900DA0020184370BDAD
:1083700070B502464A40D50F40004A00ED0740085C
:108380005208002814D0002A12D0C40DD30D410287
:108390000120C0055202490A520AE41A09181218AB
:1083A0007D34914201D3641C00E04900002C01DAC5
:1083B000002070BD0023914201D3891A0343400875
:1083C00049000028F7D100290AD0914202D10121A9
:1083D000C90705E0914201D2012101E00121C94311
:1083E000E005C018401900F05CF870BD10B500221F
:1083F0009623114600F05DF810BDC20FD207400071
:1084000040080BD0C10D0723DB01C9184002090544
:10841000400A1143C208400711437047002001463B
:108420007047000010B5002904DB0124E407404236
:108430008C412146002B04DB1C460123DB07524202
:10844000A341994200D1904210BD00000122D20701
:10845000002800DB101A002900DB511A88427047FF
:1084600010B5202A04DB0146203A9140002010BDBF
:10847000914020239C1A0346E3401943904010BDCD
:1084800010B5202A04DB0846203AD040002110BD58
:108490000B46D340D0402024A21A914008431946ED
:1084A00010BD002904DA401C490001D140084000F9
:1084B000704770B40024050C05D11024000402D1CB
:1084C000002921D01124050E01D100020834050F26
:1084D00001D10001241D850F01D18000A41C0028BA
:1084E00001DB4000641C002908D020252E1B0D460E
:1084F000F540A14000D001212943084301061B1B80
:10850000000ADB1D02D5002070BC7047DB0518187F
:1085100080180029F8DA401C4900F5D170BC4008E9
:1085200040007047064C0125064E05E0E36807CC85
:108530002B430C3C98471034B442F7D3FFF7C6FDE9
:10854000E02202000023020070B58C180578401C60
:108550006B075B0F01D10378401C2A1106D102780A
:10856000401C03E006780E70401C491C5B1EF9D1CC
:108570002B0705D40023521E0DD40B70491CFAE7BB
:108580000378401CCB1A921C03E01D780D70491C27
:108590005B1C521EF9D5A142D8D3002070BD70B526
:1085A00007F090F80524204618F036FC00252846F0
:1085B00007F07CF8204618F02FFC0126304607F023
:1085C00051F8204618F028FC284607F04BF82046C2
:1085D00018F022FC304607F069F8204618F01CFC21
:1085E00070BDB0B507F06EF80524204618F014FCF5
:1085F0000125284607F05AF8204618F00DFC2846B9
:1086000007F030F8204618F007FC002007F02AF8A1
:10861000204618F001FCB0BDF0B581B007F03EF87F
:10862000052018F0F9FB08270026012007F01AF8AA
:108630000524204618F0F0FB204618F0EDFB07F06B
:1086400023F80546204618F0E7FB002007F00AF85B
:10865000204618F0E1FB76002E437F1E3806E4D159
:10866000F0B201B0F0BD70B50446002006F0FAFF8C
:1086700007F028F8052018F0CFFB0826E0B2C00963
:1086800007F014F80525284618F0C6FB012006F06F
:10869000E9FF284618F0C0FB002006F0E3FF28465B
:1086A00018F0BAFB284618F0B7FB6400761E3006B7
:1086B000E4D1052018F0B0FB012070BDF0B583B007
:1086C000019314460E4607460120384302900325C5
:1086D00004E000F08EF86D1E280631D000F067F837
:1086E0003846FFF7C0FF00F0A7F80028F1D1304668
:1086F000FFF7B9FF00F0A0F80028EAD100F057F822
:108700000298FFF7B0FF00F097F80028E1D1019838
:1087100002280BD3451E0026FFF77EFF2070FFF7CF
:108720003EFF641C761CF0B28542F5DCFFF774FF57
:108730002070FFF756FF00F05CF8202003B0F0BD7A
:10874000102003B0F0BDF0B583B01C46009201913B
:108750000290032504E000F04CF86D1E280623D09B
:1087600000F025F80298FFF77EFF00F065F800287A
:10877000F1D10198FFF777FF00F05EF80028EAD109
:10878000002C0CD00026009F3878FFF76CFF00F01B
:1087900053F80028DFD1761C7F1CA642F4D300F0EA
:1087A00028F8082003B0F0BD102003B0F0BDB0B52C
:1087B00006F088FF0524204618F02EFB01252846E8
:1087C00006F050FF204618F027FB284606F06EFF03
:1087D000204618F021FB0025284606F067FF2046BA
:1087E00018F01AFB284606F03DFF642018F014FB31
:1087F000B0BDB0B506F066FF0524204618F00CFBAE
:108800000025284606F02EFF204618F005FB2846D6
:1088100006F04CFF204618F0FFFA0125284606F026
:1088200021FF204618F0F8FA284606F03FFF6420A2
:1088300018F0F2FAB0BD0000B0B506F02FFF052425
:10884000204618F0E9FA012006F00CFF204618F047
:10885000E3FA0B4D06F018FF044606F0FDFE002C6F
:1088600002D06D1E2804F5D10525284618F0D4FA4B
:10887000002006F0F7FE284618F0CEFA2046B0BDDC
:1088800033210000034801780B2901D8491C0170ED
:108890007047C046632F002070B584B00025039553
:1088A00002950195009506F0D7FE0F20C6430E4CA9
:1088B0001036F1B2A0206A461023FFF744FF20468D
:1088C00018F0AAFA204618F0A7FA912EF0D3A020AB
:1088D000B0216A461023FFF736FF204618F09CFAB5
:1088E0000248058004B070BD581B0000562F0020C0
:1088F00070B5022902D2EB24E0B270BD891EEB25CF
:108900000022134605E0401C5B1CDDB2A94225464F
:108910000EDB04786C40154604E034466E1C072DCF
:108920003546F0D26608E407F7D09A246640F4E7AB
:10893000E0B270BDF0B591B00C91417810AA117001
:1089400083781B025918C37804792402E3181B04A6
:1089500059180B0ED3700C0C94700D0A55700B91B6
:1089600008956918099409190A93C9180278D2431D
:108970008918427983791B029A18C379047A2402F0
:10898000E3181B049A188918130A0693C918130CC4
:108990000593C9180792120E04928918827AC37A35
:1089A0001B029A18037B0F90447B2402E3181B04DC
:1089B00098180918020A02928918020C0192891863
:1089C0000D910390000E0E9000200346014606E034
:1089D00032409A40D2B211435B1C082B0ED00126C4
:1089E00035469D400746024602E07F1C042FEFD02B
:1089F00010ACE45D2542F8D0521CF6E70E9C0D98B1
:108A00000019C3B20F98827B934205D0427A9142FB
:108A100002D1002011B0F0BD1021FFF769FF0C99C1
:108A2000CC72019A8A72029A4A72039A0A72049A62
:108A3000CA71059A8A71069A4A71079A0A710A9A46
:108A4000CA70099A8A70089A4A700B9A0A7011B013
:108A5000F0BDF0B58DB055220270002747720B783B
:108A60004370CA79059202728A790492C2714A7976
:108A7000039282710A7902924271CA7A0892427311
:108A80008A7A019202734E7AC6720C7A84720CAAA8
:108A900013704D782D02EB188D78C97809024919A9
:108AA0000904CB18190E01711D0CC57009931B0A1E
:108AB0000B90837038460A91D17007959570069394
:108AC000537031020919089A1202019BD21812043C
:108AD0005118089103990902029A8918059A1202FD
:108AE000049BD2181204511805913D463A4605E000
:108AF0002640AE4032436D1C082D0ED00124214685
:108B0000A9400346064602E05B1C042BF0D00CAFE4
:108B1000FF5C3942F8D0761CF6E70B9B5A72099835
:108B200006994018079940180A994018059A801824
:108B3000110A4018110C4018110E4018089A80189C
:108B4000110A4018110C4018110E4018563898732D
:108B500010211846FFF7CCFE0DB0F0BDF0B58FB078
:108B60000446FF20E070A07060700F20C0430290A8
:108B70000F302070704818F04FF97049086863286A
:108B800001D8642008606E4F002038806D4E01903F
:108B9000308008E00B99814222D338881030388029
:108BA00080B2A1286DD206F057FD3978A02003AA23
:108BB0001023FFF783FD30802028EED103AD0BA9F1
:108BC0002846FFF7B7FEE97B8842E6D1287855288A
:108BD000E3D15D48017800290298DBD10846D9E746
:108BE0003888A0284DD8C0B20021019105E006F0D8
:108BF00033FD3988C8B2A12943D2C1B2A02003AA4B
:108C00001023FFF75BFD3080398810313980202830
:108C100037D103AD07A92846FFF78CFEE97B8842D0
:108C2000E5D128785528E2D14748007800280299F4
:108C300000D1014607988842D9D240490A68962156
:108C400051430B9A824208D90818904219D30BA9B4
:108C50000E222046FFF70BFBC9E78918814210D38B
:108C600007A90E222046FFF702FB0BA80A99818173
:108C700007980B9008980C9009980D9038880190EF
:108C8000B5E72078617809020818A178E278120225
:108C9000511809040818401C24D100200190388084
:108CA000A020B02103AA1023FFF708FD3080202860
:108CB00018D103AD0BA92846FFF73CFEE97B88429B
:108CC00010D1287855280DD11F480078002800D1F0
:108CD00002900B980299884204D20BA90E222046DA
:108CE000FFF7C5FA2078617809020818A178E278C0
:108CF0001202511809040818401C0CD10020E0721F
:108D0000A07260722072E071A07160712071E070D9
:108D1000A070607020700198388020786178090216
:108D20000818A178E27812025118090408180749B6
:108D3000086030880FB0F0BD70110100502F002086
:108D4000562F00204C2F00204F2F00205C2F00209A
:108D5000F0B581B000910646214800250570002A33
:108D60002ED01446C036631B71190F200840102204
:108D7000101A834200D303461A480278102A01D001
:108D8000042A1AD1C809FE2707405F2F13D80127EC
:108D9000B8436038C0B29E3282420CD3009A521956
:108DA000C9B2DFB23B46FFF789FC0F490880ED19D5
:108DB000A542D8D304E0082000E004200A49088036
:108DC000094801880020042902D0082900D0012088
:108DD00003490870411E8841400001B0F0BDC04603
:108DE000622F00204E2F0020602F00200A4A01230E
:108DF00013700A4A10700A4A11600A4A0021116071
:108E0000042801D105218901102801D11D208101EB
:108E1000054801807047C0464F2F00204E2F00208C
:108E2000502F00205C2F0020542F0020F0B587B079
:108E3000994D00262E80994B1B688B4224D1994C6A
:108E40002188202925D1029000920196964C002776
:108E50002760964D964E2878062809D806F0FCFB28
:108E60002068401C2060B042F5D38D480421018069
:108E70002F70904C20880107029B31D08848202118
:108E80000180854D019E0BE001204002844908804D
:108E900006E003A8FFF762FE208081488021018060
:108EA0007F4800883F2807DD874988420BDC40283F
:108EB00012D0802810D010E004280DD008280AD045
:108EC000202809D009E001214A02904204D0C902B9
:108ED000884201D001E002262E80288807B0F0BD2C
:108EE000A128019E00D32780009A012A6A4D1ED135
:108EF000187B012856D1DF719F715F711F711F733D
:108F0000587B012804D1DF729F725F721F725F73FA
:108F100003AF38461946FFF79CFDF87320880028F8
:108F200046D01038C1B2A02003AA102344E0002A82
:108F3000B6D1614801780029B2D00270187859780A
:108F4000090208189978DA781202511809040818E9
:108F50005A490978002901D00F21C943884233D2E8
:108F6000274603AC20461946FFF773FDE0733978B6
:108F7000A02010232246FFF7E6FB029A484908800A
:108F800008288DD13888103038801078517809023F
:108F900008189178D2781202511809040818484923
:108FA00008607DE7597B012911D10128A3D0A7E7EB
:108FB000A02003AA10230146FFF7C5FB384908800B
:108FC0003D48009901706BE70120C0025EE73D4813
:108FD0000078012812D103AC20461946FFF739FD6D
:108FE000E073A020B02110232246FFF7ACFB2C49F0
:108FF00008800828E4D133480770E1E718785978E9
:10900000090208189978DA78120251180904081828
:109010002B490968214A12685118884203D2204816
:1090200040210180CCE725490978002901D00F2192
:10903000C94388422DD203AF384619461C46FFF774
:1090400008FDF8731B480178A02010233A46FFF76B
:109050007AFB134908800828B2D1164908881030D5
:1090600008802078617809020818A178E278120255
:109070005118090408181249086008490A6815219E
:109080005143FFF75DF800299AD101200D4908707E
:1090900096E70120C00291E7682F0020502F0020A2
:1090A000662F00204C2F00206C2F0020632F002003
:1090B000818D5B00562F0020582F00204F2F00205D
:1090C0005C2F0020642F0020FF010000F0B585B068
:1090D0000646434C0027278004921018414A128804
:1090E000904241D201910397404F00200290386096
:1090F0003F4C404D2078052809D806F0ADFA386875
:10910000401C3860A842F5D33748042101800298FA
:1091100020703948018839480278102A01D0042A81
:1091200032D188190346C033049C651A0F240440C9
:109130001020001B854200DB0546DC09603C01264F
:109140003002E7B27F09052F12D3B443E6B29E3254
:10915000B242234C039F0DD301984218D9B2EBB20F
:109160003046FFF7F0FA05E01F482021018011E0AA
:109170001B4C039F1C49088008280BD1E8B21E4AEB
:1091800011880818108005E0012080021649088027
:10919000134C039F144800881F2809DD202813D092
:1091A00001210A0290420FD0890288420CD00CE0C3
:1091B000042809D0082808D10F480088049988425B
:1091C00001D3022700E001272780208802210143E4
:1091D000022902D1084900220A8005B0F0BDC0462C
:1091E000682F0020542F0020662F00206C2F0020B5
:1091F000632F0020818D5B00702F00204E2F0020F8
:10920000F0B585B0044600200190042C6FD20CF01C
:1092100057F8002801D10CF0D3F80020009000BFCF
:109220000098401C00900CF04BF803900398002825
:1092300003D0484900988842F2D30398002856D1B9
:10924000042145480CF01EF8444845490880210196
:10925000444A515C4900404A505A41490A88012118
:10926000090300F055F902900120049020013D49C6
:1092700040184078002801D100264BE020013949F0
:1092800040184078012802D13548068842E0200184
:1092900034494018407802282AD120014018057925
:1092A0002901304A515C49002B4A505A2C490A88FE
:1092B0000121090300F02CF9064628012A49431828
:1092C0002801284940180289280140180021C76850
:1092D0003046B84706462801224BC018C2882801EC
:1092E000C0188178304600F087F8064612E02DE07D
:1092F00020011C4940184078032804D02001401860
:109300004078132804D1200116494018868801E0CE
:10931000002004900498002818D020011249431816
:109320002001104940180289200140183146C768C1
:109330000298B847019020010A4BC018C28820014A
:10934000C0188178019800F057F80190019805B095
:10935000F0BD000050C30000EA00002088130000A8
:10936000E40000207C190200BC190200F8B5054693
:109370000E4614460020009001211C4801751C482F
:10938000007888431A490870084680780821084305
:109390001749887000208871084600780121084329
:1093A0001349087008460572002717E01048007836
:1093B000802108430E49087000BF0E48007D002838
:1093C000FBD000200B4908750948C0892080A41CE7
:1093D0000748C1890098081800907F1CB742E5D360
:1093E00031460098FEF7ACFE80B2F8BD4061004007
:1093F000005004404060004010B50346012908D1E8
:10940000094CA41A9C4202D99C18A0B20BE0064851
:1094100009E0022906D1934202DD9C1AA0B202E0C3
:10942000002000E0184610BDFFFF000010B5044604
:109430000121202002F00CF800203249087001219F
:1094400031480175002031490875152017F0CCF915
:109450002C488078E17808432A498870084680784B
:1094600021780843274988702078802806D108464B
:109470000079E17949000843224908712148807840
:10948000E17A08431F498870A078002803D1084674
:10949000007908710FE0A078012806D119480079F9
:1094A000602108431749087105E0164800798021BA
:1094B00008431449087113488079217908431149F8
:1094C000887108468079617908430E498871207A4D
:1094D000C872607A88720846007838218843094942
:1094E0000870084600786178C9000843054908708B
:1094F000A07A0873084600780121084301490870E2
:1095000010BD000000500440406100404060004039
:10951000F8B504460E461746002E01D100250FE08F
:10952000A64201DC3D460BE00094009C20467843B7
:10953000009031460098FEF703FE0090009885B237
:109540002846F8BD0146042904D28A00024BD218ED
:10955000508800E00020704720290020014604299F
:1095600003D28A00024B985C00E0002070470000A4
:1095700020290020FFB587B004460898844203DA0A
:109580000A988068002802D12448019042E0089897
:10959000001B82B20292002625460A9880680021AC
:1095A0002F463A463346049605910690FEF722FE72
:1095B00005460E46002328463146029AFEF7EAFD8C
:1095C00005460E46304600210A46494050400143B8
:1095D00002D0124801901DE003950A98C068039DCF
:1095E000A84202D30020019014E00A98C1680398B1
:1095F000401A039009990398FEF7A2FD039003987F
:10960000000C0004002802D00448019002E00398F6
:1096100080B2019001980BB0F0BD0000FFFF000088
:1096200010B5084800788021884306490870012158
:1096300005480175002005490875152017F0D4F874
:1096400010BD0000005004404061004040600040F8
:10965000F8B505460E4614461F4621462846FEF735
:1096600085FD80B2F8BD0000FFB587B006460A98B8
:109670004068002801D1029035E00A9801684068EE
:1096800008180390002534460021274603980695C4
:109690000491059038462946049B059AFEF7AAFDD9
:1096A00004460D460A984068024600230190204671
:1096B0002946FEF76FFD04460D4600232046294645
:1096C000099AFEF767FD04460D46284607492140E2
:1096D000002359405840014303D00448C04302903E
:1096E00001E0A0B2029002980BB0F0BD0000FFFFB5
:1096F00010B5FE4800688079030017F05BF8070595
:109700009ED8F5F4F3F2F100F848006840790300C0
:1097100017F050F80805138A2A8A468A638A13F0DC
:10972000A3F80020F1490968C873F048006840793F
:10973000401CEE49096848717DE0ED494969EB4AF2
:109740001268D27A885C13F007F9E848006840791B
:10975000401CE64909684871E44800684079401CAB
:10976000E2490968487166E00AF064F8002810D1FF
:1097700013F0F2F8DD4800684079401CDB490968C5
:109780004871DA4800684079401CD8490968487136
:1097900005E013F093F80020D449096848714AE0C5
:1097A0000AF048F8002811D1112013F0D5F8CF485D
:1097B00000684079401CCD4909684871CB48006871
:1097C0004079401CC9490968487105E013F076F8F2
:1097D0000020C649096848712DE00AF02BF80028DE
:1097E0001BD1C2480068C07A401CC0490968C872D1
:1097F000BE480068C07ABE49097888420DDB002067
:10980000BA490968C872B94909684862B748006826
:109810008079401CB5490968887113F04FF8002021
:10982000B2490968487106E013F048F80020AF49D2
:109830000968487100BF00BF32E3AC480068407C53
:10984000002817D0AA48C068002803D0A848C168DB
:10985000192088470020A54909684862A348006884
:109860008079401CA1490968887100209F490968D6
:1098700048711BE09D480068406A282807D29B4831
:109880000068406A401C9949096848620EE000205F
:10989000964909684862954800688079401C934958
:1098A000096888710020914909684871F8E28F4879
:1098B00000684079030016F07DFF080518A42FA466
:1098C0004CA480A412F0D0FF002088490968C87316
:1098D000864800684079401C84490968487197E0CF
:1098E000D4E2C7E230E25DE194E0814949697F4A10
:1098F0001268D27A885C13F02FF87C4800684079AF
:10990000401C7A4909684871784800684079401CD1
:109910007649096848717BE009F08CFF002811D175
:10992000012013F019F8714800684079401C6F4914
:10993000096848716D4800684079401C6B490968A6
:10994000487105E012F0BAFF0020684909684871C3
:109950005EE009F06FFF002828D164490968C97AE0
:1099600024225143634A12688918604A1268D27BE4
:10997000885C12F0F1FF5D480068C07B401C5B49C9
:109980000968C87359480068C07B242814D3574815
:1099900000684079401C554909684871534800687F
:1099A0004079401C51490968487105E012F086FF72
:1099B00000204E49096848712AE009F03BFF002861
:1099C00018D14A480068C07A401C48490968C872E2
:1099D00046480068C07A4649097888420ADB002078
:1099E00042490968C872414800688079401C3F4973
:1099F0000968887112F062FF00203C4909684871CB
:109A000006E012F05BFF002038490968487100BF8A
:109A100000BF45E2354800684079030016F0CAFEF1
:109A20000A0614B92BB948B978B995B912F01CFFD8
:109A300000202E490968C8732C4800684079401CF2
:109A40002A4909684871ABE029494969274A1268DF
:109A5000D27A885C12F080FF244800684079401C6C
:109A6000224909684871214800684079401C1F4913
:109A70000968487194E009F0DDFE002811D14A2000
:109A800012F06AFF194800684079401C17490968BC
:109A90004871164800684079401C144909684871AB
:109AA00005E012F00BFF002010490968487177E0CB
:109AB00009F0C0FE002824D1FF2012F04DFF0B4812
:109AC0000068C07B401C09490968C87307480068E2
:109AD000C07B24281BD3054800684079401C0349FB
:109AE0000968487101480068407905E0CC0700200A
:109AF000342F0020C8070020401CEA49096848713B
:109B000005E012F0DBFE0020E6490968487147E0F5
:109B100009F090FE002811D1FF2012F01DFFE1484E
:109B200000684079401CDF4909684871DD480068D9
:109B30004079401CDB490968487105E012F0BEFE1F
:109B40000020D849096848712AE009F073FE00280E
:109B500018D1D4480068C07A401CD2490968C8723C
:109B6000D0480068C07AD049097888420ADB0020D2
:109B7000CC490968C872CB4800688079401CC94943
:109B80000968887112F09AFE0020C6490968487178
:109B900006E012F093FE0020C2490968487100BF38
:109BA00000BF7DE1BF4800684079030016F002FE67
:109BB0000C0715C32CC349C366C382C39FC312F0ED
:109BC00053FE0020B7490968C873B6480068407959
:109BD000401CB44909684871B4E0B3494969B14AC5
:109BE0001268D27A885C12F0B7FEAE4800684079FD
:109BF000401CAC4909684871AA4800684079401C7B
:109C0000A849096848719DE009F014FE002811D1A7
:109C1000772012F0A1FEA34800684079401CA149BA
:109C2000096848719F4800684079401C9D4909684F
:109C3000487105E012F042FE00209A490968487117
:109C400080E009F0F7FD002811D10C2012F084FE0D
:109C5000944800684079401C9249096848719148CD
:109C600000684079401C8F490968487105E012F08E
:109C700025FE00208B490968487163E009F0DAFD90
:109C8000002810D112F068FE864800684079401C18
:109C9000844909684871834800684079401C8149BB
:109CA0000968487105E012F009FE00207D49096845
:109CB000487147E009F0BEFD002811D1132012F0D1
:109CC0004BFE784800684079401C76490968487125
:109CD000744800684079401C72490968487105E081
:109CE00012F0ECFD00206F49096848712AE009F084
:109CF000A1FD002818D16B480068C07A401C694952
:109D00000968C87267480068C07A6749097888425C
:109D10000ADB002063490968C872624800688079DC
:109D2000401C60490968887112F0C8FD00205D4937
:109D30000968487106E012F0C1FD00205949096820
:109D4000487100BF00BFABE056480068407903008F
:109D500016F030FD080513872A874787638712F0BE
:109D600083FD00204F490968C8734E480068407958
:109D7000401C4C49096848717AE04B494969494A95
:109D80001268D27A885C12F0E7FD46480068407994
:109D9000401C444909684871424800684079401CA9
:109DA00040490968487163E009F044FD002811D179
:109DB000492012F0D1FD3B4800684079401C3949E8
:109DC00009684871374800684079401C354909687E
:109DD000487105E012F072FD0020324909684871AF
:109DE00046E009F027FD002810D112F0B5FD2D48FE
:109DF00000684079401C2B4909684871294800686F
:109E00004079401C27490968487105E012F056FD69
:109E100000202449096848712AE009F00BFD002858
:109E200018D120480068C07A401C1E490968C872D1
:109E30001C480068C07A1C49097888420ADB002067
:109E400018490968C872174800688079401C15498C
:109E50000968887112F032FD0020124909684871C2
:109E600006E012F02BFD00200E490968487100BF82
:109E700000BF15E000200B4909688871094909688D
:109E80004871062007490968C87009E012F016FDFC
:109E9000002004490968487102490968887100BFB7
:109EA00000BF10BDCC070020342F002010B56A4839
:109EB00000684079030016F07DFC090610C627C62D
:109EC00044C6608EC60012F0CFFC6348006840793B
:109ED000401C614909684871BCE0604949695E4AB3
:109EE0001268D27A885C12F037FD5B4800684079CE
:109EF000401C594909684871574800684079401C1E
:109F0000554909684871A5E009F094FC002811D171
:109F10007F2012F021FD504800684079401C4E49D6
:109F2000096848714C4800684079401C4A490968F2
:109F3000487105E012F0C2FC0020474909684871E9
:109F400088E009F077FC002810D112F005FD4248A6
:109F500000684079401C4049096848713E480068E3
:109F60004079401C3C490968487105E012F0A6FCA4
:109F700000203949096848716CE009F05BFC002851
:109F800022D135480068C07A401C33490968C8723C
:109F900031480068C07A3149097888420FDB0020D7
:109FA0002D490968C8722C4800684079401C2A492C
:109FB00009684871002028490968486208E00020C3
:109FC00025490968487103E0002023490968487160
:109FD00012F074FC3EE020480068407C002816D057
:109FE0001E48C068002803D01C48C1681920884753
:109FF00000201949096848621749096848711649DB
:10A0000009688871052014490968C8701AE0124867
:10A010000068406A282807D20F480068406A401C40
:10A020000D49096848620DE000200B490968486243
:10A030000949096848710849096888710520064975
:10A040000968C87006E012F039FC0020024909686E
:10A05000487100BF00BF10BDCC070020342F002086
:10A0600010B50024F7480068807A01287ED1F548B1
:10A070000068C07900287AD0F2480068807900280A
:10A0800004D0012874D0022873D191E1ED48006812
:10A09000007B24286ED2EB480068C07901287AD171
:10A0A000002475E0E7480068C07A24214843E64967
:10A0B00009684018E3490968097B415CE148006888
:10A0C000C07A24225043E14A12688018DD4A12689F
:10A0D000127B805C814229D0DA480068C07A242152
:10A0E0004843DA4909684018D6490968097B415C48
:10A0F000D4480068C07A24225043D34A126880189A
:10A10000D04A1268127B8154CE480068407B2428D4
:10A1100005D3CC480068007BCA4909684873C94820
:10A120000068007BC7490968887308E0C548006873
:10A13000407B242803D20120C24909688871C148A4
:10A140000068007B401CBF4909680873BD4800686F
:10A15000007B242808D3BB480068407B242803D216
:10A160000120B84909688871B64805E0D3E1CDE11E
:10A1700069E0BAE138E00EE00068007B242804D2F0
:10A18000B04800688079012800D103E0601CC4B2A7
:10A19000242C87D356E0002413E0AA480068C07A34
:10A1A00024214843A94909684018015DA548006871
:10A1B000C07A24225043A44A126880180155601CBA
:10A1C000C4B2242CE9D300209E4909684873232097
:10A1D0009C490968887301209A490968887124207C
:10A1E0009849096808732DE00020964909680873AA
:10A1F00094480068C07A401C92490968C872914826
:10A200000068C07A92490978884217DB8D48006857
:10A21000007C012804D102208A490968887106E07F
:10A22000002088490968887186490968C87100203A
:10A2300084490968C8728349096808740020814903
:10A240000968487161E17F4800684079030016F0B1
:10A25000B1FA080513A62AA651A68EA601207949AF
:10A260000968087412F000FB764800684079401CC9
:10A2700074490968487199E075494969714A1268D9
:10A28000D27A885C12F068FB6E4800684079401C06
:10A290006C49096848716B4800684079401C6949FD
:10A2A0000968487182E009F0C5FA00281BD16549A8
:10A2B0000968497B491CC8B212F04EFB614800682E
:10A2C000407B60490968C8735E4800684079401C5B
:10A2D0005C49096848715B4800684079401C5949ED
:10A2E0000968487105E012F0E9FA0020554909684B
:10A2F00048715BE009F09EFA00282BD151490968AA
:10A30000C97A24225143504A126889184D4A12686A
:10A31000D27B885C12F020FB4A480068C07B401C5E
:10A3200048490968C87347480068C07B45490968BF
:10A33000897B88421ADD434800684079401C4149C6
:10A34000096848713F4800684079401C3D490968E8
:10A3500048710BE012F0B2FA3A480068407B394984
:10A360000968C87300203749096848711EE009F080
:10A3700061FA00280CD133490968887124203149D9
:10A380000968C8732F49096848732E49096888739A
:10A3900012F094FA00202B490968487106E012F087
:10A3A0008DFA002027490968487100BF00BFACE062
:10A3B000244800684079030016F0FCF908050F8E68
:10A3C000268E4C8E688E12F04FFA1E480068407937
:10A3D000401C1C490968487185E01D494969194AB2
:10A3E0001268D27A885C12F0B7FA16480068407991
:10A3F000401C144909684871124800684079401CA3
:10A400001049096848716EE009F014FA002811D16A
:10A41000492012F0A1FA0B4800684079401C094914
:10A4200009684871074800684079401C0549096877
:10A43000487105E012F042FA0020024909684871AB
:10A4400051E00000CC070020C8070020C40700200E
:10A45000342F002009F0EEF9002810D112F07CFA18
:10A460009C4800684079401C9A490968487199489D
:10A4700000684079401C97490968487105E012F06E
:10A480001DFA00209349096848712CE009F0D2F9BF
:10A4900000281AD18F480068C07A401C8D4909688D
:10A4A000C8728C480068C07A8B49097888420CDBF6
:10A4B000002088490968C8728649096888718549F9
:10A4C0000968487183490968C87112F0F7F90020DA
:10A4D00080490968487106E012F0F0F900207D49D2
:10A4E0000968487100BF00BF0FE012F0E7F90020D3
:10A4F0007849096848717749096888717549096818
:10A50000087374490968C87200BFE2E0002071490D
:10A5100009688872DDE06F480068807A0228F4D10B
:10A520006C480068007A002879D06A480068407951
:10A53000030016F03FF90B0711BB25BB41545EBB6E
:10A540007590BB0012F090F9624800684079401C99
:10A55000604909684871B7E05F494969087812F0B5
:10A56000FBF95C4800684079401C5A490968487109
:10A57000584800684079401C564909684871A3E072
:10A5800009F058F9002810D112F0E6F95148006896
:10A590004079401C4F49096848714E48006840792D
:10A5A000401C4C490968487105E012F087F9002009
:10A5B00048490968487187E009F03CF9002807D14B
:10A5C000444800684079401C42490968487103E0EA
:10A5D000002040490968487112F070F974E012F0E7
:10A5E00043F93C4800684079401C3A490968487181
:10A5F0006AE0394949690978491CC8B212F0ACF9D6
:10A60000344800684079401C324909684871314833
:10A6100000684079401C2F490968487154E054E0B3
:10A6200009F008F900280FD112F0F0F8294909685B
:10A630008870012012F064F9264800684079401CB7
:10A6400024490968487105E012F038F900202149D1
:10A650000968487138E01F480068807811280CD1DB
:10A6600000201C4909680872AA201A4909688870E4
:10A67000002018490968487011E0164800684078C1
:10A68000401C144909684870124800684078032843
:10A6900005D309F06FF900200E490968487012F0DF
:10A6A0000DF900200B49096848710DE012F006F918
:10A6B0000020084909684871064909684870AA20BD
:10A6C00004490968887000BF03E000200149096857
:10A6D000887210BDCC070020342F0020F0B505464D
:10A6E0000C4616461F462088482806DA3A46294670
:10A6F000304604F0EFFF012800D0F0BD2088C000F4
:10A700002E502088401C208000BFF6E710B502467E
:10A710009000074BC018405C002802D00320C043C3
:10A7200010BD01209300024C1B1958540020F7E77C
:10A73000B42A002070B5002508E06D1C1B48854236
:10A7400002D20AF069FE01E0002503E00AF0B8FD3C
:10A750000028F2D100BF022100200AF0BFFD032132
:10A7600000200AF0BBFD052100200AF0B7FD0721FB
:10A7700000200AF0B3FD002408E00020A1000C4AEC
:10A780005054A10089184880601CC4B2042CF4D332
:10A7900001200849087000204870052088700020BA
:10A7A000C87005480549088070BD000050C300000E
:10A7B00020290020E600002088130000E40000208B
:10A7C000F8B58D480078030015F0F4FF060405166F
:10A7D0003D5EFDFC0EE10AF0F3FD00208649C870E5
:10A7E000487008468078002802D10320087002E0F3
:10A7F000022081490870FDE07F488078002804D05D
:10A800007D488078401E7C4988700AF059FD0028F8
:10A810000BD10AF0D5FD00207749C8700846807832
:10A8200000280FD1032008700CE07348C078401C4A
:10A830007149C8700846C078052803D30520087000
:10A840000AF0EAFDD6E00AF03BFD00280ED1042113
:10A850006A480AF017FD00206749C87048706848C8
:10A86000684908800420644908700CE06248C07898
:10A87000401C6149C8700846C078052803D30520EC
:10A8800008700AF0C9FDB5E05B49497809015E4AE4
:10A89000515C4900594A505A5A490A880121090312
:10A8A000FEF736FE009001255348407800015649D6
:10A8B00040184078002801D100243CE04E48407800
:10A8C0000001514940184078012802D14D480488C0
:10A8D00031E04948407800014B494018407802284F
:10A8E00012D1454949780901474A89180879FEF784
:10A8F00029FE0446404949780901434A89180879E4
:10A90000FEF72CFE054616E03B48407800013E4924
:10A9100040184078032806D0374840780001401896
:10A920004078132806D13448407800013649401851
:10A93000848800E00025002D2FD02F4840780001AA
:10A94000324943182C48407800012F4940180289A9
:10A9500029484078000140182146C7680098B84748
:10A960000646254840780001274BC018C288224877
:10A9700040780001C01881783046FEF73DFD06465C
:10A980001D484078800022494018468001201A491D
:10A99000497889001E4A50540AE000201649497837
:10A9A00089001B4A89184880134949788900505406
:10A9B00011484078401C10494870084640780428E7
:10A9C00009D301E013E007E00AF0FAFC00200A498D
:10A9D0004870032008700DE00AF072FC002803D1D3
:10A9E00001200549087001E00AF016FD02E0FFF7BA
:10A9F000A1FE00BF00BFF8BDE6000020EA00002075
:10AA000088130000E40000207C190200BC19020039
:10AA10002029002010B50AF01DFC002405E00020CC
:10AA2000A100074A5054601CC4B2042CF7D3002084
:10AA3000044908700520887003480449088010BD47
:10AA400020290020E600002088130000E4000020F8
:10AA500070B50446002000F0AFF8002000F0DAF8EE
:10AA6000002000F09BF8002000F0C4F8002000F067
:10AA700087F8002000F0AEF800BF012000F08EF84B
:10AA8000012000F0B7F8002521E0002000F086F852
:10AA9000002000F0AFF880202040002806D00120E0
:10AAA00000F08AF8012000F0B5F805E0002000F081
:10AAB00083F8002000F0AEF800BF012000F06EF82F
:10AAC000012000F097F86006040E681CC5B2082D3E
:10AAD000DBDB012000F054F8012000F07BF870BDB2
:10AAE00070B504460D46012000F066F8012000F024
:10AAF00091F8002000F052F8002000F07BF80020D0
:10AB000000F03EF8002000F065F800BF012000F0E2
:10AB100045F8012000F06EF8002628E0002000F043
:10AB20003DF8002000F066F880202040002803D087
:10AB3000012000F041F802E0002000F03DF8802004
:10AB40002840002803D0012000F064F802E0002033
:10AB500000F060F800BF012000F020F8012000F0B4
:10AB600049F86006040E6806050E701CC6B2082E71
:10AB7000D4DB012000F004F8012000F02BF870BDB8
:10AB800010B50446002C04D0812103200AF0D6FC25
:10AB900003E0802103200AF0D1FC10BD10B504466B
:10ABA000002C04D0812104200AF0C8FC03E080219D
:10ABB00004200AF0C3FC10BD10B50446002C04D0DC
:10ABC000812102200AF0BAFC03E0802102200AF071
:10ABD000B5FC10BD10B50446002C04D081210448FA
:10ABE0000AF0ACFC03E0802101480AF0A7FC10BD8C
:10ABF0000107000010B50446002C05D08121072074
:10AC000000020AF09BFC04E08021072000020AF009
:10AC100095FC10BD10B50446002C04D081210448D9
:10AC20000AF08CFC03E0802101480AF087FC10BD8B
:10AC30000207000010B5F920FFF70AFF8820FFF790
:10AC400007FF9020FFF704FF9820FFF701FF08217E
:10AC50000846FFF745FFE820FFF7FAFE12210846F5
:10AC6000FFF73EFFA020FFF7F3FE70210846FFF735
:10AC700037FFA820FFF7ECFE70210846FFF730FFF2
:10AC8000B020FFF7E5FE70210846FFF729FFB82046
:10AC9000FFF7DEFE00210846FFF722FFC020FFF786
:10ACA000D7FE00210846FFF71BFFC820FFF7D0FEA4
:10ACB00000210846FFF714FFD020FFF7C9FE2F211F
:10ACC0000846FFF70DFFD820FFF7C2FE2F210846E8
:10ACD000FFF706FFE020FFF7BBFE2F210846FFF736
:10ACE000FFFE4020FFF7B4FE00210846FFF7F8FE04
:10ACF0000A20FFF7ADFE002405E000210846FFF71B
:10AD0000EFFE601CC4B25A2CF7DB00240AE00020DE
:10AD10000B4908550B4908550B4908550B4908556F
:10AD2000601CC4B25A2CF2DB8120FFF791FE002098
:10AD3000074908708870C8700871487010BD00001D
:10AD400048260020A2260020FC26002056270020AE
:10AD5000BB00002010B58020FFF77AFE10BD000078
:10AD60000020044908700120034908700020487041
:10AD700070470000C0000020BB00002010B548480C
:10AD8000007800287AD046488078030015F012FD3C
:10AD90000604434A535A687E414800794149085C99
:10ADA0003F490979404A515C884209D13C480079C1
:10ADB0003E49085C3A4909793D4A515C88421BD0BA
:10ADC000374800793749085C35490979364A505483
:10ADD000334800793549085C31490979344A50547F
:10ADE0002F48C078002803D004202D49887011E036
:10ADF00001202B4988700DE000202949C8700846C1
:10AE00000079401C0871084600795A2802DB0020AE
:10AE10000871087041E04020FFF71AFE0220204927
:10AE200088703AE01E4A11791079FFF759FE032025
:10AE30001B49887031E00A20FFF70AFE04201849F8
:10AE400088702AE0164A1279194B995C144A1279D3
:10AE5000154B985CFFF744FE0520114988701CE0F3
:10AE60000F480079401C0E490871084600795A289D
:10AE700005DB002008710870C87003E00EE00120B7
:10AE80000749C87000200649887006E00020044980
:10AE900008708870C870087100BF00BF10BD000046
:10AEA000BB00002048260020A2260020FC2600200F
:10AEB0005627002010B512F00FF9012837D10720CE
:10AEC00009F08EFA002810D01C480078052805DA11
:10AED0001A480078401C1949087016E005201749E7
:10AEE00008700020164908700FE015480078052802
:10AEF00005DA13480078401C1149087005E0052068
:10AF00000F49087000200D4908700C48007805288A
:10AF100006D14B22D2000021012013F00BFE0BE0E2
:10AF20007D22D2000021012013F004FE04E0002263
:10AF30001146012013F0FEFD10BD00001D00002091
:10AF40001C00002000200349087248708870486087
:10AF500070470000580A002058221152704710B55F
:10AF600004460121022000F073FA0021022000F0C3
:10AF70006FFA10BD014600205322525C10231A4084
:10AF8000002A08D05322525C0C231A409210032A44
:10AF900018D1032016E05422525A0123DB031A4031
:10AFA000002A0ED05322525C0C231A409210032A1E
:10AFB00005D05322525C9207920F032A01D102203E
:10AFC00000E0012070470246002058239B5A0B40A6
:10AFD000002B01D0012000E0002070470146002234
:10AFE0006020405AFF231B0218400005020F100189
:10AFF000014BC018704700000055044010B5002AEE
:10B000000AD056231B5A0C0223435624235256239C
:10B010001B5A8B43235209E056231B5A0C02A343AD
:10B020005624235256231B5A0B43235210BD0000B3
:10B03000F8B504460D46012700263448844203D162
:10B040000121022000F004FA2878401EA070208818
:10B05000FF210131084320802088400840002080E3
:10B06000A878401EC1B25A20015568790007000C2B
:10B07000E97909020843A97908435C210853288922
:10B0800081B240200153A868C000C10C4220015386
:10B09000A88981B244200153E868C000C10C462051
:10B0A0000153288A81B2482001532869C000C10C8D
:10B0B0004A200153A88A81B24C2001536869C0001C
:10B0C000C10C4E2001535020005B2979090208432E
:10B0D000502108535020005B2979884350210853A0
:10B0E00000E0761C5020005B4007400F2979884221
:10B0F00002D007488642F4D15020005B4007400F41
:10B100002979884200D000273846F8BD0054044011
:10B11000FFFF000030B5034600201C898C4209DD8A
:10B12000082A05D218244C431D682C19A05C02E0A3
:10B13000002000E0002030BD10B5024613898B428C
:10B1400005DD18234B431468E318987C00E00020C9
:10B1500010BD0146FF22C889C007C00F00280AD0D1
:10B160000120C88100E0521EC889C007C00F002816
:10B1700001D0002AF7D1C889C007C00F00280FD11D
:10B180000220C8810420C881487A400840004872E3
:10B19000487A38239843487200204872012070474B
:10B1A0000020FCE70246507A012318435072507A7F
:10B1B0000B78DB0018435072087A012808D1888880
:10B1C00050814868000C0123DB031843908108E09C
:10B1D000087A002805D15081486880001A4B184031
:10B1E0009081487A012804D1507A40231843507244
:10B1F00006E0487A002803D1507A402398435072E1
:10B200000878002811D1C87A1072087B1070487B2A
:10B210005070887B9070CB7BD370087C10714B7C16
:10B220005371887C9071CB7CD371887A002803D0CD
:10B230000120C002D08101E00820D081FF20013030
:10B24000D081012070470000FC1F0000002904D0BD
:10B25000427A80231A43427203E0427A80239A435F
:10B260004272704730B5024600200F4B5024A45A5A
:10B270000D022C435025AC525024A45A8C43AC529E
:10B2800000E05B1E5024A45A6407640F8C4201D076
:10B29000002BF6D15024A45A6407640F002C01D06F
:10B2A000002000E0012030BDFFFF0000827A8023F3
:10B2B0001A40802A00D081727047000070B50446A1
:10B2C00000250023002D02D0012660200653042013
:10B2D000C88188890126F6033040002808D0012063
:10B2E00010728889C004C0084E893043506006E05F
:10B2F0000020107288890F4E304080105060087A0C
:10B30000D072002304E0CE5C10460C30C6545B1CA7
:10B31000D07A9842F7DCC88904263040002804D14E
:10B32000C889F6023040002801D0002070BDD07AD4
:10B33000FCE70000FC1F00000020024908800249D1
:10B34000088070477A0000207C000020027C802367
:10B350001A40802A00D00174704710B50246FF23BE
:10B36000D089C007C00F002802D00120D0815B1E09
:10B37000D089C007C00F002801D0002010BD507A2E
:10B38000012420435072507A3824A0435072C87A66
:10B390001072487A00280FD1087B1070487B5070DB
:10B3A000887B9070CC7BD470087C10714C7C54717D
:10B3B000887C9071CC7CD471FF200130D08140001A
:10B3C000D081107ADAE70000F8B504460D46002077
:10B3D000002C00D100BF002A00D100BF012C01D1F8
:10B3E00041263043012A01D112263043022C01D1DB
:10B3F000C0263043022A01D130263043134E30702C
:10B4000076788027BE43114F7E70012C08D1FF2132
:10B4100000BF0E4EB3781E460E4033468B42F8D125
:10B420000A4E76784027BE43084F7E70012A0BD122
:10B430000026009603E000BF009E761C0096FF27C2
:10B440006937009EBE42F6D9F8BD000000040240F4
:10B45000002905D0054A12780243044B1A7004E013
:10B46000024A12788243014B1A707047200402404E
:10B47000002905D0054A927E0243044B9A7604E0E7
:10B48000024A927E8243014B9A767047000802403E
:10B4900001200649087000BF044800788021084058
:10B4A0000028F9D00120024908707047000C0240C2
:10B4B0009C01002070B5034614460020002B01D1EA
:10B4C000C0B202E005468035E8B2012902D1051D6F
:10B4D000E8B206E0022903D105460835E8B200E0EB
:10B4E000C0B2012C02D1851CE8B200E0C0B2084D08
:10B4F000A870AD7801263543054EB570002201E0F5
:10B5000000BF521C7D252D01AA42F9D970BD000053
:10B51000000C024070B50024244800792021084026
:10B52000002801D0224D3FE000F046F805462148B2
:10B53000007880210840002836D01E4880780840D6
:10B54000002801D01A4D02E000F036F805461948EF
:10B5500080780007840F022C01DBAD0804E0012C89
:10B5600001D16D0800E000BF124880788007C00F4D
:10B57000002801D02D0101E00C2045430D48007842
:10B580004007840F002C02D1601CC4B207E0032CDA
:10B5900003D1601C4006040E01E06006040E214643
:10B5A0002846FCF7CDFD0546284670BD0004024044
:10B5B00000127A00000C024000B5C0229178F822F7
:10B5C00011401C4A12781143EA2923D00ADC0A46AA
:10B5D000E03A130015F0EEF80A181C20242A2A2A53
:10B5E0002A161A2AED291FD004DCEB2916D0EC29E3
:10B5F0001CD117E0F02903D0F82917D10E4817E025
:10B600000E4815E00E4813E00E4811E00E480FE01A
:10B610000E480DE00E480BE00E4809E00E4807E02A
:10B620000E4805E00E4803E00E4801E00D4800BF5B
:10B6300000BF00BD201C02400090D003006CDC0263
:10B640000048E80100366E010024F400001BB7003A
:10B6500000127A00808D5B0000093D00C0C62D00FD
:10B6600080841E0040420F0070B586B0044600255D
:10B67000002620680290A1796846C1736179417300
:10B6800000210173017100BF05E020460830415DD3
:10B6900004A841556D1C6846C07BA842F5D80B2212
:10B6A000D2010299881A914237D007DC2548081A3E
:10B6B0001FD023210901401A3AD113E0FF386F3817
:10B6C000002802D0012833D105E001A91E48FFF768
:10B6D00044FE06462DE001A91B484030FFF73DFE21
:10B6E000064626E001A918485030FFF736FE064608
:10B6F0001FE001A914482030FFF72FFE064613482B
:10B700000088072805DA11480088401C0F49088086
:10B7100002E000200D4908800BE005F071FC0028D4
:10B7200005D001A908486030FFF717FE064600E083
:10B7300000BF00BF002E02D1012006B070BD002066
:10B74000FBE7000020020000805504407C00002040
:10B7500010B5A8211348FCF7A3FD12481249086050
:10B7600012484860072008810020887207220F498C
:10B770000D4800F06BFA00210B48FFF797FDA02160
:10B780000B48FCF78DFD0A480A4948600A4B052220
:10B790000A49084800F01CFC00210648FFF7D6FDC6
:10B7A00010BD00006C0800204C080020B4150200F9
:10B7B000140900205808002069B60000281502006E
:10B7C0000C4A127812060B4B5B781B041A43094B88
:10B7D0009B781B021A43074BDB781A43104642083A
:10B7E0004240D20083085A401146034A5140034A5E
:10B7F00011607047130700200102000018070020A5
:10B80000F8B504460F46A07A4006400E002874D1D1
:10B810000025ACE01820684321680818407C012806
:10B820003CD10121182068432268101801740026B9
:10B830000CE018206843216808180830815D182042
:10B840006843226810188155701CC6B2082EF0D3C8
:10B8500000211820684322681018017418206843DA
:10B86000226810184174182068432268101841613A
:10B87000182068432268101881742C20684361687E
:10B880000818406A002809D018236B432268D01892
:10B890002C236B436268D218516A8847182068438A
:10B8A000216808184069FF21C94388425DD81820E3
:10B8B0006843216808184069C11918206843226844
:10B8C00010184161182068432168081841692C202C
:10B8D0006843626810188069814246D31820684323
:10B8E00021680818807C55283FD0552118206843CE
:10B8F000226810188174002624E03CE01820684378
:10B9000021680818805D2C21694362685118103144
:10B91000895D08401821694322685118885518200C
:10B92000684321680818805D2C21694362685118BA
:10B930000831895D084318216943226851188855E8
:10B94000701CC6B2082ED9D32C2068436168081831
:10B95000806A002809D018236B432268D0182C2352
:10B960006B436268D218916A8847681C85B2208947
:10B97000A84200DD4EE7F8BD01200149087070477C
:10B980008C00002010B50446002015F077FA02283C
:10B9900041D121480078002802D101201E490870B9
:10B9A0001D48007801281FD11B484078401C1A49C7
:10B9B000487021465A20FCF7C3FB17494978884252
:10B9C00029D800201449487008468078401C8870A7
:10B9D000084680780A2803D3002088700220087067
:10B9E000002015F07BFA16E00B480078022812D1EF
:10B9F00009484078401C0849487021467D20C00015
:10BA0000FCF79EFB04494978884204D8002002498B
:10BA1000487015F063FA10BD7600002000B587B0BD
:10BA2000002168460171042141710C4802904110C7
:10BA300003910B49049105910A480690FFF788FE8F
:10BA400001A815F0AFFA00F079FB00F00FF8002123
:10BA5000054809F0DFFD07B000BD0000FFFF1F0033
:10BA6000FFFFFF1FD5BC00000205000010B5FF203E
:10BA700002307249486000200872012008700020DE
:10BA80004872012088726E48FFF763FB6B496C486F
:10BA9000FFF788FB01216A48FFF7D8FB694867492F
:10BAA00048600020087201200870002048720120C0
:10BAB000887263481030FFF74CFB604960481030D3
:10BAC000FFF770FB01215E481030FFF7BFFB5D48B8
:10BAD000401E5A494860002008720120087000206A
:10BAE00048720120887256485030FFF732FB5349A4
:10BAF00053485030FFF756FB012151485030FFF7B3
:10BB0000A5FB5048C1384D4948600020087201200B
:10BB10000870002048720120887249484030FFF7C1
:10BB200018FB464946484030FFF73CFB012144489A
:10BB30004030FFF78BFBFF20123040494860002067
:10BB400008720120087000204872012088723C4869
:10BB50006030FFF7FEFA394939486030FFF722FBC1
:10BB6000012137486030FFF771FBFF202130334956
:10BB700048600020087201200870002048720120EF
:10BB800088722F48A030FFF7E4FA2C492C48A030E7
:10BB9000FFF708FB01212A48A030FFF757FB29488F
:10BBA0008F38264948600020087201200870002064
:10BBB0004872012088722248E030FFF7CAFA1F4914
:10BBC0001F48E030FFF7EEFA01211D48E030FFF793
:10BBD0003DFB1D481949486000200872012008708B
:10BBE000002048720120887215482030FFF7B1FA12
:10BBF000124913482030FFF7D5FA012110482030B0
:10BC0000FFF724FB1048CB300C4948600020087235
:10BC100001200870002048720120887208483030E6
:10BC2000FFF797FA054906483030FFF7BBFA0121C4
:10BC300003483030FFF70AFB10BD0000782A0020CF
:10BC4000105504400204000014070000F0B50B4634
:10BC5000144643600481002136E0002216E02C25C2
:10BC60004D4346687519AD5C18274F430668F619B1
:10BC7000B5542C254D4346687519AD5C18274F43C4
:10BC80000668F6190836B554551CEAB2082AE6D3F8
:10BC9000002518274F430668F619357418274F43B7
:10BCA0000668F619757418274F430668F619B574B7
:10BCB00018274F430668F619F57418274F4306688E
:10BCC000F61975614D1CA9B205898D42C5DC0025A8
:10BCD0008572F0BD70B50446606800F035FE05461B
:10BCE000E27A23460C332946094800F0F5FD09495C
:10BCF0006068884204D00749CB396068884206D121
:10BD0000E17AA28890B222460C3203F01FF870BD8F
:10BD10004C080020DF070000F8B5054600262C4639
:10BD2000002C2AD000BF03E00020A055701CC6B232
:10BD3000082EF9D304F01EFFC00008210840074672
:10BD400020688843384320606068C000C0080B4901
:10BD500009784907490F49070843606004F00AFF62
:10BD6000012801D1082000E0002007061F21090654
:10BD70000F406068884338436060F8BD7C00002055
:10BD8000F8B5054600262C46002C4FD000BF03E036
:10BD90000020A055701CC6B2082EF9D32448007BA1
:10BDA000002809D12088000A000220802088FF2175
:10BDB00009028843208015E004F0F0FF923000046F
:10BDC000070E2088000A00023843208004F0E6FFB6
:10BDD00092300002FF21090208400746208888436C
:10BDE000384320801248407B002809D16088000A2F
:10BDF000000260806088FF2109028843608015E0AE
:10BE000005F0D0F892300004070E6088000A0002A6
:10BE10003843608005F0C6F892300002FF21090225
:10BE2000084007466088884338436080F8BD0000BA
:10BE30003828002070B5054600262C46002C42D03C
:10BE400000BF03E00020A055701CC6B2082EF9D335
:10BE500005F0D6F8012817D11B480088401C80B295
:10BE600019490880032804DD002018490870164984
:10BE7000088031202070012060705920A0700820B7
:10BE8000E070002020711EE005F0BAF8022817D1FA
:10BE90000D480088401C80B20B490880032804DD4F
:10BEA00000200A49087008490880312020700120CC
:10BEB00060705920A0700820E0700120207102E01D
:10BEC00000200149088070BD7A000020D8000020C1
:10BED000FEB5054600260020019001F097FC0746BC
:10BEE00004F078FE0A210090FCF740F980B201903E
:10BEF0002C46002C3AD000BF03E00020A055701C57
:10BF0000C6B2082EF9D3FF21090260688843390CB4
:10BF10000902FF22120211400843606011026068AA
:10BF20008843390A090412021140084360606068BE
:10BF30000002000A3906090E09060843606004F091
:10BF400043FFFF2806DDFF210904206888434018CD
:10BF500020600BE004F038FF0004FF2109040840D2
:10BF6000009020688843009908432060FEBDFEB51C
:10BF70000546002600200190002704F025FC6421DE
:10BF80000090FCF7F3F880B20190002001F060FC13
:10BF900087B22C46002C1AD000BF03E00020A05529
:10BFA000701CC6B2082EF9D3FF210904206888430B
:10BFB00039120904FF22120411400843206020684E
:10BFC0000002000A3906090E090608432060FEBD7A
:10BFD000FFB581B004460F460025002600200090E2
:10BFE0002760039820810498E0600020207400BF3F
:10BFF0009DE01C206843216808586A0161688850E8
:10C000001C2068432168081880686A0161688918E3
:10C0100048601C2068432168081840686A0161680C
:10C02000891888601C20684321680818C0686A0164
:10C0300061688918C8601C20684321680818007C62
:10C040006A016168891808741C206843216808180F
:10C05000407C6A016168891848741C206843216823
:10C060000818807C6A016168891888831C206843ED
:10C0700021680818C07C6A016168891888740020EA
:10C080006A0161688918C8741C206843216808180F
:10C090004068002813D01C20684321680818C07C21
:10C0A000002805D1401E6A0161688918C8831AE01A
:10C0B0000020C0436A0161688918C88313E01C200E
:10C0C000684321680818C07C002805D000206A0158
:10C0D00061688918C88306E000206A0161688918D0
:10C0E000C88301200090002607E000216A016068F3
:10C0F000801814308155701CC6B269016068401800
:10C10000808BB042F1DC1C2068432168081840692C
:10C1100000280AD06B016268D218104614301C2324
:10C120006B432268D21851698847681CC5B22089C0
:10C13000A84200DD5DE7009805B0F0BD00B58BB00A
:10C1400068480790002108A801706846017608A891
:10C150004170002064498872082108A8C17000203D
:10C1600004E0002209A90A54411CC8B208A9C978F0
:10C170008142F6DC5D48FEF7ECFF06A95B48FFF75D
:10C1800011F85848401C0790002108A80170684623
:10C19000017608A84170002053498872082108A838
:10C1A000C170002004E0002209A90A54411CC8B251
:10C1B00008A9C9788142F6DC4C484030FEF7C9FF37
:10C1C00006A94A484030FEF7EDFF452000010790E0
:10C1D000002108A801706846017608A84170002077
:10C1E00041498872082108A8C170002004E000229B
:10C1F00009A90A54411CC8B208A9C9788142F6DCD1
:10C200003A485030FEF7A5FF06A938485030FEF7EF
:10C21000C9FF112040010790002108A8017068465D
:10C22000017608A8417000202F498872082108A8CB
:10C23000C170002004E0002209A90A54411CC8B2C0
:10C2400008A9C9788142F6DC28482030FEF781FF32
:10C2500006A926482030FEF7A5FF0B20C001079055
:10C26000002108A801706846017608A841700020E6
:10C270001D498872082108A8C170002004E000222E
:10C2800009A90A54411CC8B208A9C9788142F6DC40
:10C2900016486030FEF75DFF06A914486030FEF7CF
:10C2A00081FF1048A6300290002168460173017199
:10C2B000417381730821C173002004E0002204A9A6
:10C2C0000A54411CC8B26946C97B8142F6DC074862
:10C2D0001030FEF73EFF01A904481030FEF762FF60
:10C2E0000BB000BDEE060000782A00208055044007
:10C2F000F0B585B004460F4600250026207C400698
:10C30000400E55287ED100BF76E169016068401873
:10C31000807C002877D169016068401840686A0114
:10C32000616889188968884209D269016068401883
:10C330004068C0196A016168891848605AE169015A
:10C3400060684018C068AF49884208D869016068D1
:10C350004018C068401C6A0161688918C86069019A
:10C3600060684018C07C002821D1002607E0002129
:10C370006A016068801814308155701CC6B269016A
:10C3800060684018808BB042F1DC1C206843216853
:10C390000818406900280AD06B016268D21810465C
:10C3A00014301C236B432268D218516988476901F5
:10C3B000606840580090690160684018017C6846D8
:10C3C000017100214171690160684018017F684670
:10C3D0008171690160684018417C6846C17100261E
:10C3E00008E06901606840181430815D02A8815539
:10C3F000701CC6B2690160684018808BB042F0DCE6
:10C40000E06801E0FCE01DE0002806D06846E16835
:10C4100088476A0161688918C874690160684018B2
:10C42000C07C002804D16A01616889184860E1E095
:10C430006901606840184068C01B6A01616889181A
:10C440004860D7E069016068401880680028EED035
:10C45000690160684018C08B0028E8D069016068F5
:10C460004018C08B6A0161688918C968884207D181
:10C47000690160684018C08B6249C94388427DD118
:10C4800069016068401840686A01616889188968B4
:10C49000884209D26901606840184068C0196A0181
:10C4A000616889184860A5E000206A016168891800
:10C4B0004860690160684018C0685249884208D8DD
:10C4C000690160684018C068401C6A016168891889
:10C4D000C860002607E000216A01606880181430F7
:10C4E0008155701CC6B2690160684018808BB042EB
:10C4F000F1DC1C20684321680818406900280AD034
:10C500006B016268D218104614301C236B432268FA
:10C51000D2185169884769016068405800906901E4
:10C5200060684018017C6846017100214171690111
:10C5300060684018017F6846817169016068401831
:10C54000417C6846C171002608E0690160684018B6
:10C550001430815D02A88155701CC6B26901606803
:10C560004018808BB042F0DCE068002808D06846B4
:10C57000E16888476A016168891800E015E0C874BD
:10C58000690160684018C07C002804D16A016168B4
:10C59000891848602EE06901606840184068C01B37
:10C5A0006A0161688918486024E01C20684321689A
:10C5B0000818406800280FD00020C0436A01616855
:10C5C0008918C8831C2068432168081840686A01DC
:10C5D00061688918886008E000206A01616889182C
:10C5E000C8836A0161688918886000206A016168EF
:10C5F0008918C860681CC5B22089A84200DD84E69D
:10C6000005B0F0BD0000FFFF7CB500BF19212C482C
:10C610000078FBF795FD04462A4860432A4A8118B2
:10C62000002201200DF054F820460A2250436430C5
:10C63000001981B2002201200FF0BCF801200A226B
:10C6400062431219D1B20A22624312190090D0B289
:10C6500001231A4609F0F2FAFF220721002006F012
:10C6600081FF0120009001900B20604382B20B20DB
:10C67000604381B2002301200EF0B8FD6F206043BB
:10C6800081B201200FF03CFB1048604302460321B9
:10C6900001200BF097FD002505E0012128460BF055
:10C6A000CBFC681CC5B20F2DF7DB21460B22514392
:10C6B0006431C8B20FF08EFD0FF076FD7CBD000036
:10C6C00073000020672B0000A0860100FCB1010070
:10C6D000002005490870054908700549087005499A
:10C6E000087005490870704774000020750000202C
:10C6F000730000207200002071000020F0B589B0A6
:10C7000000BF00BF00BF00BF00BF00BF00BF00BF31
:10C7100000BF00BF5D4800783C2805DA5B48007820
:10C72000401C5A49087002E03C205849087057489C
:10C7300000781D2805DC56480078401C54490870D4
:10C740000BE053480078002802D15149087004E0FA
:10C750004F480078401E4E49087003214C4800782D
:10C76000FBF704FD4B4948430390052148480078F6
:10C77000FBF7E6FC0446032145480078FBF7F6FC8E
:10C780000B214843643080B20690414909788A0001
:10C7900088180621FBF7EAFCFF21F531484380B2F7
:10C7A000079003213A480078FBF7E0FC0B2148434F
:10C7B000643080B20890032135480078FBF7D6FC3E
:10C7C00035494843354940180490032130480078E2
:10C7D000FBF7CCFC0B2106464E4303212C48007886
:10C7E000FBF7C4FC0B2107464F4303212848007880
:10C7F000FBF7BCFC6F21484380B205900321012068
:10C80000039A0BF0DFFCE1B201200BF0A7FAE1B2D2
:10C8100001231846069A09F0EBFCFF21F531079831
:10C82000FBF7A4FCC0B20146029001200AF0C2F955
:10C830000022012008990EF0BDFF0022012004997A
:10C840000CF046FF012005990FF05AFA0120F9B2C9
:10C850000090F0B201231A46029009F0EFF9FF228E
:10C860000721002006F07EFE032109480078FBF72F
:10C870007DFC0B21484385B20120009000232A460D
:10C88000294601900EF0B2FC09B0F0BD7500002001
:10C8900074000020FCB10100672B0000A08601009D
:10C8A000002000BF06E00021044A1154044A11543C
:10C8B000411CC8B25A28F6DB704700004826002009
:10C8C000FC2600200348007A002801D10149487065
:10C8D00070470000580A0020FFB581B004460F469B
:10C8E0003D462089A8422DDD18206843216808189C
:10C8F000007C002826D1002609E00498815D1820DC
:10C9000068432268101808308155701CC6B2082E82
:10C91000F3D30121182068432268101841742C2099
:10C92000684361680818006A00280BD018236B431D
:10C930002268D218104608302C236B436268D21844
:10C94000116A884705B0F0BD01460720124BCA1A8C
:10C95000994211D008DCCA1FFA3A002A14D0102AD2
:10C960000CD01F2A14D10DE0322A0FD0C02A07D0D4
:10C97000C12A0DD100200DE001200BE0022009E0CA
:10C98000032007E0042005E0052003E0062001E085
:10C99000072000BF00BF70474103000010B50446E8
:10C9A0007D21C90061430846322103F0AFFE10BD6E
:10C9B000FF200B4908700020C0430A4908800A493B
:10C9C0000880FF2009490870094908700949087062
:10C9D0000020094908600949086009490860704752
:10C9E000580000205A0000205C0000205E0000205B
:10C9F0005F000020600000204C000020500000205C
:10CA000054000020014800687047000050000020DA
:10CA100001480068704700004C00002010B505492F
:10CA200009886522514308466421FBF79FFB80B2C9
:10CA300010BD00005A000020014800787047000037
:10CA40005F00002001480078704700005800002077
:10CA500010B510F041FB01282CD100F063F8012043
:10CA600000F066F803F0B6FE044600F043F804F068
:10CA70008FF8044600F04AF804F0E4FA012805D1E2
:10CA800000F03EF8012000F047F805E0002000F03B
:10CA900037F8002000F040F80020134908601348E0
:10CAA0000068134988421ED210480068801C0F4954
:10CAB000086018E000200D4908600B4800680C4928
:10CAC000884204D208480068801C0749086000209A
:10CAD00000F028F8012000F02BF8002000F00AF800
:10CAE000002000F013F810BD500000204C00002082
:10CAF000FFFFFF7F01490880704700005A000020B7
:10CB000001490870704700005F000020014908805B
:10CB1000704700005C000020014908707047000069
:10CB20006000002001490870704700005800002094
:10CB300001490870704700005E0000200021014A92
:10CB40001171704700600040002201494A7570472A
:10CB500000600040002201494A76704700600040B2
:10CB60000021014A11727047006000400021014A13
:10CB700011737047006000400021014A1174704732
:10CB8000006000400021014A1175704700600040BC
:10CB90000021014A117670470060004000220149DF
:10CBA0004A73704700600040002201494A74704790
:10CBB0000060004010B51C4C1C49206888421ED102
:10CBC00006221B49201DFBF776FB002817D11122F6
:10CBD000184920460A30FBF76EFB00280FD10622C9
:10CBE000154920461B30FBF766FB002807D10622BB
:10CBF000124920462130FBF75EFB00280DD000F0E3
:10CC00004BFE0A480E490860074814F098FA0C4A8F
:10CC10002821054814F0BEFA04E0282221460848DD
:10CC2000FBF725FB10BD0000000250007AA7A55AB3
:10CC3000290700202F070020230700201D070020C0
:10CC4000842E00200020084908700849087001203F
:10CC5000074908700020074908700748074908601D
:10CC600000200749087070470B0700200A070020C2
:10CC70000D070020120700202506000040070020B5
:10CC80001C07002070B5044600BF91206043054694
:10CC90000A212846FBF754FA0546284670BD0000D5
:10CCA00070B5A8B0054600240026A0216846FBF711
:10CCB000F7FA00F061FC1E490A68142169435050DC
:10CCC00000211B480268142068431018416018486E
:10CCD00002681420684310188160154840680028D5
:10CCE00024D000BF17E06006060E282E00D316E001
:10CCF0000F480168142060430858B1006A4650503C
:10CD00000B4801681420604308184168701C8000BB
:10CD10001150601CC4B20648007AA042E3DC00BF98
:10CD200062000348694643680220984728B070BDF6
:10CD3000FC2E002030B5A9B000240025A02101A8B8
:10CD4000FBF7AEFA00BF25E06006050E00F014FC0C
:10CD50001F490A6814216143505000211C48026891
:10CD60001420604310184160194802681420604381
:10CD700010188160282D0BD21548016814206043DB
:10CD80000858A90001AA50500021681C80001150C9
:10CD9000601CC4B20E48007AA042D5DC0C48406842
:10CDA000002813D00A48007A4000282806D30848F3
:10CDB000282201A943680220984707E00448007A26
:10CDC0004200034801A943680220984729B030BDBA
:10CDD000FC2E002010B510F07FF901287ED1FFF75E
:10CDE00017FE5549884216D20F2054494871887160
:10CDF00008468078002801D1052048704F48807887
:10CE0000052802D100204D49487000204B49087286
:10CE10004872087035E0FA204849487188714849DD
:10CE2000088803F0FFFD4648807800280CD143496C
:10CE3000087008464079C87008468079087100205B
:10CE40008870487048721CE001203C490870084610
:10CE5000407A022805D1012048720020C87008716C
:10CE60000FE03648407A00280BD10220334948723F
:10CE700008464078887008464079C870084680792E
:10CE800008712E4880782D494978884213DD0020AA
:10CE90002A49C87008460079401C08710846007984
:10CEA0008979884222DB002024490871084680786D
:10CEB000401E88701AE021488078204949788842CD
:10CEC00014DA00201D4908710846C078401CC8705B
:10CED0000846C0784979884208DB00E01EE000205F
:10CEE0001649C87008468078401C887014488078BD
:10CEF000002803D10120114908721BE01048008866
:10CF0000732803DB02200D49087213E00C480088E7
:10CF100070280FDC0020094908720BE00020074947
:10CF2000087008464079C87008468079087100206A
:10CF30000872487210BD0000B80B0000B409002050
:10CF4000800000200020044988704870C870087173
:10CF50000872487270470000B4090020002006499A
:10CF600008808870054988704870FA20C870087178
:10CF7000002008724872704780000020B409002029
:10CF800070B503F057FC044603F066FC054610F04C
:10CF9000A3F801282ED105211A48FEF7CDF855280F
:10CFA00004D1002018498870088027E0012D04D1A1
:10CFB000002015498870088020E0012012498870FF
:10CFC0001248844202DB201A84B200E000240A21C5
:10CFD0002046FBF7CBF8052901DB601D84B20C4825
:10CFE000844200DD04460A212046FBF7BFF80649CB
:10CFF000088003E00020044988700880FFF7EAFEFB
:10D0000070BD00004C08002080000020AA0A00002B
:10D01000C60700001CB500200090019000F0ACFA9B
:10D020000B49086000200B49096808600A4800683D
:10D0300000280CD00749096808680A21FBF780F826
:10D040000090012269460520034B1B6898471CBDD0
:10D05000DC070020D0070020D80700200020084966
:10D06000488008490880084908800849087008492C
:10D0700088720849088048800120087170470000C4
:10D08000300000202000002022000020240000208A
:10D090003008002028000020F8B503F0ADFB07465B
:10D0A00003F0BCFB0090FFF7CDFC012860D1052107
:10D0B000C548FEF741F8552802D00098012807D14D
:10D0C0000020C2490870C2490880C249887256E0EF
:10D0D000BE480078002810D10120BC4908703D46A8
:10D0E0002846E917890F091889030D0CBA488542AB
:10D0F00000DD0546B648058041E0B648807A40002C
:10D10000B4490F520846867A0EE07000B1490D5AB4
:10D11000701E4000085A7100AE4A5052701E400006
:10D1200011460D52701EC6B2002E08DD7000A949CE
:10D13000095A701E4000A74A105A8142E5DBA548F3
:10D14000807A401CA34988720846807A052816DB3D
:10D15000002088720846C5882846E917890F0918F3
:10D160008D109D48854200DD05469948058006E002
:10D17000002096490870964908809649887294481C
:10D18000058896480088A84257DA94480088281AEB
:10D1900084B292480079012827D190484088A04263
:10D1A0000BDA8E4840880A308C494880084640880F
:10D1B000A04204DD0846448001E088484480874856
:10D1C000448803212046FAF7D1FF84B2192C00DAF3
:10D1D0001924824800880019804908800846008880
:10D1E000A84201DD08460580CDE07C48408814282F
:10D1F00005DD7A48408814387849488002E00020EC
:10D20000764948807548448803212046FAF7AEFFE6
:10D2100084B2192C03DA012070490871B3E06F4819
:10D220000088A04205DD6D480088001B6B4908801E
:10D23000A9E0002069490880A5E068480088A84264
:10D2400059DD66480088401B84B264480079012893
:10D2500027D162484088142805DD6048408814388A
:10D260005E49488002E000205C4948805B48448871
:10D2700003212046FAF77AFF84B2192C03DA022040
:10D28000564908717FE055480088001953490880C5
:10D29000084600885049884275DD08464F49088095
:10D2A00071E04E484088A0420BDA4C4840880A3072
:10D2B0004A49488008464088A04204DD0846448028
:10D2C00001E0464844804548448803212046FAF757
:10D2D0004DFF84B2192C00DA19244048008829191E
:10D2E000884202DA3D4805804DE03C480088001B3A
:10D2F0003A49088047E03948448803212046FAF734
:10D3000035FF84B2192C3EDD34484088142805DDF1
:10D310003248408814383149488002E000202F49C3
:10D3200048802E48448803212046FAF71FFF84B224
:10D330002A480079012813D1192C03DA0220274941
:10D34000087120E025480088001924490880084613
:10D3500000882149884216DD08462049088012E0ED
:10D36000192C03DA01201D4908710CE01B480088C4
:10D37000A04205DD19480088001B1849088002E01A
:10D3800000201649088016480088502804DC1348FD
:10D3900000881349088016E0104800881049098861
:10D3A000884204DD0D4800880D4908800BE00B48D9
:10D3B00000880B490988081A84B2502C03DB0748FF
:10D3C000008807490880F8BD4C0800202400002090
:10D3D0002000002030080020E02E0000280000205F
:10D3E0002200002010B5044664204443A1212046B9
:10D3F000FAF7A6FE0446204610BD000010B5012035
:10D400000F49087000200F49096808600D49096834
:10D4100048600C490968886000F07EF9FFF7FAFD62
:10D42000FFF788FC08480068002807D0012205485B
:10D43000016808310020044B1B68984710BD0000AC
:10D44000A9070020A4070020A007002010B5184855
:10D4500000681849884229D117480068002804D07C
:10D46000154800688047154908701548006800286D
:10D4700004D01348006880471249087012480068B9
:10D48000002804D0104800688047104908801048E0
:10D490000068002805D00E48006880470D490880C4
:10D4A00002E00D480B49088000F078F810BD00003C
:10D4B000B40700207856341290070020A8070020F7
:10D4C00094070020AA07002098070020AC0700203E
:10D4D0009C070020AE0700201027000010B5002395
:10D4E000174C2360174C2370174C2370174C237074
:10D4F000174C2380174C2380174C2370174C13684C
:10D500002360174C53682360164C93682360164CB5
:10D51000D3682360154C1369236000280CD0144B8A
:10D520001860134C0B682468A3600023104C246817
:10D5300023600F4C246863600E4B014C236010BDC8
:10D54000B4070020B0070020A8070020AA07002089
:10D55000AC070020AE070020A9070020900700209C
:10D5600094070020980700209C070020A0070020B7
:10D57000A4070020785634120548006805498842FF
:10D5800003D105480068806870470020C043FBE76E
:10D59000B407002078563412A407002070B5002488
:10D5A000002500263048007801285CD12F480078FB
:10D5B000002858D12E480078012854D12D480588DC
:10D5C0002D490988694308462C49FAF7B9FD85B207
:10D5D000E1200001854207D8192169430846092145
:10D5E000FAF7AEFD044600E0244C254800680068C8
:10D5F000001923490968086021480068006820492B
:10D6000009684968884207D31D48006800681C49BA
:10D6100009684968461A0AE019480068406800210C
:10D62000C943081A1649096809684018461C154874
:10D63000864218D3344601462046FAF781FD044657
:10D640000F48006841680F48604308180C49096892
:10D65000486001200C49087009480068806800197A
:10D6600007490968886070BDA8070020A907002045
:10D67000AA070020AC070020AE07002010270000FA
:10D68000A4070020A0860100B007002000220C4B58
:10D690001A600C4B0A681A600B4B4A681A600B4BF5
:10D6A0008A681A600A4BCA681A600A4B0A691A60CB
:10D6B000002801D0084A1060084A014B1A607047E0
:10D6C000B40700209007002094070020980700204E
:10D6D0009C070020A0070020A407002078563412E1
:10D6E00010B50A48006800280ED0094800780128C3
:10D6F0000AD1002006490870012206480168083155
:10D700000020024B1B68984710BD0000A0070020B6
:10D71000B0070020A40700201CB500200090019055
:10D720000024FFF729FF04460E480068046000202B
:10D730000C49096848600B49096888600A48006814
:10D7400000280DD007480068006800900548006870
:10D7500040680190022269460120034B1B689847EC
:10D760001CBD0000B8070020BC070020F8B5054626
:10D770000C4616460027002D17D00E480560FFF70F
:10D78000FBFE07462068B84203D90A4800680760D4
:10D7900003E008492068096808600649606809686C
:10D7A00048600449A0680968C8600348066000F042
:10D7B00005F8F8BDB8070020BC07002070B50024AC
:10D7C0000025FFF7D9FE04460F4800680068A04214
:10D7D00000D903E00C4800680068251A0A48006870
:10D7E00040684019084909688860074800688068EF
:10D7F00005490968C968884205D903480068C068B6
:10D8000001490968886070BDB807002001480068B8
:10D8100080687047B8070020002801D0024A1060D5
:10D82000024A116070470000B8070020BC070020C2
:10D830000549002005E00A1D135C044A1354421CEC
:10D84000D0B22028F7DB704700065000B02E002031
:10D8500001461048026814204843101882680D4899
:10D860000368142048431818C06882420BD909483D
:10D870000268142048431018C26806480368142040
:10D88000484318188260034802681420484310185F
:10D8900080687047FC2E00200021002005E01A4A15
:10D8A000135C1A4A1354421CD0B20628F7DB11212C
:10D8B000002006E0164A135C144A921D1354421CC1
:10D8C000D0B28842F6DB002006E0124A135C0F4A11
:10D8D00017321354421CD0B20628F6DB002006E0B3
:10D8E0000D4A135C094A1D321354421CD0B206285B
:10D8F000F6DB002005E00023044A23321354421CC7
:10D90000D0B20128F7DB704729070020882E0020BD
:10D910002F070020230700201D07002038B50446EC
:10D9200000200090009401226946052000F068FC68
:10D9300038BD000008B5002000900122694606208D
:10D9400000F01EFC684600780D4908736846407870
:10D9500048730846007B0B4948730948407B88732D
:10D960000748807BC8730648C07B08740020087392
:10D9700005490860054908600549087008BD0000B0
:10D9800038280020C00900208400002088000020E2
:10D990008C00002008B50020009001226946062076
:10D9A00000F0EEFB6846007810490873684640783E
:10D9B000487300200E4908604860087248728872F7
:10D9C0000A48007B48730948407B88730748807B7E
:10D9D000C8730648C07B08740020087305490860B6
:10D9E000054908600549087008BD00003828002076
:10D9F000C009002084000020880000208C00002046
:10DA000038B500240025002000900121FE48FDF7D4
:10DA100093FB55280AD002F063FFFC49487302F0DB
:10DA200073FFFA4988730120087308E0F848007B07
:10DA3000F6494873F648407B887300200873062136
:10DA4000F148FDF779FB552820D002F091FF00281E
:10DA500008D002F08DFF401C002803D00120EB49C4
:10DA6000087502E00020E949087502F063FF00280C
:10DA700008D002F05FFF401C002803D00120E349DA
:10DA8000C87407E00020E149C87403E00020DF49C2
:10DA9000C8740875DD48407B002833D1DD48006834
:10DAA000DD49884208D8DB480068401CD949086035
:10DAB0000020D649487376E0D448407C012802D142
:10DAC0000020D44908600020D0494874D048007B29
:10DAD000022812D0CE48007B03280ED00121CA486C
:10DAE000FDF72AFB552803D00320C84948735AE0A4
:10DAF000C748007BC549487355E0C548007BC3490A
:10DB0000487350E0C148407B012832D1BF48407C77
:10DB1000002801D1BF4908600120BC494874BD48B4
:10DB20000068BD49884208D8BA480068401CB94915
:10DB300008600120B549487335E0B548007B0228EC
:10DB400012D0B348007B03280ED00121AE48FDF768
:10DB5000F3FA552803D00320AC49487323E0AC48BE
:10DB6000007BAA4948731EE0A948007BA749487377
:10DB700019E0A648407B022803D10020A54908608F
:10DB800011E0A248407B032806D10020A14908608B
:10DB900003209E49487306E000209E4908609C4887
:10DBA000007B9A4948739948807B002833D19B4871
:10DBB00000689949884208D898480068401C9749ED
:10DBC000086000209149887386E09048807C012895
:10DBD00002D100209149086000208C4988748C484B
:10DBE000407B022812D08A48407B03280ED00121B6
:10DBF0008548FDF7A1FA552803D00320834988738F
:10DC00006AE08348407B8149887365E08048407BB7
:10DC10007E49887360E07D48807B012832D17B4853
:10DC2000807C002801D17D490860012077498874F3
:10DC30007A4800687849884208D878480068401CCB
:10DC40007649086001207149887345E07048407B3F
:10DC5000022812D06E48407B03280ED001216A486A
:10DC6000FDF76AFA552803D003206849887333E02A
:10DC70006748407B654988732EE06548407B63496F
:10DC8000887329E06148807B022813D10020634912
:10DC9000086002F06DFE002808D002F069FE401C0A
:10DCA000002803D001205949087515E00020574984
:10DCB000087511E05548807B032806D1002057499C
:10DCC000086003205149887306E00020534908602A
:10DCD0004F48007B4D4988734C48407B4C49097B39
:10DCE000884205D14948807B4949497B88424FD0C9
:10DCF0004648407B4649097B884202D0012043497F
:10DD0000C8734248807B4249497B884202D0012047
:10DD10003E4908743D48407B022803D03B48407B85
:10DD2000032816D13948407B3949097B884210D0F5
:10DD30003648407B364908730846017B68460170C7
:10DD40003348417B6846417001226946062000F055
:10DD500057FA2E48807B022803D02C48807B03286A
:10DD600016D12A48807B2A49497B884210D027480F
:10DD7000807B274948730846017B68460170244828
:10DD8000417B6846417001226946062000F038FA5E
:10DD900002F0B0FD044602F0C3FD0546FEF752FE58
:10DDA000012878D101211848FDF7C6F9552807D177
:10DDB0000020164908724872086048608872B7E00F
:10DDC000FF2C01D0FF2D75D1FF2C3CD1FF2D3AD077
:10DDD00000200E490872012048721148086011485D
:10DDE0006843486048686621FAF7AAF9074948601D
:10DDF000084640680C49884202D9084603494860F1
:10DE000003F0C0F8112811E04C080020C0090020E0
:10DE100038280020840000207017000088000020AF
:10DE2000DE030000BE0A0000AC26000003DB03F0A6
:10DE3000A9F8192803DD01205F49887278E00020E5
:10DE40005D49887274E0FF2C2BD0FF2D29D1012071
:10DE50005949087200204872584848605848604341
:10DE6000086008686621FAF76BF9534908600846AC
:10DE700000685449884202D908464F49086002F0B8
:10DE80007DFF112803DB02F079FF192805DD012051
:10DE9000494988724CE086E00CE0002046498872CF
:10DEA00046E048484449086048600020887208728B
:10DEB00048723DE001204049087248724048604382
:10DEC000086008686621FAF73BF93B490860084694
:10DED00000683C49884202D90846374908603848FA
:10DEE00068433549486048686621FAF729F932499C
:10DEF0004860084640683349884202D908462E499E
:10DF0000486002F03BFF11280BDB02F037FF1928B5
:10DF100007DC03F037F8112803DB03F033F8192886
:10DF200003DD01202449887202E000202249887222
:10DF30002148407B002802D11F49C87315E01E48C4
:10DF4000407B012802D11C49C8730EE01A48407B6F
:10DF5000022802D11849C87307E01748407B0328FC
:10DF600003D11549C873174808601348807B0028FF
:10DF700002D1114908741DE00F48807B012802D1AD
:10DF80000D49087416E00C48807B022802D10A492A
:10DF900008740FE00848807B03280BD106490874F9
:10DFA0000848486006E0002003490872487208608B
:10DFB0004860887238BD0000C0090020DE03000000
:10DFC000BE0A0000AC260000FFB583B006460D4631
:10DFD000174600240020029000BF142078438019C7
:10DFE0000190002E57D00198002854D02B4806608D
:10DFF0002A49069848600846077200BF45E0FFF7C7
:10E00000BBFA0290200129580298814204D82001CD
:10E010002858401C002806D1204902980A6814217B
:10E020006143505006E0200129581C480268142022
:10E0300060431150200140194068401C002807D15E
:10E04000002116480268142060431018416008E05F
:10E0500020014019416811480268142060431018DB
:10E0600041602001401981680C4802681420604317
:10E070001018C16020014019017B08480268142073
:10E08000604310180161601CC4B20448007AA042C9
:10E09000B5DC00F005F807B0F0BD0000FC2E002054
:10E0A00070B5002400250026FFF766FA054600BF7C
:10E0B0004EE02A480168142060430858A84239D825
:10E0C000264801681420604308582E1A2348016826
:10E0D0001420604308184068811920480268142001
:10E0E0006043101881601D480168142060430818BF
:10E0F00081681A480268142060431018C068814281
:10E1000024D91648016814206043081800690028C3
:10E1100003D02046FEF7C4FD18E010480168142023
:10E1200060430818C1680D48026814206043101845
:10E1300081600BE0094801681420604308184068BA
:10E1400006490A681421614351188860601CC4B2F2
:10E150000248007AA042ACDC70BD0000FC2E00201A
:10E1600010B500BF14244C432318002805D0002B01
:10E1700003D0024C20606260217210BDFC2E002092
:10E18000F8B505460E4614462B0012F013FB0705A2
:10E19000131A3131212931001748FAF7DFFC1749EA
:10E1A00008701548FAF794F807466421F9F7C8FF94
:10E1B00030601EE0A004020C31462020FAF7C8FDB2
:10E1C00017E0A004020C31466020FAF7C1FD10E010
:10E1D000A004020C3146FF202130FAF7B9FD08E017
:10E1E0006004020C3146FF204130FAF7B1FD00E037
:10E1F00000BF00BF0020F8BD2A280020C500002075
:10E2000070B505460E4614462B0012F0D3FA0705EA
:10E210001D243A3A2B323A003068002802D1FAF72E
:10E220003BFB10E064223168514308461649FAF777
:10E2300059F8002015490870012264211248FAF7A4
:10E24000F5FD124908701DE0A004020C31462020A3
:10E25000FAF73CFF16E0A004020C31466020FAF702
:10E2600035FF0FE0A2B23146FF202130FAF72EFF32
:10E2700008E06004020C3146FF204130FAF726FF27
:10E2800000E000BF00BF70BD1C280020C4000020BB
:10E2900000B5AFB050211BA8FAF702F800201A9081
:10E2A000142115A8F9F7FCFF002012901390149088
:10E2B0001190402101A8F9F7F3FF00200090484990
:10E2C000086001221BA9FFF75BFF1B98401C002878
:10E2D00001D11A9001E01B981A90424815904248CB
:10E2E000169042481790002018904148199015AA9E
:10E2F0001AA94048FFF7F2F802221CA90120FFF7F3
:10E300003FFF1C98401C002801D1129001E01C988E
:10E3100012901C98401C002801D1139001E01D9818
:10E3200013903548149012A93448199AFFF71EFA31
:10E3300008221EA90220FFF723FF1E98401C002878
:10E3400001D1019001E01E9801901F9802902C4885
:10E350000390012069460874801E059029490791A1
:10E36000012101A80177881E099026490B910121FE
:10E3700009A80173881E0D9022490F9101210DA853
:10E380000173042201A92048199BFFF71DFE0122F9
:10E390001BA90520FFF7F4FE1B98401C002807D19D
:10E3A00001201A498860012208310520FFF728FF63
:10E3B00001221BA90620FFF7E3FE1B98401C002842
:10E3C00008D100216846017041700122694606208B
:10E3D000FFF716FF0E48024908602FB000BD00008D
:10E3E000C800002045CA000039CA00001DCA00004C
:10E3F00001E20000B027002076841E00BC27002028
:10E400000F2700009F860100CC270020382800201D
:10E41000A33AA55A00B585B014216846F9F740FF24
:10E4200000200F4908600F4800900F4801900F48E6
:10E430000290002003900E48049069460D48FFF7B3
:10E4400025F90D480499FFF7E7F904210B48049AD0
:10E45000FFF786FE0A480249086005B000BD0000CB
:10E46000C800002045CA000039CA00001DCA0000CB
:10E4700001E20000B0270020BC270020CC270020AC
:10E48000A33AA55A00200C4908800C4908800C4981
:10E49000088001200B49087000200B4908730B49C4
:10E4A00008804880012008710020074948800880C2
:10E4B0000749086070470000380000203A0000203B
:10E4C00040000020420000203C08002044000020C2
:10E4D0003C000020F8B502F0C9F9064602F0D0F978
:10E4E0000746FEF7AFFA012865D10521AB48FCF7D6
:10E4F00023FE552807D10020A9490870A9490880A2
:10E50000A94988805FE0012F07D10020A449087045
:10E51000A4490880A449888055E0A14800780028D3
:10E5200008D101209E49087035460A2068439D495C
:10E53000088048E09C48007B42009B48801D865232
:10E54000801F047B11E061009748801D455A601EC2
:10E5500041009548801D415A62008152601E410071
:10E560009148801D4552601EC4B2002C0ADD610036
:10E570008D48801D415A601E42008B48801D805A84
:10E580008142E0DB8848007B401C874908730846CD
:10E59000007B032807DB00200873084605890A2052
:10E5A0006843804908807F4800887F49888001202F
:10E5B0007B49087007E00020794908707949088094
:10E5C00079490873888077480088784908607448DA
:10E5D0000078002815D0084600686C21484373492C
:10E5E0000860642171480068F9F7AAFD6F49086066
:10E5F000084600686E49884206D908466B4908609B
:10E6000002E0002069490860684800686949098893
:10E61000884203D2654800680F2804D26348008806
:10E62000644908800AE06348008860490968401A24
:10E630000F2803D35D4800885E4908805A48008847
:10E64000401C59490880084600880A282CDB002015
:10E6500008805948008857490988884203DA012010
:10E660005649087108E05448008852490988884290
:10E6700002DD02205149087150480079012840D13B
:10E680004C4800884C49098888420DDB494801887C
:10E6900049480088FF309130814206DD46480088B5
:10E6A000FF3073304449088077E04248018842488F
:10E6B00000889630814205DD3F48008878303E4929
:10E6C00008806AE03B4801883B480088323081423C
:10E6D00005DD394800881E30374908805DE035483F
:10E6E0000188354800880A30814205DD32480088BB
:10E6F0000A303149088050E02E4800882E490880B1
:10E700004BE02E480079022847D12A4800882A4940
:10E710000988884239DA27480088FF309130264935
:10E720000988884206DA24480088FF38733822496D
:10E7300008802AE01F48008896301F4909888842CF
:10E7400005DA1D48008878381B4908801DE0194803
:10E750000088323018490988884205DA164800884E
:10E760001E381549088010E0124800880A30124906
:10E770000988884205DA104800880A380E4908805E
:10E7800003E00C4800880C4908800B4800880849C1
:10E79000884202DB084608490880F8BD4C08002082
:10E7A00042000020380000203C0800203C000020EF
:10E7B000C6070000400000203A000020440000206E
:10E7C00000200849088008490880084908804880D6
:10E7D000012008710020064948800880054908602A
:10E7E000704700003A000020400000204400002054
:10E7F0003C0800203C000020002004490870044927
:10E800000870002103480176704700008D00002049
:10E810008E000020380A002070B500250024FEF785
:10E8200011F9012863D103213448FCF785FC5528F0
:10E8300008D100203249087032490870002132485E
:10E84000017659E02F480078002807D102F0AEF891
:10E850002B49087001202B4908704DE001202949FF
:10E86000087002F0A3F82849097E8900264A603A18
:10E8700050502548047E10E0A000234960390D5C0B
:10E88000601E80000858A1001F4A603A5050601E68
:10E89000800011460D50601EC4B2002C0ADDA0009D
:10E8A000194960390958601E8000174A603A1058AB
:10E8B0008142E1D31448007E401CC1B21248017667
:10E8C000007E1E2818DB00210F48017601466039C2
:10E8D000896B0246603AD26B89180246603A126C24
:10E8E00088180321F9F72CFC0549087004E0002082
:10E8F000034908700349087070BD00004C080020EF
:10E900008D0000208E000020380A0020F0B5A9B04C
:10E9100004460E460025002700202890A0216846C6
:10E92000F9F7BEFCFEF728FE26490A681421614368
:10E93000505024480168142060430818C068B04251
:10E940000CD220480168142060430818C1681D4893
:10E950000268142060431018416005E019480168FE
:10E96000142060430818466016484068002826D0E6
:10E97000002517E06806070E282F00D316E011487F
:10E980000168142068430858B9006A4650500D4881
:10E9900001681420684308184168781C80001150F1
:10E9A000681CC5B20748007AA842E3DC00BF6A00D1
:10E9B0000448694643680220984701202890289817
:10E9C00029B0F0BDFC2E002010B500F0F9FD00F0DC
:10E9D000D7F810F00FFE00F00DFB00F001F810BDAD
:10E9E00070B541480078912800D070BD00F0BEF8A5
:10E9F000012876D13D4800883D4908800846807846
:10EA0000F021884320303A49887008468078000910
:10EA100000013549097A0907090F0843344988700C
:10EA20003148807A401E3049887208460089401C6F
:10EA3000088108460089C988884216DA08202C49CE
:10EA4000887200240EE0284841882848001D415C57
:10EA50002748C01C015524484088401C2249488052
:10EA6000601CC4B2072CEEDB2DE01F4800891E4954
:10EA7000C98888421CD11C4800791B498978401AF2
:10EA8000C5B2681C1A49887200240EE016484188F5
:10EA90001648001D415C1648C01C015512484088AC
:10EAA000401C11494880601CC4B2AC42EEDB0AE055
:10EAB00000F012FD00200C4908700C49088809215B
:10EAC00000F0B8F991E7012000F0C8FC084A917AFB
:10EAD0001088921C00F070F905490888002100F0A8
:10EAE000C1F800BF81E70000382C0020D42B0020A3
:10EAF000642B00201B49097E002932D01949897EE8
:10EB00000C225143174A515A174A118000200CE039
:10EB10001449897E0C225143124A8918891C0A5CC7
:10EB20001149891C0A54411CC8B20828F0DB0D4960
:10EB3000897E0C2251430B4A8918897A0A4A9172BC
:10EB40000121D1720749097E491E064A11761146F4
:10EB5000897E491C91761146897E022901DB0021BC
:10EB600091767047302B0020582B00200349487BBA
:10EB7000012802D10021014A51737047482C00201E
:10EB800010B533484068002861D13148007B03004C
:10EB900011F010FE07590512212E3D4A59002D484B
:10EBA0000078002807D000202A4908702A490888E0
:10EBB000012100F03FF947E026480078002809D0FD
:10EBC00000202449087025494A8808880123091D26
:10EBD00000F040F938E01F480078002807D00020F6
:10EBE0001C4908701C490888022100F023F92BE019
:10EBF00018480078002809D00020164908701749E5
:10EC00004A8808880923091D00F024F91CE01148EE
:10EC10000078002807D000200E4908700E490888A7
:10EC2000092100F007F90FE00A480078002809D010
:10EC300000200849087009494A8808880323091DEB
:10EC400000F008F900E000BF00BF00F045FC10BD77
:10EC5000482C0020382C0020D42B0020702B0020C2
:10EC60007047000070B504460D4634480088A04245
:10EC700063D1002D61D13248007822284ED004DCC7
:10EC800020283DD0212856D141E0902802D091285B
:10EC900051D115E02A48C08801280AD1002028490E
:10ECA000087000F019FC27490888002100F0C2F81C
:10ECB00005E0032000F0D2FBA020214908703BE0D2
:10ECC0001F4800891E49C98888420AD100201C4972
:10ECD000087000F001FC1B490888002100F0AAF828
:10ECE0000DE01748807A002806D000F0F5FB1449A3
:10ECF000087B00F095FB02E0032000F0AFFB1BE077
:10ED0000062000F0ABFB11200D49087014E006202E
:10ED100000F0A4FB11200A4908700DE0002008490A
:10ED2000087000F0D9FB08494A8808880923091DA2
:10ED300000F090F800E000BF00BF70BD4C2B002039
:10ED4000382C0020D42B0020702B002070B50346F7
:10ED5000184C247E022C00DB70BD164C647E0C2502
:10ED60006C43144D2B5300200AE0155C114C647E5B
:10ED70000C2674430F4EA419A41C2554441CE0B265
:10ED80008842F2D30B4C647E0C267443094EA419BE
:10ED9000A1723446247E641C35462C762C46647E53
:10EDA000641C6C762C46647E022C01DB00246C769D
:10EDB00000BFD1E7302B0020F0B585B007460D46E7
:10EDC00016461A480780002406E031781748801C50
:10EDD0000155761C601CC4B2AC42F6DB2C4605E043
:10EDE000AA211248801C0155601CC4B2082CF7DB14
:10EDF0000E480088019008216846C17200214172C6
:10EE000001720170002406E00848801C015D03A81F
:10EE10000155601CC4B2082CF6DB69460448FCF7B7
:10EE20009CFA01200149887205B0F0BD4C2B0020EE
:10EE30009055044070B504460D462946204610F012
:10EE4000FBFA70BD70B504460D462946204610F009
:10EE500001FB70BDF8B504460D4616461F463B46FD
:10EE600032462946204610F0F6FAF8BDF8B50746B6
:10EE70000E4615465C480078002804D00921384623
:10EE8000FFF7D8FFF8BD002D01D0602D04DD09216A
:10EE90003846FFF7CFFFF5E7544807804580002448
:10EEA00006E031785148001D0155761C601CC4B243
:10EEB000AC42F6DB00204C49487008468580FF20B4
:10EEC00088727F2008730846808808282EDA01207F
:10EED000C88008468088488001200881434800880F
:10EEE0004349088008468078F0218843404988706B
:10EEF00008468078000900013B4909790907090F94
:10EF000008433B49887038480079401C88720024C7
:10EF100007E03648001D015D3548C01C0155601CE6
:10EF2000C4B231488088A042F3DC4AE00721681C63
:10EF3000F9F71CF9002907D0072128460830F9F70E
:10EF400015F92949C88005E00721681CF9F70EF971
:10EF50002549C8800620244948800120088123488B
:10EF600000882349088008468078F02188431030C3
:10EF70001F49887008468078000900011A4989886D
:10EF80000905090F08431A49887008464088FF217F
:10EF900009028843144989880902FF22120211409C
:10EFA00008431349488008208872002407E00F486E
:10EFB000001D015D0E48001D0155601CC4B2062CE9
:10EFC000F5DB012000F04AFA094A917A1088921C78
:10EFD000FFF7F2FE902004490870054908880021D7
:10EFE000FFF740FE00BF4DE7382C0020D42B002057
:10EFF000642B002010B5FFF77DFD1448C07A00286F
:10F0000022D0124880780009002806D0012807D0B5
:10F0100002280AD0032810D10CE000F0A7F90FE075
:10F0200000F09EF800F066FA0AE000F011F800F037
:10F0300061FA05E000F000F902E0FFF711FE00BF01
:10F0400000BF00200149C87210BD0000582B0020ED
:10F0500010B53F480078112800D010BD3D48008809
:10F060003D49884200D0F8E73A4880780007000F11
:10F070003749097A0907090F88420CD00020344922
:10F08000087000F029FA35494A8808880423091DC8
:10F09000FFF7E0FEE1E72E480089401C2C4908817B
:10F0A0000846807A401E887208460089C9888842CE
:10F0B0001BDA2848807A082800D0CEE700240EE02A
:10F0C0002448C01C015D224842882448001D815408
:10F0D0001F484088401C1E494880601CC4B2072C51
:10F0E000EEDB062000F0BAF930E0194880881849B4
:10F0F0004988401A1749897A884203DA1548807A84
:10F10000082800D0A9E700240EE01248C01C015DC9
:10F110000F4842881148001D8154601CC4B20C483D
:10F120004088401C0A494880094840880849898825
:10F130008842EADB00200649087000F0CDF9074953
:10F140004A8808880023091DFFF784FE00BF84E772
:10F15000382C0020582B002014070000702B0020B2
:10F1600070B53148007880210840802800D170BDFA
:10F170002E4800882E49884200D0F8E72B48807A34
:10F18000082800D0F3E72948807805072D0F2D02C5
:10F1900026484088000A0543082D00DAE7E70020EA
:10F1A0002149487006204880084685800120088152
:10F1B000082088720020C8728988481C0721F8F747
:10F1C000D5FF002909D01849898808460830072149
:10F1D000F8F7CCFF1449C88007E013498988481C18
:10F1E0000721F8F7C3FF1049C8801048008811496B
:10F1F000088008464580002407E00C48001D015D9A
:10F200000C48001D0155601CC4B2062CF5DB04201F
:10F2100000F024F9102004490870064A518810882B
:10F22000FFF710FE00BFA2E7382C0020582B00206B
:10F2300014070000702B002010B548480078A02863
:10F2400008D046480078912804D044480078A12886
:10F2500000D010BD42480088424988420AD0424945
:10F2600008880921FFF7E6FD00F036F900203B4948
:10F270000870EEE73A48807A08280AD03A490888A8
:10F280000921FFF7D7FD00F027F900203349087066
:10F29000DFE7334880780007000F002804D00128FA
:10F2A0002DD002284BD136E02C484078002800D0E1
:10F2B00050E02B48C078002803D10120274948702E
:10F2C00003E02748C07825498872244800789128AF
:10F2D0000BD023480079002803D101201F4908736F
:10F2E00003E01F4800791D49087391201B490870ED
:10F2F00000F0F2F81949087B00F092F82AE017486C
:10F300004078002800D025E0A1201449087003208F
:10F3100000F0A4F81EE011484078002800D019E061
:10F320000E480078A02809D10F4908880821FFF766
:10F3300081FD00F0D1F80020084908700AE00A4970
:10F3400008880521FFF776FD00F0C6F80020034984
:10F35000087000BF00BF00BF7BE70000382C002012
:10F36000582B002014070000D42B002010B528488B
:10F37000007880210840802800D110BD2448007802
:10F38000002805D0234800882349884200D0F4E7AC
:10F390002048807A1F4989780907090F884203DDD0
:10F3A0001C48807A082800D0E7E71A4880780007D0
:10F3B000000F002805D0174880780007000F0728A5
:10F3C00000DDDAE713480088144908801148807886
:10F3D0000007000F4880002407E00E48C01C015DB4
:10F3E0000E48001D0155601CC4B20C484088A04264
:10F3F000F3DC00200649087000F06EF807494A88DF
:10F4000008880023091DFFF725FD00BFB5E70000B0
:10F41000382C0020582B002014070000702B0020EF
:10F420007F2805DC7D21C90041430A4A91600DE037
:10F43000F12808DBF92806DC0107090F6422514393
:10F44000044A916002E00449024A91600221014AA3
:10F4500051737047482C002018F0010000B50300DC
:10F4600011F0A8F90729050B11171D232900012107
:10F47000144A11731449516022E00221114A117398
:10F48000114951601CE003210E4A11730F4951606C
:10F4900016E004210B4A11730D49516010E005215B
:10F4A000084A1173002151600AE00621054A1173D0
:10F4B0000849516004E00021024A1173516000BF05
:10F4C00000BF00BD482C0020A8610000F824010006
:10F4D00028230000F049020000200149087370470A
:10F4E000482C0020024909880918014A11807047F8
:10F4F000482C002010B52E480078102818D12D482F
:10F50000408860280ADD2C48807800090001801CB2
:10F510002949887022202649087025E026488078ED
:10F5200000090001244988702020214908701BE04F
:10F530001F480078112816D11D48807A002800D075
:10F5400010BD1B484078002800D0F9E70820184972
:10F5500088721948807800090001174988702020B6
:10F560001349087000E0EBE7144813490880084687
:10F570008078F021884330300F4988700846C07881
:10F580000020C87008460079142008710320887292
:10F590000220FFF763FF084A917A1088921CFFF758
:10F5A0000BFC054908880021FFF75CFB00BFC7E79B
:10F5B000382C0020702B0020642B002094070000C2
:10F5C000244A118852888A4242D0224A52888A426A
:10F5D00004DA204A52888A1A90B207E01D4A5288FB
:10F5E0000023DB439A1A521C521890B2194A5180D8
:10F5F000127B002A10D0174A5268002A0CD0154AF4
:10F600005268824205D9134A5268121A114B5A6045
:10F6100002E000220F4B5A600E4A527B022A17D199
:10F620000C4A9268002A0CD00A4A9268824205D994
:10F63000084A9268121A074B9A6002E00022054BB2
:10F640009A60044A9268002A02D10122014B5A733F
:10F6500070470000482C002010B506F0B5F810BD2A
:10F6600000BF704710B504468020204301460320A8
:10F67000400205F063FF10BD10B5102103204002C9
:10F6800005F05CFF10BD000010B50224024805F033
:10F69000A5FF0446204610BD0106000010B500215C
:10F6A000014805F04BFF10BD0106000010B50446EF
:10F6B000802020430146024805F040FF10BD0000B5
:10F6C0000106000010B51021014805F037FF10BDFC
:10F6D0000106000030B503460C46002101250D4807
:10F6E000834201D0002B01D1022030BD012A01D17B
:10F6F0000120FAE7002108E0C8002058984202D112
:10F7000000252846F1E7481C81B29142F4DB2846E7
:10F71000EBE70000FFFF0000002000BF14E0002125
:10F72000C200134B9950C200D2189180C200114BF5
:10F730009950C200D2189180C2000F4B9950C2005C
:10F74000D2189180411C88B24828E8DB0B490C4A4A
:10F7500011600C495160002191600B4911610B4906
:10F76000D16000210A4A11800A4A117070470000D6
:10F77000881F0020C821002008240020F50B01006C
:10F78000741F0020910C01003B0D01002D0D0100A4
:10F79000B6000020BA000020F0B585B00646674FDD
:10F7A000384603900290002500240020019000902C
:10F7B00063480068002803D061490868804707460D
:10F7C0005F484068002803D05D494868804703903F
:10F7D0005B488068002803D05949886880470290B8
:10F7E00057480069002803D05549086980470090B0
:10F7F0005348C068002803D05149C868804705466F
:10F80000482D00DD48250098002876D0002D74DDB5
:10F810004C480088A8420BDA2B463A4649494A48E8
:10F82000FAF75CFF2B4647494748039AFAF756FF19
:10F8300044480088002833DD42480088A84202D1AD
:10F84000002040490880002415E0E0003F490858A6
:10F85000E1003D4A515888420BD0E000114608585B
:10F86000E1003A4A5050E00011460858E100384A99
:10F870005050601C84B2AC42E7DB0120354908706F
:10F880002C460BE00020E100314A5050E1002F4AA5
:10F890005050E1002C4A5050601C84B2482CF1DBDF
:10F8A0002B4800682549884246D0294880882A4943
:10F8B000884205DA264880888019254988803BE0FF
:10F8C000002023498880084600680190012D33DD1F
:10F8D000002408E0601CC0001D490858E1001C4AD3
:10F8E0005050601C84B2681EA042F3DC691EC9003F
:10F8F000174A019850501FE0FFE700201549087093
:10F90000002414E00020E100114A5050E100891861
:10F910008880E1000C4A5050E10089188880E1009D
:10F920000A4A5050E10089188880601C84B2482C33
:10F93000E8DB00200349088005B0F0BDFFFF0000B0
:10F94000741F0020B6000020C821002008240020D9
:10F95000881F0020BA000020881300002E4800787D
:10F96000401C2D4908702D480078401C2B49087018
:10F970002B480078401C2A4908702A480068401C1F
:10F980002849086008460068FF219131884202D961
:10F9900000202449086020480078C82802D90020A7
:10F9A0001D4908701D480078842802D900201B4991
:10F9B00008701B480078502802D9002018490870A8
:10F9C000194818490968405C1849087018481249D4
:10F9D0000978405C17490870174810490978405C5D
:10F9E0001649087016480E490978405C1549087098
:10F9F000154809490978405C1449087014480649BB
:10FA00000978405C13490870134803490978405C41
:10FA100012490870704700004F070020500700206F
:10FA20005107002054070020171D0200480700203E
:10FA3000A71E0200490700206F1F02004A0700208E
:10FA4000BB2002004C070020F31F02004B070020E0
:10FA50000B2102004D070020D32102004E07002099
:10FA600010B58200054BD218525C012A04D1002245
:10FA70008300024C1B195A5410BD0000B42A002008
:10FA800010B50446204600F04FFA204600F002F878
:10FA900010BD000010B50446B248007800287DD1A2
:10FAA000B1480088B149884278DAB1480078002826
:10FAB0004FD0B0480078002803D0AB480088AE494A
:10FAC0000880AE480078002818D1A7480188AA48C5
:10FAD00000880F30814206D30120A8490870A2484F
:10FAE0000088A5490880A0480088A3490988884261
:10FAF0001CDA9D480088A049088017E09E480188CC
:10FB0000994800880F30814206D300209B49087035
:10FB10009548008898490880934800889649098844
:10FB2000884203DD90480088934908809348007814
:10FB3000002857D192480078042803D08D480078D7
:10FB4000002807D088480088822803DA05208C49DD
:10FB50000870A1E08A480078032803D0854800781F
:10FB6000002809D080480088FF211931884203DA33
:10FB70000420834908708FE081480078022803D070
:10FB80007C48007800280AD077480088FF21AF31F0
:10FB9000884204DA03207A4908707DE0E0E0784882
:10FBA0000078012803D073480078002808D06E48F8
:10FBB00000887449884203DA0220714908706BE0BA
:10FBC0006F480078002803D06A480078002863D086
:10FBD000654800886B49C83188425DDA0120684970
:10FBE000087059E065480078012855D164480078CC
:10FBF000012803D05F480078002809D05A480088BF
:10FC00006049C831884203DB00205D49087043E049
:10FC10005B480078022803D056480078002808D0B6
:10FC2000514800885749884203DB01205449087035
:10FC300032E053480078032803D04E48007800286B
:10FC400009D049480088FF21AF31884203DB0220F8
:10FC50004B49087020E04A480078042803D0454802
:10FC60000078002809D040480088FF2119318842D7
:10FC700003DB0320424908700EE041480078052864
:10FC800003D03C480078002806D0374800888228F6
:10FC900002DB04203A490870FCF7BAFE33496439A4
:10FCA00088425DD3384800680019374908603148F8
:10FCB0000078002808D000202E49087032490860DA
:10FCC0002F4800783149087000F084FD00281FD1CA
:10FCD0002D4800682E49884239D300202A490860FF
:10FCE0002A48007826490978884205DA27480078AA
:10FCF000401C264908702AE02448007820490978E9
:10FD0000884224DD21480078401E204908701EE00A
:10FD10001D4800681F49884219D300201A4908600D
:10FD20001A48007816490978884205DA1748007899
:10FD3000401C164908700AE01448007810490978F8
:10FD4000884204DD11480078401E104908700F48B1
:10FD500000780B490978884202D100200A490860DE
:10FD600010BD00000B000020020000201C0C000051
:10FD70001200002008000020040000200A000020DB
:10FD800006000020C6020000180000200700002026
:10FD9000C05D0000407E050000200B4908700B4943
:10FDA000087001200A4908700A49087000200A49B1
:10FDB00008700A4908700A4908800A4908800A49F7
:10FDC00008800A49087070470600002007000020DC
:10FDD00008000020090000200A0000200B0000207D
:10FDE0000C0000200E000020100000201200002057
:10FDF00000200B4908700B49087001200A4908705F
:10FE00000A49087000200A4908700A4908700A491E
:10FE100008800A4908800A4908800A490870704722
:10FE20000600002007000020080000200900002034
:10FE30000A0000200B0000200C0000200E00002013
:10FE40001000002012000020F1B500273048007893
:10FE5000002809D00320F9F781FB002804D00320F3
:10FE6000F9F770FB2B4908802B4800880A2847D3F4
:10FE700000202949088029480078282829D2032011
:10FE8000F9F760FB0746002407E060002449085AA0
:10FE9000B84200DD05E0601CC4B22048007884420E
:10FEA000F3DB00BF1D48057808E0681E40001C49D0
:10FEB000085A69001A4A5052681EC5B2A542F4DCBD
:10FEC000600017490F5215480078401C134908700C
:10FED00016E000260F2405E060001149085A861933
:10FEE000601CC4B2192CF7D30A213046F8F728F960
:10FEF0000849088000200949087001200949087054
:10FF0000054801880098081803490880F8BD0000DA
:10FF10000900002002000020160000200000002040
:10FF2000E0070020120000203A4909881E2928DA3B
:10FF30000021394A1180394A118039490988394AE2
:10FF4000914207DC38490978002914D034490988DE
:10FF5000914210DC0121354A11700021344A1170A0
:10FF6000344A1170304A11700121334A1170002156
:10FF7000324A11704CE02A4909880918284A118030
:10FF800046E024490988274A643291422BDB00214C
:10FF9000234A1180214A11801F490988AF2212018A
:10FFA000914207DC20490978002916D01A490988AE
:10FFB000914212DC02211D4A117000211C4A11706D
:10FFC00005211C4A11700021174A117001211A4A9B
:10FFD00011700021194A11701AE00F490988091897
:10FFE0000D4A118014E000210D4A11800A4A118047
:10FFF0000A4909880B4A914205DD00210B4A11701C
:020000040001F9
:10000000094A117004E0054909880918034A11805A
:100010007047000002000020100000200C000020AB
:100020000E000020B80B0000090000200B0000208B
:100030000600002007000020080000200A00002021
:100040000148007870470000B40900200148007A98
:1000500070470000B4090020014880787047000014
:10006000B40900200148008870470000800000208B
:10007000F8B50023002500950024002200BF94E07D
:1000800001259D40ACB20D8825400095009DA542FC
:100090006FD11A468D79012D0DD1464D03263602BA
:1000A000AD192D5C012696403543424E03273F0291
:1000B000F61935540CE03F4D03263602AD192D5C80
:1000C00001269640B5433B4E03273F02F6193554AF
:1000D000CD78002D4ED1374D60352D5CCE78002E79
:1000E00001D1012600E000269640B543314E60362E
:1000F00035548D78002D2ED12E4D19267601AD194F
:100100002D5C8E78002E01D1012600E0002696405D
:10011000B543284E19277F01F61935540D79002D66
:100120000ED1244D50352D5C0E79002E01D10126C3
:1001300000E000269640B5431E4E5036355423E06D
:100140001C4D50352D5C0E7996403543EEB2194D5D
:1001500050352E5418E0174D19267601AD192D5C37
:100160008E7896403543134E19277F01F619355482
:100170000AE018E00F4D60352D5CCE78964035438F
:10018000EEB20C4D60352E544D79012D0AD1094D3A
:1001900030352D5C012696403543EEB2054D3035A5
:1001A0002E5400E000BF5D1CABB2082B00DA67E7FD
:1001B000F8BD000000000440FFB5074615461E4686
:1001C00000243846019900F01FF8002802D00120D1
:1001D00004B0F0BD00240CE00A2060430949085C2B
:1001E000B04204D12946204600F05EF807E0601CCA
:1001F00084B20A2060430349085C0028ECD100BFA8
:100200000020E5E7A80100200246002A03D140298A
:1002100001DD01207047032A03D1022901DD0120FD
:10022000F8E7042A03D1202901DD0120F2E7052A9D
:1002300003D1202901DD0120ECE70C2A03D110298C
:1002400001DD0120E6E70D2A05D1012903DD402962
:1002500001DA0120DEE70E2A03D1202901D1012095
:10026000D8E70020D6E7000010B5064A03231B029A
:10027000D218125C8A43034B032424021B191A541C
:1002800010BD00000000044010B5064A03231B0205
:10029000D218125C0A43034B032424021B191A547C
:1002A00010BD00000000044070B502460020B1E01F
:1002B0000A2353435A4C1B195B1C440004191B1995
:1002C0009B788B427DD10A235343554C1B195B1CF1
:1002D000440004191B195B78082B33D10A235343BC
:1002E0004F4C1B195B1C440004191B574D4C4E4DC1
:1002F0006419E35C012423430A245443484D6419E0
:10030000641C450045196457464D474EAD192B55A1
:100310000A235343424C1B195B1C440004191B570E
:10032000404C35466419E35C022423430A245443B9
:100330003B4D6419641C450045196457394DAD198E
:100340002B5564E00A235343354C1B195B1C4400B6
:1003500004191B195B78092B34D10A235343304C01
:100360001B195B1C440004191B572E4C2E4D64199D
:10037000E35C402423430A245443294D6419641C3C
:10038000450045196457274D274EAD192B550A23B3
:100390005343234C1B195B1C440004191B57214C6D
:1003A00035466419E35C8024A3430A2454431C4D5E
:1003B0006419641C4500451964571A4DAD192B5535
:1003C00025E025E00A235343154C1B195B1C440010
:1003D00004191B57134C144D6419E35C0A2454434D
:1003E0000F4D6419641C4500451964196578012492
:1003F000AC402343DCB20A235343094D5B195B1C19
:10040000450045195B57074D074EAD19EC5404E004
:10041000431CD8B2032800DA4AE700BF70BD0000D1
:10042000A80100200000044075080000F8B5002471
:10043000FCF708FB012861D100F084FB0446FF2291
:100440000721002003F08EF8012C21D100F078FC68
:1004500000280ED000F088FB054600F079FB064628
:1004600001200346024629460090304605F0E6FB8F
:1004700050E000F079FB054600F06AFB06460120DB
:100480000023024629460090304605F0D7FB41E0A4
:10049000022C21D100F054FC00280ED000F064FBA7
:1004A000054600F055FB0646012003460246294654
:1004B0000090304605F0C2FB2CE000F055FB0546ED
:1004C00000F046FB0646002001231A46294600900C
:1004D000304605F0B3FB1DE000F032FC054600F0AD
:1004E00043FB064600F034FB0746012003462A463C
:1004F00031460090384605F0A1FB0BE00020034692
:1005000002460146009005F099FB002207211046A3
:1005100003F028F8F8BD0000FEB50024724800780A
:10052000012827D1FCF78EFA012815D1FCF76CF8C9
:1005300000BF0EE0182C0AD0152C08D00D2C06D0C8
:100540001A2C04D0FF222146002003F00BF8601C77
:10055000C4B2242CEEDBC6E0FCF7A2F9002406E0CE
:1005600000222146104602F0FDFF601CC4B2242C7C
:10057000F6DBB8E0FCF766FA012876D1FCF748FA1A
:100580005A4988426ED300F0E9FA064600F000FBB3
:1005900007460A21F7F7D4FD0546324629460120D1
:1005A0000BF008F900F032FD064600F0BFFC0A210E
:1005B0000290F7F7C5FD054600F0D0FA074632462F
:1005C000294609F085F8FFF731FF00F0A9FA054642
:1005D0002946012007F0C2FB00F0D4FA0646FF21AD
:1005E000F531F7F7C3FDC5B22946012006F0E2FA5E
:1005F000FFF726FD0546FFF735FD0646FFF72CFD04
:1006000007462B4632463946012005F0F1FD00F041
:10061000E7F80546294601200BF072FB00F0ACFC20
:10062000054600F0A5FB064600F0ACFC074600F0CE
:10063000A5FB00233A460146009601950290012051
:100640000AF0D4FD00F066FC054600F05DFC0646AD
:1006500000F066FC07462A46314607F0B3FD42E04B
:1006600003E0FFE7FCF74AF83DE0FCF719F9002248
:100670002321104602F076FF00222221104602F0CC
:1006800071FF00220721104602F06CFF00220821B2
:10069000104602F067FF00220921104602F062FFB7
:1006A00000220A21104602F05DFF002213211046AD
:1006B00002F058FF00221121104602F053FF0022E1
:1006C0001221104602F04EFF00220E21104602F0C9
:1006D00049FF00220F21104602F044FF00221021A2
:1006E000104602F03FFFFEBDE1000020B80B000005
:1006F00001490860704700007C070020024800683C
:10070000401C01490860704778070020F3B581B0AC
:10071000064600200E49086000F01EF8044600F06E
:100720001BF805462F1B3046029903F0D9FE0090B6
:100730000AE000F011F805462F1B06480068002863
:1007400002D004480068804700988742F1D3FEBD7C
:10075000780700207C0700200148006870470000EF
:10076000780700200B490978012901D101200FE009
:1007700008490978022901D1022009E005490978D0
:10078000032901D1042003E00121024A1170012054
:10079000704700000D07002010B5094B1B8899B267
:1007A0000A12C8B2D3433133064C2370C3432333F8
:1007B000637013465633A37003467133E37010BD64
:1007C0004007002013070020014800887047000000
:1007D00020000020014800887047000038000020F9
:1007E00001480078704700008D0000200148007823
:1007F000704700008E00002010B500220521064839
:10080000FAF788FC0402012205210348FAF782FC6A
:10081000201880B210BD00004C08002010B5062240
:1008200005210348FAF776FCC006C00F10BD000092
:100830004C08002010B5042205210648FAF76AFC8E
:100840000402052211460348FAF764FC201880B21E
:1008500010BD00004C08002010B5062205210248FA
:10086000FAF758FCC01110BD4C08002010B5022248
:1008700005210248FAF74EFC10BD00004C0800208C
:1008800010B5062205210348FAF744FC8006C00F84
:1008900010BD00004C08002010B5042202210348BE
:1008A000FAF738FCC007C00F10BD00004C0800204C
:1008B00010B5052202210348FAF72CFCC007C00F2F
:1008C00010BD00004C08002010B500220421034890
:1008D000FAF720FC4006400F10BD00004C08002035
:1008E00010B5042201210248FAF714FC801110BD52
:1008F0004C08002010B5002201210248FAF70AFC3A
:1009000010BD00004C08002010B50522012103484D
:10091000FAF700FC8007800F10BD00004C08002093
:1009200010B5012211460248FAF7F4FB10BD000091
:100930004C08002010B5002206210C48FAF7EAFB0B
:100940000402012206210948FAF7E4FB20180402F8
:10095000022206210548FAF7DDFB201804020322D3
:1009600006210248FAF7D6FB201810BD4C080020DB
:1009700010B5042206210C48FAF7CCFB040205222C
:1009800006210948FAF7C6FB201804020622114680
:100990000548FAF7BFFB2018040207220621024887
:1009A000FAF7B8FB201810BD4C08002010B5022241
:1009B00003210248FAF7AEFB10BD00004C080020EE
:1009C00010B5032200210248FAF7A4FB10BD000075
:1009D0004C08002010B5002211460248FAF79AFB95
:1009E00010BD00004C08002010B504220021024870
:1009F000FAF790FB10BD00004C08002010B5012252
:100A000000210248FAF786FB10BD00004C080020C8
:100A100010B5052200210248FAF77CFB10BD00004A
:100A20004C080020322815DA3C498978012903DD79
:100A300001213A4A517070E038498978002905DD72
:100A40002F286ADC0021354A517066E00021334AC4
:100A5000517062E03E2817DA322815DB2F49897879
:100A6000022903DD02212D4A517056E02B49897875
:100A7000012905DD3B2850DC0121284A51704CE05A
:100A80000121264A517048E0502817DA3E2815DB2C
:100A900022498978032903DD0321204A51703CE073
:100AA0001E498978022905DD4D2836DC02211B4AC2
:100AB000517032E00221194A51702EE0622817DA93
:100AC000502815DB15498978042903DD0421134AD0
:100AD000517022E011498978032905DD5F281CDC6B
:100AE00003210E4A517018E003210C4A517014E0A2
:100AF00073280FDA62280DDB08498978042905DD9F
:100B000070280ADC0421054A517006E00421034ADA
:100B1000517002E00521014A51707047B40900206C
:100B20000148007870470000070000200148006875
:100B300070470000881F00200148007870470000BF
:100B4000D50000200148007870470000D400002044
:100B50000148007870470000D90000200148007962
:100B60007047000038280020014840787047000096
:100B7000D90000200148007A704700003828002082
:100B800000207047014800887047000022000020C4
:100B900010B50024FFF7E2FF00280AD10A480088B8
:100BA0000A49884202DB084607490880064804884B
:100BB00008E005480088FCF715FC84B2044884422C
:100BC00000DB0446204610BD3A000020C6070000A6
:100BD000CE040000002005490988054A914202DB45
:100BE0001146024A11800149088870473A000020E6
:100BF000C6070000F8B50027002500260024FFF7EF
:100C0000E9FE0546FFF7FAFE0646F02028400011EF
:100C10000A2805DBF02028400011C01C044303E033
:100C2000F02028400011044324022807000F0A285E
:100C300004DB2807000FC01C044302E02807000F54
:100C400004432402F020304000110A2805DBF02084
:100C500030400011C01C044303E0F020304000117C
:100C6000044324023007000F0A2804DB3007000F7A
:100C7000C01C044302E03007000F0443002C01D1E4
:100C80000248F8BD27463846FBE70000FFFF00009A
:100C9000F8B50027002500260024FFF7A5FE05462D
:100CA000FFF7B6FE0646F020284000110A2805DBB3
:100CB000F02028400011C01C044303E0F02028402D
:100CC0000011044324022807000F0A2804DB280728
:100CD000000FC01C044302E02807000F0443240255
:100CE000F020304000110A2805DBF02030400011D0
:100CF000C01C044303E0F0203040001104432402F0
:100D00003007000F0A2804DB3007000FC01C044323
:100D100002E03007000F0443002C01D10248F8BD67
:100D200027463846FBE70000FFFF000010B500240F
:100D3000FFF746FE0446204610BD01207047000024
:100D400001480078704700004907002001480078FA
:100D5000704700004B0700200148C07B704700002F
:100D6000C00900200148C07C70470000C009002075
:100D70000148007A70470000C009002010B5002427
:100D800005480088323084B264212046F7F7EEF936
:100D900084B2204610BD0000C009002070B50024B8
:100DA00007490868FBF76EFF05466421F7F7C8F9A5
:100DB00084B20448844200DD0446204670BD000031
:100DC000C0090020DE03000010B5002400F014F874
:100DD000012800D10CE000F00FF8022802D1FF2416
:100DE000373405E00A2103480088F7F7BFF984B2D9
:100DF000204610BD02000020014800787047000026
:100E00000B000020002005490968002903D0034990
:100E10000968086800E00248704700005C01002093
:100E20003075000010B50024044804F0D7FB0028FA
:100E300001D0012400E00024204610BD030700007B
:100E400010B50024044804F0C9FB002801D0012497
:100E500000E00024204610BD0507000010B5002466
:100E6000044804F0BBFB002801D0012400E000246A
:100E7000204610BD0707000010B50024062004F02E
:100E8000ADFB002801D0012400E00024204610BD65
:100E900010B50024052004F0A1FB002801D0012496
:100EA00000E00024204610BD10B50024044804F0E2
:100EB00095FB002801D0012400E00024204610BD4D
:100EC0000607000010B50024044804F087FB002842
:100ED00001D0012400E00024204610BD03050000DD
:100EE00010B50024044804F079FB002801D0012447
:100EF00000E00024204610BD040500000148807A6F
:100F000070470000C0090020014880787047000049
:100F1000580A00200148406870470000580A002025
:100F20000148407870470000580A002070B500243E
:100F3000FFF714FE002803D1FCF768FC04460DE01F
:100F4000FFF70CFE012806D1FCF760FC0546FCF714
:100F500049FA044602E0FCF759FC0446204670BDFD
:100F60000148007C70470000C00900200148007D56
:100F700070470000C00900200148407A7047000017
:100F8000C009002010B5002405488088323084B2A2
:100F900064212046F7F7EAF884B2204610BD00002D
:100FA000C009002070B5002407494868FBF76AFEB5
:100FB00005466421F7F7C4F884B20448844200DD92
:100FC0000446204670BD0000C0090020DE0300007A
:100FD00070B50BF0A3F905460BF0A0F904490860C1
:100FE000002D01D1012400E00024204670BD000046
:100FF000680100200148007B70470000C009002004
:101000000148007870470000D800002070B5002427
:10101000FFF7A4FD002803D1FCF71AFC04460FE0FB
:10102000FFF79CFD012807D10020FCF711FC0546C5
:10103000FCF7D8F9044603E00020FCF709FC04465D
:10104000204670BD01480078704700004200002033
:1010500070B505460024032D00D170BD002D01D0D0
:10106000012D1BD181210320800204F067FA802129
:10107000134804F063FA32211248FFF747FB0024BB
:1010800009E0A200104BD2189178A200985A04F0FF
:1010900055FA601CC4B23B2CF3DB0FE0022D0DD1DE
:1010A000002409E0A200094BD2189178A200985AB6
:1010B00004F044FA601CC4B23B2CF3DB00BFCCE765
:1010C00002060000A0860100501302003C1402003A
:1010D000F8B5002100240023002200BF0AE001250A
:1010E0008D40ABB205881D402C469C4200D10A467B
:1010F0004D1CA9B21029F2DB0588FF2D1FDC284DFD
:101100006D7E0688B543264E757635462D7E06885B
:10111000B543234E357635466D7E8678F607F60F55
:10112000964035431E4E757635462D7E86780227CD
:101130003E40760896403543194E357622E0184DEC
:10114000ED7E0688B543164EF5763546AD7E0688AB
:10115000B543134EB5768578ED07ED0F1646083E7C
:10116000B5400F4EF67E35430D4EF5768578022656
:1011700035406D081646083EB540094EB67E3543EB
:10118000074EB5760025009505E000BF6D462D7829
:101190006D1CEEB200966D462D78012DF5D9F8BD87
:1011A000206B0440C107C90F002905D00021394A2E
:1011B0001171002238490A7102210140002905D02D
:1011C0000021344A1172002233490A72042101407D
:1011D000002905D000212F4A117300222E490A73DD
:1011E00008210140002905D000212A4A117400225B
:1011F00029490A7410210140002905D00021254AFF
:101200001175002224490A7520210140002905D0CA
:101210000021204A117600221F490A764021014010
:10122000002904D000221B494A711B494A718021C0
:101230000140002904D0002216494A7216494A7218
:10124000FF2101310140002904D0002211494A73D5
:1012500011494A73012149020140002904D00022AA
:101260000C494A740C494A74012189020140002941
:1012700004D0002207494A7507494A750121C9026D
:101280000140002904D0002202494A7602494A76E8
:10129000704700000060004000610040C107C90FB6
:1012A000002905D001223C490A7100213B4A1171F5
:1012B00002210140002905D0012237490A7200218C
:1012C000364A117204210140002905D00122324919
:1012D0000A730021314A117308210140002905D009
:1012E00001222D490A7400212C4A11741021014059
:1012F000002905D0012228490A750021274A1175C5
:1013000020210140002905D0012223490A7600212D
:10131000224A117640210140002905D001221E49B0
:101320004A7100221D494A7180210140002905D0DF
:10133000012219494A72002218494A72FF210131DB
:101340000140002905D0012213494A7300221349A4
:101350004A73012149020140002905D001220E49AA
:101360004A7400220D494A74012189020140002972
:1013700005D0012208494A75002208494A75012111
:10138000C9020140002905D0012203494A76002202
:1013900002494A767047000000610040006000404A
:1013A00010B50C480078002803D00B4A50689168AB
:1013B000884708484078002803D0084A5068916858
:1013C000884704488078002803D0054A506891680F
:1013D000884710BD00600040F8020020780400201B
:1013E000F805002010B508480079002803D0074A06
:1013F00010695169884704484079002803D0044A9D
:1014000050689168884710BD00600040F8020020D5
:101410008404002010B50848007A002803D0074A49
:10142000D069116A88470448407A002803D0044AEA
:1014300050689168884710BD00600040F8020020A5
:101440009004002010B50848007B002803D0074A0C
:10145000906AD16A88470448407B002803D0044A38
:1014600050689168884710BD00600040F802002075
:101470009C04002010B50848007C002803D0074ACF
:10148000506B916B88470448407C002803D0044A85
:1014900050689168884710BD00600040F802002045
:1014A000A804002010B50848007D002803D0074A92
:1014B000106C516C88470448407D002803D0044AD2
:1014C00050689168884710BD00600040F802002015
:1014D000B404002010B50848007E002803D0074A55
:1014E000D06C116D88470448407E002803D0044A20
:1014F00050689168884710BD00600040F8020020E5
:10150000C004002010B50848407F002803D0074AD7
:101510005068916888470448007F002803D0044A37
:10152000906DD16D884710BD00600040CC04002054
:10153000F802002010B508484078002803D0074A78
:1015400050689168884704480078002803D0044A0E
:10155000506E916E884710BD20600040D804002076
:10156000F802002010B509480079002803D0084A85
:10157000106F516F88470548001D4078002803D040
:10158000044A50689168884710BD00002060004000
:10159000F8020020E404002010B5034AD06F78322E
:1015A0009168884710BD0000F802002010B5024A7B
:1015B00050689168884710BD7C03002010B5094829
:1015C000007C002803D0084A506891688847054885
:1015D00010304078002803D0044A5068916888474A
:1015E00010BD000020600040880300200805002096
:1015F00010B5024A50689168884710BD94030020D6
:1016000010B5024A50689168884710BDA0030020B9
:1016100010B50948007F002803D0084A5068916837
:10162000884705481C304078002803D0044A506899
:101630009168884710BD000020600040AC03002086
:101640002C05002010B50C480078002803D00B4A68
:1016500050689168884708484078002803D0084AB5
:1016600050689168884704488078002803D0054A6C
:1016700050689168884710BD40600040B803002062
:1016800038050020B806002010B50D480079002864
:1016900003D00C4A5068916888470948001D40787B
:1016A000002803D0084A5068916888470448001D04
:1016B0008078002803D0054A50689168884710BD9B
:1016C00040600040C403002044050020C406002000
:1016D00010B50D48007A002803D00C4A5068916874
:1016E0008847094808304078002803D0084A5068E5
:1016F00091688847044808308078002803D0054A5C
:1017000050689168884710BD40600040D0030020B9
:1017100050050020D006002010B50D48007B0028A1
:1017200003D00C4A50689168884709480C304078CB
:10173000002803D0084A50689168884704480C3054
:101740008078002803D0054A50689168884710BD0A
:1017500040600040DC0300205C050020DC06002027
:1017600010B50D48007C002803D00C4A50689168E1
:101770008847094810304078002803D0084A50684C
:1017800091688847044810308078002803D0054AC3
:1017900050689168884710BD40600040E803002011
:1017A00068050020E806002010B5024A50689168DC
:1017B000884710BDF403002010B50948007E0028BA
:1017C00003D0084A50689168884705481830407827
:1017D000002803D0044A50689168884710BD000073
:1017E00040600040000400208005002010B509483A
:1017F000007F002803D0084A506891688847054850
:101800001C304078002803D0044A5068916888470B
:1018100010BD0000406000400C0400208C0500203A
:1018200010B508480078002803D0074A506891682E
:10183000884704484078002803D0044A50689168DB
:10184000884710BD60600040180400209805002003
:1018500010B509480079002803D0084A50689168FB
:1018600088470548001D4078002803D0044A506886
:101870009168884710BD000060600040240400208B
:10188000A405002010B50948007A002803D0084AB2
:10189000506891688847054808304078002803D090
:1018A000044A50689168884710BD0000606000409D
:1018B00030040020B005002010B5024A506891683D
:1018C000884710BD3C04002010B5024A506891685A
:1018D000884710BD4804002010B50948007D002845
:1018E00003D0084A5068916888470548143040780A
:1018F000002803D0044A50689168884710BD000052
:101900006060004054040020D405002010B5094850
:10191000007E002803D0084A50689168884705482F
:1019200018304078002803D0044A506891688847EE
:1019300010BD00006060004060040020E005002051
:1019400010B50948007F002803D0084A5068916804
:10195000884705481C304078002803D0044A506866
:101960009168884710BD0000606000406C04002052
:10197000EC05002010B5FE4800688079002806D0EC
:1019800001286ED002286DD003286CD104E2F848FB
:101990000068407903000EF00DFF0A0614BC2BBC52
:1019A00047BC67BC9BBC0AF05FFF0020F049096898
:1019B000C873EF4800684079401CED4909684871D8
:1019C000AEE0EC490969EA4A1268D27A885C0AF00A
:1019D000C3FFE74800684079401CE5490968487141
:1019E000E34800684079401CE1490968487197E084
:1019F00001F020FF002810D10AF0AEFFDC4800689B
:101A00004079401CDA4909684871D9480068407932
:101A1000401CD7490968487105E00AF04FFF0020D3
:101A2000D349096848717BE001F004FF002811D117
:101A300001200AF091FFCE4800684079401CCC4953
:101A400009684871CA4800684079401CC84909685B
:101A5000487105E00AF032FF0020C5490968487165
:101A60005EE05FE0FEE0A3E101F0E4FE002828D1A3
:101A7000BF490968C97A24225143BF4A12688918AC
:101A8000BB4A1268D27B885C0AF066FFB8480068DF
:101A9000C07B401CB6490968C873B5480068C07B64
:101AA000242814D3B24800684079401CB049096822
:101AB0004871AF4800684079401CAD4909684871D9
:101AC00005E00AF0FBFE0020A9490968487127E0FB
:101AD00001F0B0FE002815D1A5480068C07A401C6E
:101AE000A3490968C872A2480068C07AA149097868
:101AF000884207DB00209E490968C87201209C4982
:101B0000096888710AF0DAFE00209949096848716D
:101B100006E00AF0D3FE002095490968487100BF2D
:101B200000BF4FE192480068407903000EF042FE8A
:101B3000080513912A91479170910AF095FE0020B3
:101B40008B490968C8738A4800684079401C8849F5
:101B50000968487184E087490969854A1268D27A20
:101B6000885C0AF0F9FE824800684079401C804990
:101B7000096848717E4800684079401C7C490968C2
:101B800048716DE001F056FE002811D126200AF0C0
:101B9000E3FE774800684079401C75490968487140
:101BA000734800684079401C71490968487105E034
:101BB0000AF084FE00206E490968487150E001F087
:101BC00039FE00281DD101200AF0C6FE68480068D1
:101BD000C07B401C66490968C87365480068C07BC3
:101BE000242814D3624800684079401C6049096881
:101BF00048715F4800684079401C5D490968487138
:101C000005E00AF05BFE002059490968487127E0A9
:101C100001F010FE002815D155480068C07A401C1C
:101C200053490968C87252480068C07A5149097816
:101C3000884207DB00204E490968C87202204C49DF
:101C4000096888710AF03AFE00204949096848711C
:101C500006E00AF033FE002045490968487100BFDC
:101C600000BFAFE042480068407903000EF0A2FDDB
:101C70000805138B2A8B478B638B0AF0F5FD002038
:101C80003B490968C8733A4800684079401C3849A4
:101C9000096848717EE037490969354A1268D27A85
:101CA000885C0AF059FE324800684079401C30498F
:101CB000096848712E4800684079401C2C49096821
:101CC000487167E001F0B6FD002811D125200AF027
:101CD00043FE274800684079401C2549096848713F
:101CE000234800684079401C21490968487105E093
:101CF0000AF0E4FD00201E49096848714AE001F03D
:101D000099FD002810D10AF027FE19480068407993
:101D1000401C174909684871154800684079401C03
:101D200013490968487105E00AF0C8FD0020104910
:101D3000096848712EE001F07DFD002815D10C489E
:101D40000068C07A401C0A490968C87208480068DF
:101D5000C07A08490978884207DB002004490968ED
:101D6000C87203200249096888710AF0A7FD05E0DE
:101D7000CC070020342F0020C80700200020124983
:101D80000968487106E00AF099FD00200E490968CB
:101D9000487100BF00BF15E000200B490968887139
:101DA000094909684871062007490968C87009E0AF
:101DB0000AF084FD00200449096848710249096855
:101DC000887100BF00BF10BDCC07002010B56A4865
:101DD0000068407903000EF0EDFC090610C627C626
:101DE00044C6608EC6000AF03FFD63480068407933
:101DF000401C614909684871BCE0604909695E4A54
:101E00001268D27A885C0AF0A7FD5B4800684079C6
:101E1000401C594909684871574800684079401C7E
:101E2000554909684871A5E001F004FD002811D169
:101E30004F200AF091FD504800684079401C4E49FF
:101E4000096848714C4800684079401C4A49096853
:101E5000487105E00AF032FD0020474909684871E1
:101E600088E001F0E7FC002810D10AF075FD424837
:101E700000684079401C4049096848713E48006844
:101E80004079401C3C490968487105E00AF016FD9C
:101E900000203949096848716CE001F0CBFC00284A
:101EA00022D135480068C07A401C33490968C8729D
:101EB00031480068C07A3149097888420FDB002038
:101EC0002D490968C8722C4800684079401C2A498D
:101ED00009684871002028490968486208E0002024
:101EE00025490968487103E00020234909684871C1
:101EF0000AF0E4FC3EE020480068407C002816D050
:101F00001E48C068002803D01C48C16819208847B3
:101F1000002019490968486217490968487116493B
:101F200009688871052014490968C8701AE01248C8
:101F30000068406A282807D20F480068406A401CA1
:101F40000D49096848620DE000200B4909684862A4
:101F500009490968487108490968887105200649D6
:101F60000968C87006E00AF0A9FC00200249096867
:101F7000487100BF00BF10BDCC070020342F0020E7
:101F800010B50024F7480068807A01287ED1F54812
:101F90000068C07900287AD0F2480068807900286B
:101FA00004D0012874D0022873D191E1ED48006873
:101FB000007B24286ED2EB480068C07901287AD1D2
:101FC000002475E0E7480068C07A24214843E649C8
:101FD00009684018E3490968097B415CE1480068E9
:101FE000C07A24225043E14A12688018DD4A126800
:101FF000127B805C814229D0DA480068C07A2421B3
:102000004843DA4909684018D6490968097B415CA8
:10201000D4480068C07A24225043D34A12688018FA
:10202000D04A1268127B8154CE480068407B242835
:1020300005D3CC480068007BCA4909684873C94881
:102040000068007BC7490968887308E0C5480068D4
:10205000407B242803D20120C24909688871C14805
:102060000068007B401CBF4909680873BD480068D0
:10207000007B242808D3BB480068407B242803D277
:102080000120B84909688871B64805E0D3E1CDE17F
:1020900069E0BAE138E00EE00068007B242804D251
:1020A000B04800688079012800D103E0601CC4B208
:1020B000242C87D356E0002413E0AA480068C07A95
:1020C00024214843A94909684018015DA5480068D2
:1020D000C07A24225043A44A126880180155601C1B
:1020E000C4B2242CE9D300209E49096848732320F8
:1020F0009C490968887301209A49096888712420DD
:102100009849096808732DE000209649096808730A
:1021100094480068C07A401C92490968C872914886
:102120000068C07A92490978884217DB8D480068B8
:10213000007C012804D102208A490968887106E0E0
:10214000002088490968887186490968C87100209B
:1021500084490968C8728349096808740020814964
:102160000968487161E17F480068407903000EF01A
:1021700021FB080513A62AA651A68EA6012079499F
:10218000096808740AF070FB764800684079401CC2
:1021900074490968487199E075490969714A12687A
:1021A000D27A885C0AF0D8FB6E4800684079401CFF
:1021B0006C49096848716B4800684079401C69495E
:1021C0000968487182E001F035FB00281BD16549A0
:1021D0000968497B491CC8B20AF0BEFB6148006827
:1021E000407B60490968C8735E4800684079401CBC
:1021F0005C49096848715B4800684079401C59494E
:102200000968487105E00AF059FB00205549096842
:1022100048715BE001F00EFB00282BD151490968A1
:10222000C97A24225143504A126889184D4A1268CB
:10223000D27B885C0AF090FB4A480068C07B401C57
:1022400048490968C87347480068C07B4549096820
:10225000897B88421ADD434800684079401C414927
:10226000096848713F4800684079401C3D49096849
:1022700048710BE00AF022FB3A480068407B39497C
:102280000968C87300203749096848711EE001F0E9
:10229000D1FA00280CD133490968887124203149CA
:1022A0000968C8732F49096848732E4909688873FB
:1022B0000AF004FB00202B490968487106E00AF087
:1022C000FDFA002027490968487100BF00BFACE053
:1022D00024480068407903000EF06CFA08050F8E60
:1022E000268E4C8E688E0AF0BFFA1E480068407930
:1022F000401C1C490968487185E01D490969194A53
:102300001268D27A885C0AF027FB16480068407988
:10231000401C144909684871124800684079401C03
:102320001049096848716EE001F084FA002811D163
:1023300025200AF011FB0B4800684079401C094930
:1023400009684871074800684079401C05490968D8
:10235000487105E00AF0B2FA0020024909684871A4
:1023600051E00000CC070020C8070020C40700206F
:10237000342F002001F05EFA002810D10AF0ECFAA8
:10238000644800684079401C6249096848716148A6
:1023900000684079401C5F490968487105E00AF00F
:1023A0008DFA00205B49096848712CE001F042FA7F
:1023B00000281AD157480068C07A401C554909685E
:1023C000C87254480068C07A5349097888420CDBC7
:1023D000002050490968C8724E49096888714D4902
:1023E000096848714B490968C8710AF067FA00200A
:1023F00048490968487106E00AF060FA002045493A
:102400000968487100BF00BF0FE00AF057FA0020CA
:102410004049096848713F49096888713D49096820
:1024200008733C490968C87200BF71E0002039494F
:10243000096888726CE037480068807A022867D1A2
:1024400034480068007A00285ED03248006840793D
:10245000002804D001280CD0032846D11BE00AF044
:1024600003FA2C4800684079401C2A4909684871E1
:1024700049E000200AF070FA264800684079401CC4
:10248000244909684871234800684079401C214963
:102490000968487137E00AF0B1F9002812D11D48E7
:1024A00000684078401C1B4909684870194800685A
:1024B0004078032812D301F05DFA0020154909681D
:1024C00048700BE00020134909680872AA201149DE
:1024D0000968887000200F49096848700AF0EEF911
:1024E00000200C49096848710DE00AF0E7F9002066
:1024F000084909684871074909684870AA200549D0
:102500000968887000BF03E00020024909688872EA
:1025100010BD0000CC070020342F0020F8B5044681
:102520000D4600260C2060431D49085C002801D0A0
:102530000120F8BD0C2060431949401885600C202B
:10254000604340188068002801D10120F1E7012193
:102550000C206043124A115400222046E317DB0E80
:102560001B185B115B01E31A9B000E4FDB19E71789
:10257000FF0E3F197F11DA550EF04EF9002220466A
:10258000E317DB0E1B185B115B01E31A9F00064B80
:10259000FB18E717FF0E3F197F11DA553046C8E7E1
:1025A000F8020020006000400061004000BFFEE72C
:1025B00009480088401C08490880084600880749E7
:1025C000884208DD06480078002804D00846024901
:1025D0000880012088707047D0000020DC050000D2
:1025E000D400002010B515488078012824D1144863
:1025F000007801280CD113480078012808D1002068
:1026000011498870084602F0B7FD00200D49087096
:102610000B48007802280CD10C480078012808D11A
:10262000002009498870084602F0A6FD00200749ED
:10263000087000200249087010BD0000D000002082
:10264000D4000020D6000020D9000020D7000020B0
:102650007047000010B500F05DFE012803D1002096
:1026600001490880887010BDD0000020F0B50546F3
:102670000E46174600243A463146284600F058FEDA
:1026800000BF42E000202101394A12685052210166
:10269000374A12688918488000212001344A12689C
:1026A000801881802001324A12688018C180200180
:1026B0002F4A12688018017220012D4A1268801872
:1026C000417220012A4A1268801881722001284A2A
:1026D00012688018C17200202101254A12688918E9
:1026E000087300212001224A1268801841730020DB
:1026F00021011F4A126889188873002120011C4A91
:1027000012688018C173601CC4B21A484078A04295
:10271000B8DC64201849096808807D20C00016498B
:102720000968488015481449096888807D2000019F
:1027300011490968C88010490968088110480E4984
:10274000096848810F480C490968888140000A4996
:102750000968C8813220084909680882FF20F530DD
:10276000054909684882044909688882F0BD00006B
:102770008C07002080070020880700204C04000000
:10278000102700003075000038B5002404E0002058
:1027900013490855601C84B2282CF8D301216846DF
:1027A000417001706A460F490D48FFF75FFF7D21B8
:1027B000C900322000F0ACF90B490C4800F0C6F912
:1027C0000948643000F058F90748C83000F064F94F
:1027D000074800F077F9074800F08AF938BD000093
:1027E000482800200819020028230000B80B000028
:1027F000542400001027000010B524480078002859
:1028000003D10120214908703EE0204800780128CA
:1028100010D11F480078012808D100201D49887078
:10282000084602F0A9FC0020194908700220174947
:10283000087029E015480078022810D11648007861
:10284000012808D1002013498870084602F094FC42
:1028500000201149087003200C49087014E00B484F
:102860000078032803D10520084908700CE00748C8
:102870000078052803D005480078062804D10020F8
:10288000024908700549087010BD0000D4000020FE
:10289000D6000020D9000020D7000020D80000205A
:1028A000F8B50024002500263548007800281ED100
:1028B00034480078002803D101203249087016E01E
:1028C00030480078012803D102202E4908700EE01C
:1028D0002C480078022803D103202A49087006E01A
:1028E00028480078032802D100202649087024488F
:1028F000007801280ED10124172500262248012343
:10290000324629460090204601F048FE01201F492A
:10291000087034E01A48007802280FD101243B25C2
:1029200000261948401C01233246294600902046C3
:1029300001F034FE01201649087020E010480078AC
:1029400003280DD1FEF70AF9002803D1012011490F
:10295000087102E000200F4908710DF0FDFE0EE045
:1029600007480078052803D106200549087006E0CD
:1029700003480078062802D1052001490870F8BDF7
:10298000D4000020D5000020D9000020D60000206F
:10299000D70000203828002010B5044623000DF091
:1029A00009FF095B060E16171819595A5E00FAF747
:1029B0002FF82C49884201D3FFF772FF50E0FAF755
:1029C00027F82849884201D3FFF716FF48E047E07F
:1029D00046E045E0FAF71CF82249884239D301F075
:1029E0008DFD21480078032814D120480078002864
:1029F00010D1FEF7BFF8002806D101201C498860DD
:102A00008868FAF78BFF05E000201949886088681C
:102A1000FAF784FF14480078012805D1134800789C
:102A2000002801D1FAF786F910480078052803D16B
:102A30000120104908700AE00C480078062803D1EC
:102A400002200C49087002E000200A4908700BF0CF
:102A500023FC05E004E003E0FFF7AAFD00E000BF6F
:102A600000BF10BDB80B0000D5000020D40000202E
:102A700038280020D800002001460020054A1268AE
:102A800052898A4201DC012002E0024A1268118167
:102A9000704700008807002001460020084A12689D
:102AA00012898A4201DB012009E0054A12689289F5
:102AB0008A4201DC012002E0014A1268518170471C
:102AC0008807002001460020084A126852898A427D
:102AD00001DB012009E0054A1268D2898A4201DC43
:102AE000012002E0014A12689181704788070020A6
:102AF00001460020054A126892898A4201DB0120C2
:102B000002E0024A1268D181704700008807002065
:102B1000024600200C4B1B681B8A934201DD0120FA
:102B200010E08A4201DB01200CE0074B1B689B8808
:102B30008B4201DC012005E0034B1B681A80024B2D
:102B40001B6859807047000088070020024600205B
:102B50000C4B1B681B8A934201DD012010E08A4266
:102B600001DB01200CE0074B1B685B88934201DB13
:102B7000012005E0034B1B689A80024B1B68D9803B
:102B8000704700008807002070B5044600250C201F
:102B90006043FE49096840184068002807D00C21AE
:102BA0006143FA4A126889184868804705460C2034
:102BB0006043F6490968085C002873D10C20604323
:102BC000F249096840188068002874D02001F04953
:102BD00009684018C07A02280AD1032D08D10C20B8
:102BE0006043EA4A1268801881680120884762E0E1
:102BF0002001E74909684018C07A02280AD1042D4B
:102C000008D10C206043E14A1268801881680220D4
:102C1000884750E02001DE4909684018C07A022840
:102C20000AD1052D08D10C206043D84A12688018BB
:102C30008168032088473EE02001D5490968401893
:102C4000C07A02280AD1062D08D10C206043CF4A51
:102C5000126880188168042088472CE02001CC4944
:102C600009684018C07A02280AD1072D08D10C2023
:102C70006043C64A126880188168052088471AE0B8
:102C80002001C34909684018C07A02280BD1082DD9
:102C900009D10C206043BD4A126880188168062063
:102CA000884708E00DE00C206043B84A126880189D
:102CB0008168002088472001B54909684018C5721D
:102CC0000CE30C206043B1490968085C012873D10A
:102CD0000C206043AD49096840188068002874D012
:102CE0002001AB4909684018C07A03280AD1022D97
:102CF00008D10C206043A54A126880188168012021
:102D0000884762E02001A24909684018C07A042877
:102D10000AD1022D08D10C2060439C4A1268801809
:102D200081680220884750E02001994909684018CD
:102D3000C07A05280AD1022D08D10C206043934A9D
:102D4000126880188168032088473EE0200190497E
:102D500009684018C07A06280AD1022D08D10C2033
:102D600060438A4A126880188168042088472CE0F2
:102D70002001874909684018C07A07280AD1022D26
:102D800008D10C206043814A1268801881680520B0
:102D900088471AE020017E4909684018C07A08284F
:102DA0000BD1022D09D10C206043784A126880189B
:102DB00081680620884708E00DE00C206043734AD4
:102DC00012688018816800208847200170490968CE
:102DD0004018C57282E20C2060436C490968085CA7
:102DE0000228F7D1002D7DD1200169490968085AD0
:102DF00068490968098A884275DA200164490968C6
:102E0000085A0A3081B22001614A12681152200129
:102E10005F490968085A5F490968098A884231DBB5
:102E200020015B490968401840885A4909680988A7
:102E3000884227DB200156490968401840885549D7
:102E40000968498888421DDC00202101504A126827
:102E50008918488020014E4909684018807A002866
:102E6000B8D10C206043494909684018806800289F
:102E7000B0D00C206043454A126880188168012058
:102E800088472BE2200142490968085A41490968EC
:102E9000098A88429EDB20013D4909684018408824
:102EA0003C4909688988884294DB200138490968CF
:102EB0004018408837490968C98888428ADC002060
:102EC0002101334A12688918488020013049096875
:102ED0004018807A0028D4D10C2060432B4909681F
:102EE000401801E063E00BE080680028C9D00C20A6
:102EF0006043264A12688018816802208847EDE105
:102F000000202101224A1268891848802101204AA4
:102F100012688918C872002120011D4A12688018A1
:102F2000C18020011A4A1268801841722001184A93
:102F3000126880188172184801782001144A1268BA
:102F40008018017200202101114A126889188880B6
:102F500021010F4A12688918087321010C4A12686E
:102F60008918487321010A4A126889188873002158
:102F70002001074A12688018C1730C20604303497E
:102F80000968401880680028B9D007E0840700204D
:102F90008C07002088070020800700200C20604359
:102FA000CF4A1268801881680020884796E1012D79
:102FB000A5D12001CB4909684018C07AA84225D084
:102FC00000212001C74A1268801841800020210199
:102FD000C44A12688918C8802001C249096840188B
:102FE000C572C14800782101BE4A1268891848722A
:102FF00000202101BB4A126889188880BA480178EC
:103000002001B84A12688018017267E12001B549B1
:1030100009684018007AB4490978884220D0B2483B
:1030200000782101AF4A1268891808722001AD4961
:1030300009684018407AAC490978884209D02001D3
:10304000A8490968401880882101A64A1268891891
:10305000C88000212001A34A12688018818012E0F4
:103060002001A049096840188088A04988420AD2F6
:1030700020019C490968401880880A302101994A3A
:10308000126889188880200196490968401840888C
:10309000964988420AD2200192490968401840881E
:1030A0000A3021018F4A12688918488020018D4911
:1030B00009684018407A8C490978884205D0012077
:1030C0002101884A12688918887220018549096897
:1030D00040184088864909680988884204DB002135
:1030E0002001804A1268115220017E490968401867
:1030F000807A00287ED10C20604379490968401805
:103100008068002877D020017649096840184088F7
:10311000774909680989884214DB200171490968E7
:103120004018007B00280DD10C2060436C4A1268C7
:10313000801881680320884701202101694A1268AC
:103140008918087320016749096840184088684950
:1031500009684989884214DB2001624909684018DE
:10316000407B00280DD10C2060435D4A1268801816
:10317000816804208847012021015A4A1268891871
:103180004873200157490968401840885849096820
:103190008989884214DB2001524909684018807BE4
:1031A00000280DD10C2060434D4A126880188168B8
:1031B00005208847012021014A4A1268891888732E
:1031C0002001484909684018408849490968C98967
:1031D000884210DB2001434909684018C07B002861
:1031E0007CD10C2060433E4A12688018816806201A
:1031F000884701E007E03BE001202101394A1268DD
:103200008918C8736AE02001364909684018407A75
:1032100001282ED13448007802282AD120013149D2
:1032200009684018C08832490968498A884255DBD4
:1032300020012C490968401880882D490968898A2D
:1032400088424BDB0C2060432549096840188068A0
:10325000002843D00C206043214A126880188168FE
:1032600007208847002021011E4A126889184872E9
:1032700034E020011B4909684018407A02282DD10A
:1032800019480078012829D12001164909684018F9
:10329000C08817490968898A88421FDB20011149C3
:1032A00009684018808812490968498A884215DBF4
:1032B0000C2060430A4909684018806800280DD036
:1032C0000C206043064A12688018816808208847ED
:1032D00000202101034A12688918487270BD00005D
:1032E000840700208C07002080070020F0FF0000EA
:1032F0008807002010B5002400BF04E02046FFF737
:1033000043FC601CC4B202484078A042F6DC10BD09
:103310008007002010B50024044802F05FF900285F
:1033200000D000E00124204610BD0000030400008E
:1033300010B5074B14781C7054785C70054B1960FD
:10334000054B186003461833044C236010BD000081
:103350008007002084070020880700208C070020B9
:1033600010B50446012C09D1FF220C21002000F0E9
:10337000F9F80121022004F05FFE08E000220C2190
:10338000104600F0EFF80021022004F055FE10BDB9
:1033900010B5002404210848F7F7CEFE552801D1C6
:1033A000012407E0042001F01BF8002801D00024CC
:1033B00000E00124204610BD4C08002010B5044652
:1033C000012C09D1FF221C21002000F0CBF80121A3
:1033D000062004F031FE08E000221C21104600F017
:1033E000C1F80021062004F027FE10BD10B500240E
:1033F000062000F0F5FF002801D0012400E00024A1
:10340000204610BD10B50446012C09D1FF2217211A
:10341000002000F0A7F80121042004F00DFE08E0D0
:1034200000221721104600F09DF80021042004F02E
:1034300003FE10BD00200449097A002901D00120B3
:1034400000E0002070470000580A002010B5044634
:10345000022C1CD100220D21104600F083F8FDF74C
:103460006FFC002809D0FF220B21002000F07AF821
:1034700001210D2004F0E0FD58E000220B21104650
:1034800000F070F800210D2004F0D6FD4EE0032C72
:103490001CD100220B21104600F064F8FDF750FC0F
:1034A000002809D0FF220D21002000F05BF8012147
:1034B0000D2004F0C1FD39E000220D21104600F07E
:1034C00051F800210D2004F0B7FD2FE0042C0ED19F
:1034D000FF220D21002000F045F800220B211046AC
:1034E00000F040F801210D2004F0A6FD1EE0012CA3
:1034F0000ED100220D21104600F034F8FF220B21DE
:10350000002000F02FF801210D2004F095FD0DE0C2
:1035100000220D21104600F025F800220B21104654
:1035200000F020F800210D2004F086FD10BD000001
:1035300010B500240A480078012801D101240CE0CC
:10354000FCF784FD012801D1032406E0FCF77EFD91
:10355000022801D1022400E00424204610BD00000E
:10356000E100002010B5064B1B78834207DD2429BB
:1035700005D224234343034C24681B195A5410BD1D
:10358000342F0020C407002010B57448006840792B
:1035900003000DF00FF90B0711D325D35A6D77D324
:1035A0008DA8D30009F060F96C4800684079401C90
:1035B0006A4909684871CFE069494969087809F0A2
:1035C000CBF9664800684079401C64490968487135
:1035D000624800684079401C604909684871BBE056
:1035E00000F028F9002811D17F2009F0B5F95B48D7
:1035F00000684079401C594909684871574800687B
:103600004079401C5549096848711DE053480068DD
:103610004078401C5149096848705048006840781B
:1036200003280BD300204D4909684870AA204B4954
:1036300009688870032049490968C87009F03EF993
:10364000002046490968487186E000F0F3F8002838
:1036500007D1424800684079401C404909684871D8
:1036600003E000203D490968487109F027F973E03B
:1036700009F0FAF8394800684079401C3749096870
:10368000487169E0364949690978491CC8B209F0AE
:1036900063F9324800684079401C30490968487134
:1036A0002E4800684079401C2C490968487153E055
:1036B00000F0C0F800280FD109F0A8F827490968E0
:1036C0008870012009F01CF9244800684079401CEA
:1036D00022490968487105E009F0F0F800201F4907
:1036E0000968487138E01D480068807818280CD1B6
:1036F00002201A49096808700020184909684870B2
:10370000042016490968C87011E014480068407820
:10371000401C124909684870104800684078032826
:1037200005D300F027F900200C490968487009F01A
:10373000C5F800200949096848710DE009F0BEF894
:103740000020064909684871044909684870AA20A0
:1037500002490968887000BF00BF10BDCC07002077
:10376000342F002010B5314800684079002804D07B
:1037700001280CD0032848D11DE009F075F82B482A
:1037800000684079401C2949096848714BE0284984
:103790000969087809F0E0F8244800684079401C7D
:1037A000224909684871214800684079401C1F4936
:1037B0000968487137E000F03DF800280CD101207D
:1037C0001A490968087000201849096848700420DF
:1037D00016490968C87011E0144800684078401C18
:1037E000124909684870114800684078032805D3D9
:1037F00000F0C0F800200D490968487009F05EF833
:1038000000200A49096848710DE009F057F80020C6
:10381000064909684871054909684870AA200349A2
:103820000968887000BF00BF10BD0000CC070020F1
:10383000342F002010B508F0E1FF04461F4800684F
:103840000078002838D01D480068C078042833D399
:10385000002C09D1002119480068C07A820017485D
:1038600000681430815027E014480068C07A810055
:1038700012480068143040581149884211D20F484C
:103880000068C07A81000D48006814304058401C20
:103890000A490968C97A8A000849096814318850B8
:1038A0000AE000F067F8002104480068C07A82004E
:1038B0000248006814308150204610BDCC0700201B
:1038C000B80B000000B587B00120694608710848B0
:1038D000029008480390084804900848059008485A
:1038E000069001A9074800F00FF807B000BD0000DE
:1038F0002D3C0100C9570100410902007519020061
:1039000074190200B0280020F8B506460F460024BE
:1039100000253946304600F0EFF900BF14E00025DD
:103920000EE00021242060430B4A126880184155A4
:1039300024206043094A126880184155681CC5B2AA
:10394000242DEED3601CC4B205480078A042E6DC0A
:1039500000F010F8F8BD0000C4070020C8070020E0
:10396000342F0020012002490968087170470000C7
:10397000CC07002010B500F073F900200349096856
:10398000087002490968C87010BD0000CC0700200B
:1039900007480068C078062808D105480068C07943
:1039A000002803D1012002490968C871704700004E
:1039B000CC07002010B555480068C07803000CF013
:1039C000F9FE08671D1A1714110E05665048406865
:1039D000002803D04E4841680020884793E000F05B
:1039E000E5F890E000F0C6F88DE000F0D1F88AE04C
:1039F000FFF7B8FE87E0FFF7C7FD84E04448406862
:103A0000002803D042484168012088473F480068A9
:103A1000407C00281AD03E48C068002803D03C48AB
:103A2000C168C8208847002038490968486237487B
:103A300000680078002804D0042034490968C87060
:103A400024E0022031490968C8701FE02F4800684F
:103A5000406A401C2D49096848622C480068406A49
:103A60007D21C900884211D3002028490968486295
:103A7000264800680078002804D0042023490968FB
:103A8000C87003E0022021490968C8703BE000BF0C
:103A90001F484068002803D01D484168002088471F
:103AA0001A480068407C002813D01948C0680028D4
:103AB00003D01748C168C820884700201349096807
:103AC000486212480068C078401C10490968C870F4
:103AD00018E00E480068406A401C0C4909684862BA
:103AE0000A480068406A7D21C90088420AD3002044
:103AF00006490968486205480068C078401C0349C7
:103B00000968C87000BF00BF10BD0000CC070020CE
:103B1000342F002010B515480068C078072824D03D
:103B2000012012490968487408E01148806800289B
:103B300002D00F4988688047FFF73CFF0B480068B8
:103B4000C0780628F1D109480068007A0028ECD135
:103B500006480068C0790028E7D104480068807AE8
:103B60000028E2D101490968487410BDCC07002043
:103B7000342F002010B5054800680078012802D1D4
:103B8000FDF7F8FE01E0F5F7B3FD10BDCC0700200E
:103B900010B5054800680078012802D1FEF716F933
:103BA00001E0F6F783F910BDCC07002010B51D48E1
:103BB0000068807A002829D11A480068007A002815
:103BC00003D0022017490968887216480068C07936
:103BD000002803D001201349096888721148006841
:103BE0000079012812D100200E49096808710D4999
:103BF0000968887207200B490968C8700A4840683C
:103C0000002803D00848416800208847054800681C
:103C10000078012802D1FEF7B3F901E0F6F720FAA7
:103C200010BD0000CC070020342F002010B5044642
:103C30002146084801F0EEFC07480078002805D12D
:103C4000002C03D032210548FCF760FD02480470C7
:103C500010BD000001030000E200002050C300007E
:103C60000020244909684870AA2022490968887000
:103C700000202049096848621E49096808711D49E9
:103C8000096848711B49096888711A490968C8712F
:103C9000184909680872174909688872154909683E
:103CA000C8721449096808732420124909684873C6
:103CB0001049096888730F490968C87300200D49C5
:103CC000096808740B49096848740A4909688874C6
:103CD00008490968C874074909684861002105480E
:103CE0000068816103480068C161024800680162A0
:103CF00070470000CC07002010B50A780D4B186003
:103D0000034628330C4C23602423534304462834B1
:103D10001B190A4C23600A4C4B6863608B68A360D4
:103D2000CB68E3604B6963610B6923610B78237097
:103D300010BD0000CC070020C4070020C8070020E9
:103D4000342F002007480068C078062808D10548AD
:103D50000068007A002803D101200249096808722E
:103D600070470000CC07002010B50446012C09D193
:103D7000FF2220210020FFF7F5FB0121084604F077
:103D80005BF908E0002220211046FFF7EBFB002141
:103D9000012004F051F910BD10B50024032000F0FB
:103DA0001FFB002801D0012400E00024204610BDA4
:103DB00010B50446032C0ED1FF2215210020FFF779
:103DC000D1FB002214211046FFF7CCFB01210E206D
:103DD00004F032F939E0022C1CD1FCF7B1FF0028C5
:103DE00009D0FF2214210020FFF7BCFB01210E2087
:103DF00004F022F908E0002214211046FFF7B2FB7C
:103E000000210E2004F018F9002215211046FFF7BA
:103E1000A9FB1AE0012C0ED1FF2214210020FFF78C
:103E2000A1FB01210E2004F007F900221521104604
:103E3000FFF798FB09E0002215211046FFF792FBDF
:103E4000002214211046FFF78DFB10BD10B5002491
:103E5000F8F7DEFD094988420DD3FCF7CDFF0028B5
:103E600007D1FCF75DFE012801DD032404E00224F4
:103E700002E0022400E00124204610BDB80B00003F
:103E800010B50446012C09D1FF221D210020FFF7A7
:103E900069FB0121002004F0CFF808E000221D2179
:103EA0001046FFF75FFB0021084604F0C5F810BD7F
:103EB00010B50024022000F093FA002801D001245C
:103EC00000E00024204610BD10B50446012C09D1A5
:103ED000FF221E210020FFF745FB0121092004F0ED
:103EE000ABF808E000221E211046FFF73BFB002143
:103EF000092004F0A1F810BD70B5002400250026AB
:103F0000FCF7CAFC0546FCF7D3FC0646022108482C
:103F1000F7F712F9552800D108E0012E01D100244D
:103F200004E0012D01D1012400E00024204670BDF1
:103F30004C08002010B50446012C09D1FF221F2196
:103F40000020FFF70FFB0121082004F075F808E0BE
:103F500000221F211046FFF705FB0021082004F076
:103F60006BF810BD70B500240025FCF71FFD054659
:103F700003211A48F7F7E0F8552806D1012018491F
:103F8000088000201749088023E01648008801288F
:103F900011D114490880FCF723FC762803DA0120AC
:103FA0000F49088015E0FCF71BFC782811DB002086
:103FB0000B4908800DE001200A490880FCF710FC3D
:103FC000762803DA01200649088002E0002004492F
:103FD000088003480488204670BD00004C0800207B
:103FE000FE0000200001002010B50446012C09D17C
:103FF000FF2221210020FFF7B5FA0121072004F05C
:104000001BF808E0002221211046FFF7ABFA00213F
:10401000072004F011F810BD10B50024FCF7D8FFFC
:10402000012801D1012400E00024204610BD10B574
:104030000446012C09D1FF2216210020FFF792FA35
:104040000121032003F0F8FF08E0002216211046AA
:10405000FFF788FA0021032003F0EEFF10BD10B532
:104060000024052000F0BCF9002801D0012400E064
:104070000024204610BD10B50446012C09D1FF22B2
:1040800019210020FFF76EFA0121052003F0D4FF6B
:104090003CE0022C17D1FCF753FE002809D0FF2288
:1040A00019210020FFF75EFA0121052003F0C4FF6B
:1040B0002CE0002219211046FFF754FA00210520B8
:1040C00003F0BAFF22E0032C17D1FCF73FFE0028D3
:1040D00009D0FF2219210020FFF744FA0121052011
:1040E00003F0AAFF12E0002219211046FFF73AFA66
:1040F0000021052003F0A0FF08E00022192110464E
:10410000FFF730FA0021052003F096FF10BD0000F4
:1041100010B50024FCF72EFD01282FD104211948E9
:10412000F7F70AF8552801D1012428E0FCF7CCFB69
:1041300001280BD0FCF7C8FB022807D0FCF7C4FB12
:10414000032803D0FCF7C0FB052801D1012416E0A9
:10415000FCF7BAFB042801D1022410E0FCF7B4FB01
:10416000062801D103240AE0FCF7AEFB002803D0A7
:10417000FCF7AAFB072802D1002400E00024204617
:1041800010BD00004C08002010B50446012C0ED1D3
:10419000FF221B210020FFF7E5F900221A2110461B
:1041A000FFF7E0F901210A2003F046FF1EE0022C90
:1041B0000ED1FF221A210020FFF7D4F900221B2183
:1041C0001046FFF7CFF901210A2003F035FF0DE07B
:1041D00000221A211046FFF7C5F900221B211046C4
:1041E000FFF7C0F900210A2003F026FF10BD0000F0
:1041F00010B5002410480078012801D1012418E0EE
:10420000FCF7AAFD022803D0FCF7AAFE02280FD172
:10421000FCF774FE012809D1FCF7A4FD012803D0A6
:10422000FCF7A4FE012801D1012402E0022400E0F1
:104230000224204610BD0000E100002010B5F8F770
:1042400001FC0446204610BD10B5034B082203496B
:10425000034800F013F910BD3D420100141902009B
:104260007028002070B506465C488068002804D09D
:104270005A4988688047054600E000250024A6E0EA
:10428000564841680C20604308184088A84207D06F
:10429000524841680C2060430818408802287DD1AC
:1042A0004E4841680C2060430818806800280CD0F4
:1042B0004A494A680C216143511888688047474938
:1042C0000968E2008918487009E0444841680C20F8
:1042D0006043095C41480068E200801841703F4833
:1042E0000068E100401840783C490968E200895CB8
:1042F00088420FD039480068E100401841783748BB
:104300000068E2008154002034490968E2008918FD
:1043100048605AE031480068E100401841782F4871
:1043200042680C2060431018407881421FD12B480E
:104330000068E10040184168284842680C2060434A
:104340001018808881420BD824480068E10040188A
:104350004068801921490968E2008918486034E002
:1043600001201E490968E200891848802DE01B4899
:104370000068E10040184168184842680C2060431A
:104380001018C08881420DD814480068E100401818
:104390004068811911480068E20000E009E08018D7
:1043A000416012E000200D490968E2008918488048
:1043B0000BE0002009490968E200891848800021C3
:1043C00006480068E20080184160601C84B203481F
:1043D0008089A04200DD53E770BD0000EC2E002074
:1043E0000146064A92898A4205DD044A1268CB00DA
:1043F000D218508800E0002070470000EC2E00200A
:10440000002000BF14E00D494A680C2141435118B7
:10441000498801290AD10021084A1268C300D2182C
:104420005180064A1268C300D2185160411C88B2FC
:10443000024989898142E6DC70470000EC2E0020A9
:10444000002000BF13E00C494A680C214143511879
:104450004988002909D1084A1268C300D21851803E
:10446000054A1268C300D2185160411C88B2024943
:1044700089898142E7DC7047EC2E0020F0B50446C4
:104480000020164DAB6069602C60AA8100BF1FE060
:10449000124D6E680C254543755D104E3668C70099
:1044A000F61975700D4D6E680C254543755D0B4E04
:1044B0003668C700F5550025084E3668C700F6195E
:1044C0007580064E3668C700F6197560451CA8B29F
:1044D000024DAD898542DBDCF0BD0000EC2E0020F2
:1044E00070B505460E46002E05D031462846F3F736
:1044F00027FE044600E02C46204670BD10B5FCF7B0
:1045000067FD012817D10C480078012813D00A480C
:10451000007803280FD00948007800280BD1FCF759
:1045200071FC0749884202D108F075F803E07D204C
:10453000000108F077F810BDD5000020D40000205D
:104540008813000008B5002000900122694605206C
:10455000F9F716FE054900988860002004490870A4
:10456000044908700449087008BD0000382800207C
:10457000D4000020D6000020D700002008B500207D
:104580000090012269460520F9F7FAFD0020024952
:1045900008710098886008BD3828002070B5049C18
:1045A0002578914216DD01280AD18D4206DAFF26D0
:1045B000F61AAE420ED3EE18F5B20BE0154609E03E
:1045C000022807D1954204DD9D4203DBEE1AF5B2C5
:1045D00000E00D46257070BD0D4A4168516081694B
:1045E0009161C168D160416A5162016A11620168DA
:1045F00011604169516181689160C169D16101694E
:104600001161816A91620021024A117070470000B5
:10461000082F0020C007002010B5FFF7F1FEF8F7C3
:1046200057F800210148F6F791FE10BD5808002008
:1046300010B5F8F74DF8FFF703FF0AF0A1F80AF0FC
:104640003DF9FBF7A9FBFAF7D7F8FFF77BFFF8F77F
:1046500079FCF6F777FCF9F76DF955210548F6F77F
:1046600075FEF8F7A7FAF9F7E3F8FBF755F8F6F750
:1046700063FE10BD580800201CB5002033490870A7
:1046800008F0A2F80020FCF7E3FC0CF0BBFBF7F706
:10469000C5F9F8F78FFAF9F7CBF8F6F74BF8F6F714
:1046A000C9FAE12040020BF0EFFF00F079FAF6F7CB
:1046B00049FC08F069FAF8F70BF8F9F7E3FEF8F7A8
:1046C000CDFCF8F74BFCFFF7BFFDFEF75DF8FFF7F9
:1046D000F9F8FFF71FFAF9F7DBFDFBF789FBFAF7AB
:1046E0008BF81B4AFF21913101200AF0ADF900221D
:1046F000114601200AF0ECF807F0D4FF0AF026F882
:104700000AF0DCF8FFF73AFFF9F744F90020114905
:1047100088714871087101208870487014200870F1
:1047200007226846F3F7A3FD0199009800F0C2FF45
:104730000221012000F09AFEFAF7EEFFF6F7FCFDE9
:1047400055210548F6F702FE1CBD0000E1000020DF
:104750000090D003F20000205808002070470000AD
:1047600010B50446552C03D105494869804702E03D
:1047700003490868804700200249087010BD000006
:10478000082F0020C007002010B54648007803001D
:104790000CF010F80A06111B26303B46505173816D
:1047A00041484068002802D03F49486880470120BE
:1047B0003C49087000BF3C488068002804D03A4952
:1047C000886880473749087069E03748C068002822
:1047D00002D03549C868804703203249087000BFBD
:1047E00031480069002804D02F49086980472D49C5
:1047F000087054E02C484069002802D02A494869D2
:10480000804700202749087049E027488069002830
:1048100002D025498869804706202249087000BFD8
:104820002148C069002804D01F49C86980471D4934
:10483000087034E000BF1B48007807280AD11A48E6
:10484000006A002802D01849086A804709201549E3
:10485000087011E01348007808280AD11248406A0D
:10486000002802D01049486A804709200D49087085
:1048700002E000200B49087000BF0A4800780028B9
:1048800008D00948806A002804D00749886A804710
:104890000449087003E000200249087000BF00BF0F
:1048A00010BD0000C0070020082F00207047000046
:1048B00010B500200CF062FB09F040F809F094F804
:1048C00009F0AAF800F0C6FCF6F744FA0220FCF75B
:1048D000BFFB002007490870FFF71CF9FFF742F8FB
:1048E000FFF768F8F6F796F810200AF0C3FC00F01E
:1048F000B1FD10BD9401002010B5012408F0ECFBBF
:10490000012801D1052407E0F8F77CF80349884223
:1049100001D2012400E00224204610BD204E0000F8
:1049200010B5062408F0D8FB002800D1002408F0B8
:10493000D9FB012803D008F0D5FB072800D90924AA
:10494000204610BD10B5F6F705FA002211460120E9
:104950000AF0F0F800213C48F6F7F8FC00203B494B
:104960000880002400BF00F02FFF32217D200001CD
:10497000FBF7CCFE0020364908700AE000223448DC
:1049800001781046FEF7EEFD31480078401C3049B2
:1049900008702F4800782428F0DB00202D4908708B
:1049A00009E000212B48007809F0D8FC294800785C
:1049B000401C28490870274800780D28F1DBFEF7D5
:1049C000F9FFF5F7FDFE08F0D9FA23480078401CFE
:1049D0002149087008460078052812D30020087085
:1049E000FEF7D6FF1D4800780A2805D300201B4992
:1049F0000870FFF7A7F904E018480078401C174931
:104A0000087008F06FFB0128ADD908F06BFB072890
:104A1000A9D200200F49087008E00E48007809F07C
:104A2000B7FC0C480078401C0A4908700948007817
:104A30000D28F2DBF6F7FEF855210348F6F786FC61
:104A4000F7F7B6FF204610BD580800207C00002074
:104A5000FB000020F9000020FA000020FC000020EC
:104A600010B5032408E000F0AFFE012000F0B6FD11
:104A7000002801D0042400E0F5E700BF204610BD67
:104A800010B500202A49086007F09EFE0120FCF7BF
:104A9000DFFAF6F7C3FF55212648F6F757FCF8F77B
:104AA00089F8F8F7C5FE0CF0ADF9F5F743FEF9F714
:104AB000B1FCF6F7BFF808F071FAF9F7E3FCF9F783
:104AC0007FFEF8F7CBFAFFF7BFFBFDF75DFEFFF7C0
:104AD000B7FCFFF737FDFEF7F5FEFFF71BF800F018
:104AE0005FF8E12040020BF0CFFDF6F72BFAFBF761
:104AF0007FF9F9F781FE104AFF219131012009F079
:104B0000A3FF00221146012009F0E2FE09F01EFE7B
:104B100009F0D4FEF8F70EFF0221012000F0A6FCF8
:104B2000FAF7FAFD07F0E0FDF6F706FC10BD00000D
:104B300050000020580800200090D00370B50646B1
:104B40000D4614460E4806600E4805600E49206862
:104B500008600E49606808600D49A06808600D494A
:104B6000206908600C49E06808600C4960690860C9
:104B700005480068002802D003480068804770BDDF
:104B8000A8000020B0000020900000209400002029
:104B9000980000209C000020A0000020A40000201D
:104BA00000B587B00C4801900C4802900C48039067
:104BB0000020049005900B48069000200A490860E8
:104BC00048600A490860486001AA0121C9020848F2
:104BD000FFF7B4FF07B000BDF54B0100994F01008E
:104BE000214F01004D4E01006C120020640A00208C
:104BF0007417002001207047F3B5C3B00446449EEB
:104C00000020009057E002E0641C761E00BF022ED8
:104C100005D32078EB28F7D160789028F4D1072EBF
:104C200000D24AE0A778FD1CB54200D945E0A81E95
:104C3000205C0002691E615C08434290042D38D953
:104C4000291FA01C0CF0F8F84299884226D11D4873
:104C50000068002804D0B91EE01C1A4A1268904768
:104C600019480068002824D0E1786846017120794D
:104C700081116846417120798106890E68468171EB
:104C8000381FC1B26846C171C279611D02A8F3F72D
:104C9000EEFA01A80C49096888470AE00020009054
:104CA00002E00098401C00900098A842F9D3002030
:104CB00000906419761B072EA5D200BF4498801B74
:104CC00045B0F0BD9C000020A4000020F7B5C0B0A6
:104CD000154600260027E81DFF210131884202DD2C
:104CE000002043B0F0BDEB21684601709021417077
:104CF000281DC1B2684681700021C1704098C1B2C0
:104D0000684601710524002605E04198805D6946EA
:104D10000855641C761CAE42F7DBA11E00A80230C9
:104D20000CF08AF80746381269460855641C0F557E
:104D3000641C06480068002805D021466846034ADE
:104D400012689047CDE70020CBE7000094000020D8
:104D500070B50024002500261B4840681A490968E0
:104D6000884200D170BD18484068174909688842D8
:104D700005D91548406814490968451A07E01248E2
:104D8000006811494968401A012189020D1AFF2D56
:104D900001D9FF2600E02E4600240DE00A480168F4
:104DA0000830405C0949085507480088401C8005C8
:104DB000800D05490860641CB442EFD3B1B20348CA
:104DC0000BF0BEFC00BFCDE76C1200207416002073
:104DD00070B500251A480068002830D0194A12889A
:104DE000FF230133991A184A1268164B1B88D018F2
:104DF000134A126890470546002D20D011480088BC
:104E0000401910490880084601880F480068FFF7DC
:104E1000F3FE0446002C0DDD0A480088844209DABE
:104E200008480088021B0848006801190648006805
:104E3000F3F71DFA03480088001B0249088070BD83
:104E400098000020AC000020A800002038B50446DF
:104E500000200090A07810280CD120792D490870EE
:104E600008460078012853D1002211462020FFF780
:104E70002DFF4DE0A078122803D120792549087232
:104E800046E0A078052803D12079224988723FE0C6
:104E9000A07802281DD120791E4948720846407A20
:104EA000012806D10090012269460420FFF70EFF79
:104EB0002EE01848407A02282AD100BFBFF34F8F56
:104EC00015481649C860BFF34F8F00BF00BF00BF31
:104ED000FDE7A07801281BD12079332803D10120D8
:104EE0000C49487005E02079352802D10020094995
:104EF0004870607907498870607A0006217A090451
:104F00000843E17909020843A1790843014948604F
:104F100038BD0000580A00200400FA0500ED00E04A
:104F200070B503460022002400251A484068194E37
:104F30003668B04201D1002070BD16484068154E59
:104F40003668B04205D913484068124E3668841B53
:104F500007E0104800680F4E7668801B0126F602B5
:104F6000341AA14201D9254600E00D4600220CE08A
:104F7000084806680830805D985406480088401C40
:104F80004005400D034E3060521CAA42F0D3284623
:104F9000D2E70000640A002070B503460022002416
:104FA00015484068144D2D68A84208D3124840683F
:104FB000114D2D68401B0125AD022C1A04E00E484E
:104FC00000680D4D6D68441BA14201D9012070BDE0
:104FD00000220CE09D5C084846680830855508387A
:104FE0008088401C8005800D034D6860521C8A42F9
:104FF000F0D30020EBE700006C12002010B502484F
:10500000FFF7EAFA10BD0000FC1902000021014A76
:105010001175704740600040014600BFF020084015
:1050200000110A23584302460807000F8018C0B237
:1050300070470146002204E0501CC2B208460A38FC
:10504000C1B20A29F8DA1007000E084370470000C1
:1050500010B5044601218020F6F7FAF9607A01289C
:1050600005D14248C078102108434049C870607A91
:10507000A22805D13E48007F802108433C4908779B
:10508000607A3B49087700203A4948770846407FD4
:105090002178084337494877E07B002805D0084647
:1050A000407F20210843334948773248407FC00879
:1050B000C000A17A08432F4948770846807FF7212E
:1050C00008402C498877E078FFF7B3FF29498874B6
:1050D000A078FFF7AEFF2749C8746078FFF7A9FFF3
:1050E000244908752078002805D10846007D2179DB
:1050F000084320490875E079FFF79BFF1D49887533
:105100006079FFF796FF1B494875A079FFF791FF7B
:105110001849C875207AFFF78CFF164908760846AB
:10512000807F4006400E8877E07A002806D0084647
:10513000807F402108430F49887703E00D48807F36
:105140000C498877A07BFFF774FF0A498876607B5B
:10515000FFF76FFF0749C876207B08770846807FF6
:10516000102188430349887710BD000020040240C5
:1051700060040440404F044010B504461B48807F43
:1051800001210843194988772078FFF752FF174912
:1051900008756078FFF74DFF1449C874A078FFF7D1
:1051A00048FF1249887420780C2806DD0846407FA5
:1051B000082108430D49487709E00C48407F0B4916
:1051C00048770846007DE178084308490875074894
:1051D000807F400840000549887700BF0348807FF2
:1051E000022108400028F9D110BD0000404F0440C2
:1051F00010B500201449087616200BF001FB0021A1
:10520000124801761248407F8021084310494877B0
:105210000846807F012108430D49887700BF0C486C
:10522000807F022108400028F9D00948807F40088B
:1052300040000749887700BF0548807F0221084069
:105240000028F9D110BD00004060004040610040DE
:10525000404F044010B5002007490870002120206D
:10526000F6F7F6F801210548017500200449087594
:1052700015200BF0ADFA10BD005004404061004015
:105280004060004070B504460D46002C14D0002D3F
:1052900012D0042D10D800F013F800280CD10026ED
:1052A00008E00649885D22460121F4F75FF8A41C56
:1052B000701CC6B2AE42F4DB70BD0000781902006B
:1052C00000200549897DC907C90F002901D00120A7
:1052D00000E00020704700000050044030B585B069
:1052E00005460C4600200390049000900190029027
:1052F000072C0BDC0120A04081B26846818101218E
:10530000C17303A90220FAF7B3FE3EE0082C01D0D6
:10531000092C0BD10120A04081B268468181012176
:10532000C17303A90120FAF7A3FE2EE00A2C03D0D3
:105330000B2C01D00D2C0BD10120A04081B268466E
:1053400081810121C17303A90020FAF791FE1CE0BD
:105350000C2C01D00F2C0BD10120A04081B268464B
:1053600081810121C17303A90E20FAF781FE0CE0AF
:105370000E2C0AD10120A04081B268468181012112
:10538000C17303A90C20FAF773FE0021684601706F
:10539000C17041700121817000210171C1720D2124
:1053A0008172FF21017200214172F4F73FF8034935
:1053B0001520FDF7B3F805B030BD00000D50010019
:1053C00010B500201049087515200BF001FA0021D6
:1053D0000E4801751520002809DB00BF00BFC2067A
:1053E000D20E012191400A4A116000BF00BF00BFE8
:1053F000084880798011032805D00648007880216C
:1054000008430449087010BD4060004040610040FE
:1054100000E100E00050044010B5F4F701F910BDC0
:1054200010B501231A4600211846F5F7CDFF0122D9
:1054300011461046F6F73EF8F6F72AF803480BF047
:10544000D3FC02480249086010BD00000090D00360
:105450004407002000BF04480069042108430249B2
:10546000086130BF00BF704700ED00E0F3B585B0C4
:105470000546002400270026002003900490EEB289
:105480002804070E0F2F54DA082E52DA002009E004
:105490000C214143284A515AA94201D1044603E054
:1054A000411CC8B21728F3D300BF0120B04086B218
:1054B0000C20604320494018C3780C2060434018FA
:1054C0008278F8B231460190FAF776FE6846868116
:1054D000012181730021C17302214174F8B203A933
:1054E000FAF7C6FD0C216143134A8918C888FBF7F7
:1054F000D5FE0C20604310494018C18868460181E0
:1055000069460698887202A8FBF7E2FD0C22624306
:10551000094BD21891680C226243D218042010560D
:10552000FCF7FCFF0C216143034A8918C888FBF78C
:1055300039FE07B0F0BD0000941B0200FEB5054621
:105540000C460020C0430290EFB22804060E0F2E36
:1055500042DA082F40DA0120B840694608808020EE
:105560002040002816D101208870A007800F022853
:1055700001D1487109E0A007800F012802D16946D6
:10558000487102E0002069464871F0B26946FAF7B6
:105590006FFD1FE00020694688700E202040002823
:1055A00000D000BF10202040002802D169460871B9
:1055B00002E0012069460871E007C00F002802D10F
:1055C0006946887102E0012069468871F0B2694637
:1055D000FAF74EFD002002900298FEBD30B501465C
:1055E000CAB20C04230E00200F2B0FDA082A0DDAA2
:1055F00001249440A2B2064C03252D026419E45CF8
:105600001440002C01D0012000E0002030BD00003B
:1056100000000440F8B504460F460020C043009047
:10562000E6B22004050E0F2D11DA082E0FDA012044
:10563000B04086B2002F04D1E8B23146FAF714FE2A
:1056400003E0E8B23146FAF71FFE00200090009810
:10565000F8BD00001649897F01221143144A917751
:1056600000BF1349897F022211400029F9D0104957
:10567000897C81700E49C97C41700D49097D01709A
:105680000B498A7D8271497D01710949CA7D427148
:105690000A7EC271897F49084900054A917700BF97
:1056A0000349897F022211400029F9D17047000087
:1056B000404F044003B585B0002001900290039054
:1056C0000490002168464173817E01A8C17068463C
:1056D000417E01A881706846017E4171002101A8C8
:1056E0000171082168460171817D01A8C171684678
:1056F000C17D4172417D01A881716846017D01A88B
:105700000172002168468173C17301A881730C2165
:1057100041734121684601740021C17401A8FFF75B
:1057200097FC1A200449888204491620FCF7F6FEEB
:1057300000F006F807B000BD204F0440350F02000E
:1057400010B5FFF755FD10BD70B504460D46601E3F
:105750000D49884200D90124002C00D101244020A9
:105760000A490870084600786043094948610321E6
:10577000081F0BF05DF800200549886107200861CB
:105780000448056070BD0000FFFFFF0070010020AD
:1057900000E000E06C0100200020C043002809DB8D
:1057A000C206D20E01219140054A1160BFF34F8F0E
:1057B000BFF36F8F00BF0020024908618861704706
:1057C00080E100E000E000E010B50AF0D7FF10BD76
:1057D0001A20084908722B2048723C2088724D20FC
:1057E000C8727F20044909680860AC2003494870EA
:1057F00070470000000402407401002000100240C5
:1058000010B51C480078012812D11B480078642884
:1058100009DB0220194948710871002016490870F7
:105820001449087004E014480078401C12490870BC
:105830001348007801281CD112480078012804D1AF
:10584000002010490870104908700F48007832286D
:105850000ADBF7F7F7F900210C48F5F727FD55218A
:105860000B48F5F773FD04E007480078401C064933
:10587000087010BD1107002010070020000700204D
:105880000A0700200C0700200B0700204C0800200E
:1058900058080020F8B504460D4600270020009067
:1058A00003200003204000130090102C04D0122C81
:1058B00002D01148844217D122202840222806D144
:1058C00027073F0F39460098F4F720FF06461220BD
:1058D000284012280ED12007000F471C3946009897
:1058E000F4F714FF064605E02107090F0098F4F7C6
:1058F0000DFF06463046F8BD10100000F8B504460E
:105900000D46002600270120000320400713102C1D
:1059100004D0122C02D00F48844215D122202840F6
:10592000222805D12607360F31463846FAF798F86F
:105930001220284012280CD12007000F461C3146A7
:105940003846FAF78DF804E02107090F3846FAF7D0
:1059500087F8F8BD10100000FFB58BB01C46002082
:105960000790069005903848049010210B98084045
:10597000002801D0022707E040210B9808400028AA
:1059800001D0012700E00027002C04D014980470F7
:105990000120089001E010200890002548E0002C2C
:1059A00008D025466000294A115A0C98F2F7C8FB26
:1059B000079006E06800254A115A0C98F2F7C0FBE0
:1059C00007903E4630E0711C0798F2F7B9FB40089B
:1059D00006900D98F2F70AFD03900D9A0699881A21
:1059E000F2F704FD18490190F2F785FC0290039943
:1059F000F2F7BEFC05900598F2F7FFFC4900490854
:105A0000039102900498F2F7F8FC490049080191CB
:105A10000090039B029AF2F705FD03D20A950996BE
:105A200005980490701CC6B27F2ECCDD681CC5B2F0
:105A300008988542B3DB14990A980870149909985C
:105A4000487004980FB0F0BD0000C842A81C0200C6
:105A50000246412A2ED010DC212A2AD006DC102A48
:105A600045D0122A4BD0202A59D11CE0222A26D018
:105A7000232A2AD0402A52D116E081235B01D01A72
:105A80009A4228D008DC422A1AD0432A1ED0254840
:105A90001018002843D13AE0012822D020281BD03A
:105AA00021283CD11EE000BF1F4803890B4303811E
:105AB00036E000BF1C4843890B43438130E000BF00
:105AC000194883890B4383812AE000BF1648C389A4
:105AD0000B43C38124E000BF144883880B438380B9
:105AE0001EE000BF1148C3880B43C38018E00E4876
:105AF00043890B43438103890B43038110E00A4828
:105B0000C3890B43C38183890B43838108E0074822
:105B1000C3880B43C38083880B43838000E000BFAE
:105B200000BF7047F0EFFFFF001104400014044075
:105B3000F0B505460E46412D30D010DC212D2CD07D
:105B400006DC102D51D0122D56D0202D62D11CE034
:105B5000222D2AD0232D30D0402D5BD116E081217B
:105B60004901681A8D4230D008DC422D1ED0432DE9
:105B700024D02A48281800284CD144E001282CD0F1
:105B8000202823D0212845D128E000BF244F388881
:105B9000314600F049F804463DE000BF204F7888C8
:105BA000314600F041F8044635E000BF1C4FB8888C
:105BB000314600F039F804462DE000BF184FF88850
:105BC000314600F031F8044625E000BF154F388813
:105BD000314600F029F804461DE000BF114F7888D7
:105BE000314600F021F8044615E00D4F7888314623
:105BF00000F01AF804460EE0094FF888314600F02C
:105C000013F8044607E0074F7888314600F00CF897
:105C1000044600E000BF00BF2046F0BDF0EFFFFFEC
:105C200000110440001404400246002013460B40BB
:105C3000002B01D0012000E000207047FFB581B0AB
:105C40000E461746012F07D1F748407D0009000195
:105C5000C01DF549487505E0F348407D0009000185
:105C6000F1494875049801287ED10A210198F2F77C
:105C700067FA0546ED48445DE007C00F002807D0ED
:105C8000E948007C00090001C01DE749087405E0EF
:105C9000E548007C00090001E34908740220204027
:105CA000002807D0E048C07BF02188437030DE49EF
:105CB000C87305E0DC48C07BF0218843DA49C8732B
:105CC00004202040002807D0D748807C000900012C
:105CD000C01DD549887405E0D348807C00090001C7
:105CE000D149887408202040002807D0CE48407C45
:105CF000F02188437030CC49487405E0CA48407CA4
:105D0000F0218843C849487410202040002807D05B
:105D1000C548407C00090001C01DC349487405E026
:105D2000C148407C00090001BF4948742020204040
:105D3000002807D0BC48007CF02188437030BA4965
:105D4000087405E0B848007CF0218843B64908741F
:105D500040202040002808D0B348807CF0218843B0
:105D60007030B149887406E08BE0AF48807CF02148
:105D70008843AD4988740A210198F2F7E1F90D468C
:105D8000AA48445DE007C00F002807D0A648807BE2
:105D9000F02188437030A449887305E0A248807BD5
:105DA000F0218843A049887302202040002807D0B2
:105DB0009D48807B00090001C01D9B49887305E058
:105DC0009948807B0009000197498873042020408E
:105DD000002807D09448007DF02188437030924914
:105DE000087505E09048007DF02188438E490875CC
:105DF00008202040002807D08B48007D00090001C2
:105E0000C01D8949087505E08748007D000900012B
:105E10008549087510202040002807D08248C07CA2
:105E2000F021884370308049C87405E07E48C07C0A
:105E3000F02188437C49C87420202040002807D0E6
:105E40007948C07B00090001C01D7749C87305E08F
:105E50007548C07B000900017349C8734020204089
:105E6000002807D07048C07C00090001C01D6E49A1
:105E7000C87454E06C48C07C000900016A49C874C9
:105E80004DE06948007C0009000167490874084634
:105E9000C07BF02188436449C8730846807C0009B0
:105EA000000188740846407CF02188435E494874AC
:105EB0000846407C0009000148740846007CF02137
:105EC0008843594908740846807CF0218843564924
:105ED00088740846807BF0218843534988730846BC
:105EE000807B0009000188730846007DF02188430B
:105EF0004D4908750846007D0009000108750846EF
:105F0000C07CF02188434849C8740846C07B00091A
:105F10000001C8730846C07C00090001C8740A98D3
:105F200001287DD10A213046F2F70AF905463F489B
:105F3000445DE007C00F002807D03B48407B0009C4
:105F40000001C01D3849487305E03748407B00090F
:105F500000013549487302202040002807D032480C
:105F6000007BF021884370302F49087305E02E48EC
:105F7000007BF02188432C4908730420204000282E
:105F800007D02948807DF0218843703026498875E4
:105F900005E02548807DF021884323498875082045
:105FA0002040002807D02048807D00090001C01D46
:105FB0001D49887505E01C48807D000900011A49CB
:105FC000887510202040002807D01748407DF02118
:105FD000884370301449487505E01348407DF0212E
:105FE00088431149487520202040002807D00E48DA
:105FF000407BF021884370300B49487305E00A4824
:10600000407BF02188430849487340202040002805
:106010000ED00548C07D00090001C01D024900E006
:1060200092E0C8750AE0000048260020E816020049
:106030006D48C07D000900016B49C8750A213046D2
:10604000F2F77EF80D466948445DE007C00F00286E
:1060500007D06548C07AF021884370306249C87221
:1060600005E06148C07AF02188435F49C872022088
:106070002040002807D05C48C07A00090001C01DFC
:106080005949C87205E05848C07A000900015649CC
:10609000C87204202040002807D05348407E0009E1
:1060A0000001C01D5049487605E04F48407E000978
:1060B00000014D49487608202040002807D04A4872
:1060C000007EF021884370304749087605E0464855
:1060D000007EF021884344490876102020400028A3
:1060E00007D04148007E00090001C01D3E490876E6
:1060F00005E03D48007E000900013B49087620206C
:106100002040002807D03848007B00090001C01D4E
:106110003549087305E03448007B00090001324925
:10612000087340202040002807D02F48C07DF02170
:10613000884370302C49C87554E02B48C07DF0214D
:1061400088432949C8754DE02748407B0009000174
:10615000254948730846007BF0218843224908738B
:106160000846807DF02188431F4988750846807D58
:106170000009000188750846407DF02188431A49CE
:1061800048750846407BF021884317494873084604
:10619000C07D00090001C8750846C07AF021884317
:1061A0001149C8720846C07A00090001C872084641
:1061B000407E0009000148760846007EF0218843B1
:1061C000094908760846007E00090001087608465D
:1061D000007B0009000108730846C07DF021884358
:1061E0000149C87505B0F0BD48260020E816020038
:1061F000FFB581B00E461746019801287ED104985C
:10620000002826D1FA480078012822D0F6F700FCB1
:10621000F84988421DD3FAF793FD00280DD0F648BF
:10622000807DF02188437030F34988750846C07C32
:1062300000090001C01DC87418E0EF48807DF021FE
:106240008843ED4988750846C07C00090001C87480
:106250000CE0E948807DF02188437030E64988757C
:106260000846C07C00090001C01DC874E248C07C1B
:10627000F02188437030E049C8740846007EF02160
:1062800088437030DC4908760846807D00090001AB
:10629000401C88750846407DF02188431030D6495F
:1062A00048750846407D00090001401C48750846B5
:1062B000007DF02188431030CF4908750846007DE5
:1062C00000090001401C087533000AF073FA062E1D
:1062D000261E140C042FC848007D00090001C01DB3
:1062E000C549087500BFC448007DF021884370305F
:1062F000C149087500BFC048407D00E0ADE100091C
:106300000001C01DBC49487500BFBB48407DF0215D
:1063100088437030B849487500BFB748807D000990
:106320000001C01DB449887500BF00E000BF00BF78
:10633000049800285ED1AE48007801285AD0F6F7BC
:1063400067FBAC49884255D3AB48C07FF0218843F6
:10635000A949C8770846807F000900018877084668
:10636000407FF0218843A44948770846007FF02108
:106370008843A14908770846C07DF02188439E499B
:10638000C8750846C07F00090001C8770846807FAD
:10639000F0218843984988770846407F000900012A
:1063A000C01D48770846807EF02188439249887650
:1063B0000846807E0009000188760846407E000974
:1063C000000148760846007E00090001087608466C
:1063D000007F0009000108770846C07EF02188434D
:1063E0008549C8760846407EF0218843703082494E
:1063F0004876B8E164213846F1F7A2FE0546012D42
:1064000007D17D48C07FF021884370307A49C87732
:1064100005E07948C07FF02188437749C8770A2191
:106420003846F1F78DFE0A210090F1F789FE0D46FE
:10643000642F02D37148445D01E07148445DE00778
:10644000C00F002807D06C48807F00090001C01DE4
:106450006949887705E06848807F0009000166493E
:10646000887702202040002807D06348407FF02131
:10647000884370306049487705E05F48407FF021ED
:1064800088435D49487704202040002807D05A48B7
:10649000007FF021884370305749087705E056485F
:1064A000007FF021884354490877082020400028C5
:1064B00007D05148C07DF021884370304E49C875DF
:1064C00005E04D48C07DF02188434B49C875102038
:1064D0002040002807D04848C07F00090001C01DA7
:1064E0004549C87705E04448C07F0009000142499A
:1064F000C87720202040002807D03F48807FF02127
:10650000884370303C49887705E03B48807FF02124
:1065100088433949887740202040002807D03648F2
:10652000407F00090001C01D3349487705E032482B
:10653000407F00090001304948770A213846F1F7C9
:10654000FFFD0D462D48445DE007C00F002807D031
:106550002948807EF021884370302749887605E0FD
:106560002548807EF02188432349887602202040F8
:10657000002807D02048807E00090001C01D1E4968
:10658000887605E01C48807E000900011A4988765B
:1065900004202040002807D01748407E0009000151
:1065A000C01D1549487605E01348407E00090001EA
:1065B0001149487608202040002807D00E48007E68
:1065C00000090001C01D0C49087605E00A48007E5C
:1065D000000900010849087610202040002811D049
:1065E0000548007F00090001C01D034908770FE03E
:1065F000E1000020B80B00001C270020E816020074
:10660000FB1602005948007F00090001574908772E
:1066100020202040002807D05448C07EF021884325
:1066200070305249C87605E05048C07EF02188435A
:106630004E49C87640202040002807D04B48407E75
:10664000F02188437030494948768CE04748407EC5
:10665000F02188434549487685E04448807D00091B
:106660000001424988750846407DF02188433F4932
:1066700048750846407D0009000148750846007DC0
:10668000F0218843394908750846007D000900015A
:1066900008750846C07C00090001C8740846807D62
:1066A000F0218843314988750846C07CF021884331
:1066B0002E49C8740846007EF02188432B4908768D
:1066C0000846C07FF02188432849C8770846807F64
:1066D0000009000188770846407FF021884323495C
:1066E00048770846007FF02188432049087708460C
:1066F000C07DF02188431D49C8750846C07F000948
:106700000001C8770846807FF021884317498877C1
:106710000846407F0009000148770846807EF02146
:106720008843124988760846807E000900018876F1
:106730000846407E0009000148760846007E0009B0
:10674000000108760846007F000900010877084626
:10675000C07EF02188430549C8760846407EF02176
:1067600088430249487605B0F0BD00001C27002090
:1067700010B50146002200200A0EFE4B985CC307AC
:10678000DB0F002B07D0FC4BDB7FF024A3437033DF
:10679000F94CE37705E0F84BDB7FF024A343F64C9C
:1067A000E37702230340002B07D0F34BDB7F1B0969
:1067B0001B01DB1DF04CE37705E0EF4BDB7F1B0992
:1067C0001B01ED4CE37704230340002B07D0EA4B79
:1067D0009B7F1B091B01DB1DE74CA37705E0E64B04
:1067E0009B7F1B091B01E44CA37708230340002B6C
:1067F00009D0E14B20335B781B091B01DB1DDE4C0C
:106800002034637007E0DC4B20335B781B091B01ED
:10681000D94C2034637010230340002B09D0D64B91
:1068200020331B78F024A3437033D34C20342370DF
:1068300007E0D14B20331B78F024A343CE4C203407
:10684000237020230340002B09D0CB4B20331B782F
:106850001B091B01DB1DC84C2034237007E0C64B0D
:1068600020331B781B091B01C34C203423704023A9
:106870000340002B07D0C04B9B7FF024A343703311
:10688000BD4CA37705E0BC4B9B7FF024A343BA4CDF
:10689000A377FF231B040B401A0CB64B985CC3076D
:1068A000DB0F002B07D0B44B1B7F1B091B01DB1D2B
:1068B000B14C237705E0B04B1B7F1B091B01AE4C8D
:1068C000237702230340002B07D0AB4BDB7EF02461
:1068D000A3437033A84CE37605E0A74BDB7EF0249E
:1068E000A343A54CE37604230340002B07D0A24B1F
:1068F0009B7EF024A34370339F4CA37605E09E4B10
:106900009B7EF024A3439C4CA37608230340002BDA
:1069100007D0994B5B7FF024A3437033964C637789
:1069200005E0954B5B7FF024A343934C63771023E2
:106930000340002B07D0904B5B7F1B091B01DB1D25
:106940008D4C637705E08C4B5B7F1B091B018A4CE8
:10695000637720230340002B07D0874B1B7FF02455
:10696000A3437033844C237705E0834B1B7FF024D3
:10697000A343814C237740230340002B07D07E4B59
:10698000DB7E1B091B01DB1D7B4CE37605E07A4BAC
:10699000DB7E1B091B01784CE376FF231B020B40B7
:1069A0001A0A744B985CC307DB0F002B07D0724B9D
:1069B0001B7EF024A34370336F4C237605E06E4BAF
:1069C0001B7EF024A3436C4C237602230340002B50
:1069D00007D0694B1B7E1B091B01DB1D664C237610
:1069E00005E0654B1B7E1B091B01634C23760423CA
:1069F0000340002B07D0604BDB7D1B091B01DB1D17
:106A00005D4CE37505E05C4BDB7D1B091B015A4CBB
:106A1000E37508230340002B07D0574B9B7E1B09CF
:106A20001B01DB1D544CA37605E0534B9B7E1B09D9
:106A30001B01514CA37610230340002B07D04E4B73
:106A40005B7EF024A34370334B4C637605E04A4BE6
:106A50005B7EF024A343484C637620230340002B45
:106A600007D0454B5B7E1B091B01DB1D424C637647
:106A700005E0414B5B7E1B091B013F4C63764023C5
:106A80000340002B07D03C4BDB7DF024A343703345
:106A9000394CE37505E0384BDB7DF024A343364CDD
:106AA000E375CAB2334B985CC307DB0F002B07D0EA
:106AB000314B1B7DF024A34370332F4C237505E02D
:106AC0002D4B1B7DF024A3432B4C23750223034045
:106AD000002B07D0284B1B7D1B091B01DB1D264CFF
:106AE000237505E0244B1B7D1B091B01224C2375DC
:106AF00004230340002B07D01F4BDB7C1B091B0129
:106B0000DB1D1D4CE37405E01B4BDB7C1B091B01EB
:106B1000194CE37408230340002B07D0164B9B7CD1
:106B2000F024A3437033144CA37405E0124B9B7CF8
:106B3000F024A343104CA37410230340002B07D070
:106B40000D4B5B7DF024A34370330B4C637505E064
:106B5000094B5B7DF024A343074C6375202303405E
:106B6000002B0BD0044B5B7D1B091B01DB1D024C72
:106B7000637509E0E8160200FC2600200C4B5B7DE3
:106B80001B091B010A4C637540230340002B07D0EF
:106B9000074BDB7CF024A3437033054CE37405E022
:106BA000034BDB7CF024A343014CE37410BD0000D5
:106BB000FC26002000B501287ED1FE4AD278F023C1
:106BC0009A437032FB4BDA701A461279120912019D
:106BD000D21D1A711A461279F0239A437032F54B7E
:106BE0001A711A46527912091201D21D5A711A46A7
:106BF0005279F0239A437032EE4B5A711A46D27989
:106C000012091201D21DDA711A46D279F0239A4381
:106C10007032E84BDA711A46527A12091201D21D0B
:106C20005A721A46527AF0239A437032E14B5A72E2
:106C30001A46927AF0239A437032DE4B9A721A46C1
:106C40009278F0239A437032DA4B9A701A46D27ACD
:106C500012091201D21DDA721A4652781209120173
:106C6000D21D5A701A46D27AF0239A437032D14B11
:106C7000DA721A46203AD27FF0239A437032CD4B13
:106C8000203BDA77CB4A127B12091201D21D203346
:106C90001A731A46203A927F12091201D21D203B24
:106CA0009A77C44A127BF0239A437032C14B1A730D
:106CB0001A46203A127F00E0F2E1F0239A43703244
:106CC000BC4B203B1A77BB4A527B12091201D21DE2
:106CD00020335A731A46203AD27E12091201D21D6D
:106CE000203BDA76B44AD278F0239A437032B24B22
:106CF000DA701A46127B12091201D21D1A731A4653
:106D0000127912091201D21D1A711A46927AF023D1
:106D10009A437032A84B9A721A461279F0239A431A
:106D20007032A54B1A711A46527912091201D21DFE
:106D30005A711A46927912091201D21D9A711A4695
:106D4000127A12091201D21D1A721A46127AF0230F
:106D50009A437032984B1A721A46527A12091201EB
:106D6000D21D5A72934A927912091201521C914B08
:106D70009A711A469279F0239A4310328D4B9A7188
:106D80001A46127A12091201521C1A721A46127A03
:106D9000F0239A431032874B1A721A46927A1209DC
:106DA0001201521C9A721A46D27812091201521C10
:106DB000DA701A46927812091201521C9A701A4619
:106DC0005278F0239A4310327A4B5A701A4612784E
:106DD000F0239A431032774B1A701A461278120930
:106DE0001201521C1A701A46203AD27F120912015F
:106DF000521C203BDA771A46927FF0239A431032D6
:106E00006C4B203B9A771A46527FF0239A431032FC
:106E1000684B203B5A771A46527F12091201521CC6
:106E20005A771A46127F12091201521C1A771A4613
:106E3000D27EF0239A4310325E4B203BDA761A461C
:106E4000927EF0239A4310325A4B203B9A765A4A4C
:106E5000127BF0239A431032574B1A731A46D27A98
:106E6000F0239A431032544BDA721A46D27A12093E
:106E70001201521CDA721A46927A12091201521C3D
:106E80009A721A46527AF0239A4310324A4B5A7237
:106E90001A465279F0239A431032474B5A711A46D8
:106EA000D279F0239A431032434BDA710B0009F088
:106EB00081FC19F3E9DFD5CBC1B7ADA3998F8778F2
:106EC0006E645A50463E362E261E160EF5003A4A7D
:106ED000D279F0239A437032374BDA7100BF364AC9
:106EE0005279F0239A437032334B5A7100BF324AC1
:106EF000527AF0239A4370322F4B5A7200BF2E4AB7
:106F0000927A12091201D21D2B4B9A7200BF2A4AA3
:106F1000D27A12091201D21D274BDA7200BF264A1B
:106F2000D27AF0239A437032234BDA7200BF224A9E
:106F3000127BF0239A4370321F4B1A7300BF1D4A15
:106F4000203A927EF0239A4370321A4B203B9A7675
:106F500000BF184A203AD27EF0239A437032154B74
:106F6000203BDA7600BF134A203A127F1209120141
:106F7000D21D104B203B1A7700BF0E4A203A527F99
:106F800012091201D21D0B4B203B5A7700BF094A50
:106F9000203A527FF0239A437032064B203B5A77B7
:106FA00000BF044A203A927FF0239A437032014B8B
:106FB000203B03E0682600203C2700209A7700BF92
:106FC000DC4AD27F12091201D21DDA4BDA7700BFF8
:106FD000D84A2032127812091201D21DD54B203323
:106FE0001A7000BFD34A20321278F0239A437032CD
:106FF000D04B20331A7000BFCE4A20325278F02393
:107000009A437032CB4B20335A7000BFC94A2032AA
:10701000927812091201D21DC64B20339A7000BF1C
:10702000C44A2032D27812091201D21DC14B20333A
:10703000DA7000BFBF4A2032927A12091201D21DC3
:10704000BC4B20339A7200BFBA4A2032127AF02326
:107050009A437032B74B20331A7200BFB54A2032C0
:10706000127A12091201D21DB24B20331A7200BFDC
:10707000B04A20329279F0239A437032AD4B2033DC
:107080009A7100BFAB4A2032927912091201D21DC7
:10709000A84B20339A7100BF01E0FFE700BF47E132
:1070A000A44A2032D278F0239A43A24B2033DA70DC
:1070B0001A461279120912011A711A461279F0232E
:1070C0009A439C4B20331A711A46527912091201C5
:1070D0005A711A465279F0239A43964B20335A71CB
:1070E0001A46D27912091201DA711A46D279F023BE
:1070F0009A43904B2033DA711A46527A12091201E0
:107100005A721A46527AF0239A438A4B20335A72A3
:107110001A46927AF0239A43864B20339A721A4683
:107120009278F0239A43834B20339A701A46D27A8E
:1071300012091201DA721A465278120912015A70B3
:107140001A46D27AF0239A437A4B2033DA72794A7C
:10715000D27FF0239A43774BDA771A462032127B9C
:107160001209120120331A73724A927F1209120116
:10717000203B9A771A462032127BF0239A436D4BBC
:1071800020331A736B4A127FF0239A43694B1A77A4
:107190001A462032527B1209120120335A73654A73
:1071A000D27E12091201203BDA76634AD278F023AC
:1071B0009A43614BDA701A46127B120912011A7354
:1071C0001A461279120912011A711A46927AF0239C
:1071D0009A43594B9A721A461279F0239A43564BA6
:1071E0001A711A465279120912015A711A46927985
:1071F000120912019A711A46127A120912011A72B0
:107200001A46127AF0239A434B4B1A721A46527A54
:10721000120912015A72474A203292791209120158
:10722000444B20339A711A469279F0239A43414B8A
:1072300020339A711A46127A120912011A721A46EA
:10724000127AF0239A433B4B20331A721A46927AF1
:10725000120912019A721A46D27812091201DA70D2
:107260001A469278120912019A701A465278F0233F
:107270009A43304B20335A701A461278F0239A43BF
:107280002C4B20331A701A461278120912011A7008
:10729000284AD27F12091201203BDA771A46927FE0
:1072A000F0239A43234B9A771A46527FF0239A434E
:1072B000204B5A771A46527F120912015A771A4602
:1072C000127F120912011A771A46D27EF0239A43CE
:1072D000184BDA761A46927EF0239A43154B9A762B
:1072E000154A127BF0239A43134B1A731A46D27A2B
:1072F000F0239A43104BDA721A46D27A120912011D
:10730000DA721A46927A120912019A721A46527A5F
:10731000F0239A43084B5A721A465279F0239A4343
:10732000054B5A711A46D279F0239A43024BDA710F
:1073300000BD0000482600203C270020F7B582B0A1
:1073400006461746002500200190002E7ED1F9F751
:10735000F9FB05285FD1F9F7F3FC00280DD0FA48B6
:107360004079F02188437030F749487108468078A9
:1073700000090001C01D88700AE0F3484079F0213F
:107380008843F149487108468078000900018870F7
:10739000ED48C07900090001EB49C87108468079C1
:1073A0000009000188710846407900090001487110
:1073B0000846007AF0218843E34908720846007ABB
:1073C0000009000108720846C079F0218843DE49AF
:1073D000C8710846C07800090001C8700846807866
:1073E000F0218843D849887008464078F0218843C6
:1073F000D5494870084640780009000148700846A1
:1074000000790009000108710846C078F02188431E
:10741000CD49C87029E2CC484079F02188437030CA
:10742000C94948710846807800090001C01D88706C
:107430000846C07900090001C87108468079000932
:107440000001887108464079000900E034E000013D
:1074500048710846007AF0218843BB490872084603
:10746000007A0009000108720846C079F0218843BB
:10747000B549C8710846C07800090001C8700846BF
:107480008078F0218843B049887008464078F02120
:107490008843AD49487008464078000900014870AB
:1074A000084600790009000108710846C078F021FB
:1074B0008843A549C870ADE7012E5FD1F9F740FCBC
:1074C00000280DD0A0484079F021884370309E49B3
:1074D00048710846807800090001C01D88700AE0E4
:1074E00099484079F0218843974948710846807847
:1074F0000009000188709448C07900090001924990
:10750000C8710846807900090001887108464079F1
:107510000009000148710846007AF02188438A4931
:1075200008720846007A0009000108720846C0790E
:10753000F02188438449C8710846C07800090001D9
:10754000C87008468078F02188437F4988700846D3
:107550004078F02188437C4948700846407800090B
:1075600000014870084600790009000108710846CA
:10757000C078F02188437449C870EAE3022E7DD1B7
:10758000F9F7E0FA05287AD1F9F7DAFB002877D085
:10759000012F76D10A210398F0F7D2FD0546F9F7BD
:1075A000EFFA002802D16948445D01E06848445D73
:1075B000E007C00F002807D06348C0790009000128
:1075C000C01D6149C87105E05F48C079000900012C
:1075D0005D49C87102202040002807D05A488079B0
:1075E00000090001C01D5849887105E0564880799E
:1075F000000900015449887104202040002807D068
:107600005148407900090001C01D4F49487105E00B
:107610004D484079000900014B494871082020403D
:10762000002807D04848007AF02188437030464946
:10763000087205E04448007AF02188434249087204
:1076400010202040002807D03F48007A00090001A0
:10765000C01D3D49087205E03B48007A0009000161
:10766000394908722020204000280BD03648C079C4
:10767000F021884370303449C87109E0AEE242E13C
:10768000F4E0A4E03048C079F02188432E49C87165
:1076900040202040002807D02B484079F021884323
:1076A00070302949487105E027484079F021884326
:1076B000254948710A210398F0F742FD0D462348F9
:1076C000445DE007C00F002807D01F48C0780009BC
:1076D0000001C01D1C49C87005E01B48C0780009A6
:1076E00000011949C87002202040002807D0164820
:1076F0008078F021884370301349887005E0124883
:107700008078F021884310498870042020400028A8
:1077100007D00D484078F021884370300A494870FE
:1077200005E009484078F02188430749487008205F
:10773000204000280ED00448407800090001C01DF8
:10774000014948700CE0000088260020E81602007D
:10775000FB160200FE48407800090001FC49487011
:1077600010202040002807D0F948007900090001C6
:10777000C01DF749087105E0F548007900090001CE
:10778000F349087120202040002807D0F048C07835
:10779000F02188437030EE49C87005E0EC48C078AD
:1077A000F0218843EA49C87040202040002807D0D3
:1077B000E748807800090001C01DE5498870C8E2EB
:1077C000E348807800090001E1498870C1E2E0489F
:1077D0004079F02188437030DD494871084680784F
:1077E00000090001C01D88700846C0790009000129
:1077F000C8710846807900090001887108464079FF
:107800000009000148710846007AF0218843D049F8
:1078100008720846007A0009000108720846C0791B
:10782000F0218843CA49C8710846C07800090001A0
:10783000C87008468078F0218843C549887008469A
:107840004078F0218843C2494870084640780009D2
:1078500000014870084600790009000108710846D7
:10786000C078F0218843BA49C87072E2B8484079BC
:10787000F0218843B6494871084680780009000124
:1078800088700846C07900090001C87108468079EF
:10789000000900018871084640790009000148711B
:1078A0000846007AF0218843A94908720846007A00
:1078B0000009000108720846C079F0218843A449F4
:1078C000C8710846C07800090001C8700846807871
:1078D000F02188439E49887008464078F02188430B
:1078E0009B494870084640780009000148700846E6
:1078F00000790009000108710846C078F02188432A
:107900009349C87025E2012F73D10A210398F0F73B
:1079100017FC0546F9F734F9002802D18D48445D7B
:1079200001E08D48445DE007C00F002807D088487B
:10793000C07900090001C01D8549C87105E084486F
:10794000C079000900018249C87102202040002846
:1079500007D07F48807900090001C01D7C498871EB
:1079600005E07B488079000900017949887104208D
:107970002040002807D07648407900090001C01D4A
:107980007349487105E07248407900090001704967
:10799000487108202040002807D06D48007AF02167
:1079A000884370306A49087205E06948007AF0211E
:1079B00088436749087210202040002807D0644897
:1079C000007A00090001C01D6149087205E06048A5
:1079D000007A000900015E4908722020204000283A
:1079E00008D05B48C079F021884370305849C8718D
:1079F00006E09DE05648C079F02188435449C8719B
:107A000040202040002807D051484079F021884389
:107A100070304F49487105E04D484079F021884366
:107A20004B4948710A210398F0F78AFB0D464948F3
:107A3000445DE007C00F002807D04548C078000922
:107A40000001C01D4249C87005E04148C0780009E6
:107A500000013F49C87002202040002807D03C4860
:107A60008078F021884370303949887005E03848C3
:107A70008078F0218843364988700420204000280F
:107A800007D033484078F02188437030304948703F
:107A900005E02F484078F02188432D4948700820A0
:107AA0002040002807D02A48407800090001C01D66
:107AB0002749487005E0264840780009000124491C
:107AC000487010202040002807D021480079000984
:107AD0000001C01D1E49087105E01D48007900091C
:107AE00000011B49087120202040002807D01848B9
:107AF000C078F021884370301549C87005E01448FB
:107B0000C078F02188431249C870402020400028E6
:107B100007D00F48807800090001C01D0C4988700B
:107B200017E10B488078000900010949887010E1CD
:107B300007484079F021884370300549487108466C
:107B4000807800090001C01D88700846C07905E0F2
:107B500088260020E8160200FB160200000900013A
:107B6000C87108468079000900018871084640798B
:107B70000009000148710846007AF02188437649DF
:107B800008720846007A0009000108720846C079A8
:107B9000F02188437049C8710846C0780009000187
:107BA000C87008468078F02188436B498870084681
:107BB0004078F021884368494870084640780009B9
:107BC0000001487008460079000900010871084664
:107BD000C078F02188436049C870BAE0032E9FD175
:107BE000F8F7B0FF05285FD1F9F7AAF800280DD003
:107BF00059484079F0218843703057494871084608
:107C0000807800090001C01D88700AE05248407960
:107C1000F0218843504948710846807800090001E6
:107C200088704D48C079000900014B49C871084669
:107C30008079000900018871084640790009000137
:107C400048710846007AF021884343490872084683
:107C5000007A0009000108720846C079F0218843C3
:107C60003D49C8710846C07800090001C87008463F
:107C70008078F02188433849887008464078F021A0
:107C8000884335494870084640780009000148702B
:107C9000084600790009000108710846C078F02103
:107CA00088432D49C87054E02B480079F02188435F
:107CB00070302949087108464079F02188437030B6
:107CC000254948710846807800090001C01D887068
:107CD0000846C07900090001C8710846807900098A
:107CE0000001887108464079000900014871084682
:107CF000007AF0218843184908720846007A000982
:107D0000000108720846C079F02188431249C87101
:107D10000846C07800090001C87008468078F02144
:107D200088430D49887008464078F02188430A4905
:107D300048700846407800090001487008460079FC
:107D40000009000108710846C078F0218843024903
:107D5000C87005B0F0BD00008826002070B505464B
:107D60000C46012D7ED1B148407D00090001C01DA7
:107D7000AE4948750846007DF02188431030AB4974
:107D800008750846007D00090001401C087508467A
:107D9000C07CF02188431030A449C8740846807C18
:107DA000F02188431030A14988740846807C00097E
:107DB0000001401C8874F9F71FF8022803D0F9F776
:107DC0001BF801286CD19A480078012868D0F4F794
:107DD0001FFE9849884263D3F8F7B2FF00282FD0DE
:107DE0009248007DF021884370309049087508461C
:107DF000007D00090001C01D08750846C07CF02107
:107E0000884370308949C8740846807CF0218843D3
:107E10007030864988740846807C00090001C01DC6
:107E200088740846407DF021884370307F4948754A
:107E30000846407CF021884370307C494874F4E067
:107E40007A48007DF021884310307849087508464B
:107E5000007D00090001401C08750846C07CF02127
:107E6000884300E0B4E010307049C8740846807C54
:107E7000F021884310306D4988740846807C0009E1
:107E80000001401C88740846407DF0218843674902
:107E900048750846407CF021884364494874C4E032
:107EA000F8F73EFE002824D1F4F7B2FD614988427C
:107EB0001FD3F8F745FF00280ED05C48407DF02125
:107EC00088437030594948750846407CF021884302
:107ED0007030564948741AE05448407DF021884378
:107EE000524948750846407CF02188434F49487400
:107EF0000DE04E48407DF021884370304B49487575
:107F00000846407CF0218843703048494874F8F7AF
:107F100007FE01282AD146480078012826D0F4F728
:107F200077FD4449884221D34048407DF021884371
:107F300070303E4948750846407CF02188437030D7
:107F40003A494874F8F7FCFE002807D03748007D0E
:107F5000F021884370303549087566E03348007D6C
:107F6000F02188431030314908755EE0230008F0A5
:107F700021FC062C241C140C042D2C48807C0009A8
:107F80000001C01D2949887400BF2848807CF02169
:107F9000884370302549887400BF2448C07CF02194
:107FA000884370302149C87400BF2048007D000913
:107FB0000001C01D1D49087500BF1C48007DF0214F
:107FC000884370301949087500BF00E000BF2CE0FD
:107FD0001648407DF0218843144948750846007DC5
:107FE000F0218843114908750846007D0009000109
:107FF00008750846C07CF02188430C49C8740846BF
:10800000807CF0218843094988740846807C0009F7
:10801000000188740846407D000900014875084643
:10802000407CF02188430149487470BD68260020D7
:10803000E1000020B80B000030B50246002901D154
:10804000002000E00720130008F0B4FB0F09141F04
:108050002B3743505D67727C88929FA9B500574BC0
:108060005B7EF024A3430401F0252C402343534CB2
:108070006376A1E0524B9B79F024A3430401F025E1
:108080002C4023434E4CA37196E04D4B2033DB79BB
:108090001B091B010407240F2343494C2034E371BF
:1080A0008AE0464B2033DB7C1B091B010407240FAD
:1080B0002343424C2034E3747EE0404B40331B7832
:1080C0001B091B010407240F23433C4C403423703D
:1080D00072E03A4B2033DB7FF024A3430401F02508
:1080E0002C402343354C2034E37765E0334B203379
:1080F0005B7BF024A3430401F0252C4023432F4C49
:108100002034637358E02E4B9B791B091B01040735
:10811000240F23432A4CA3714EE0294B9B7CF0246F
:10812000A3430401F0252C402343254CA37443E0D2
:10813000234BDB7E1B091B010407240F2343204C28
:10814000E37639E01D4B2033DB7F1B091B0104075D
:10815000240F2343194C2034E3772DE0174B9B7EEB
:108160001B091B010407240F2343144CA37623E0AF
:10817000134B20339B79F024A3430401F0252C40BA
:1081800023430F4C2034A37116E00D4BDB7D1B09FC
:108190001B010407240F2343094CE3750CE0074B34
:1081A00020335B7C1B091B010407240F2343034C72
:1081B0002034637400E000BF00BF30BD48260020BB
:1081C0001C270020F7B582B007461546002600247C
:1081D000FE480078012804D0F4F71AFCFC498842D4
:1081E00079D2FC48407CF02188437030F9494874CA
:1081F0000846807C00090001C01D88740846007D87
:1082000000090001C01D08750846007DF021884363
:108210007030F04908750846807CF0218843703042
:10822000EC4988740846C07C00090001C01DC87470
:108230000846C07CF02188437030E649C87408467F
:10824000407C00090001C01D48740846407D0009BB
:108250000001C01D48750846407DF02188437030FC
:10826000DC4948750846007CF02188437030D949C4
:1082700008740846007C00090001C01D0874084607
:10828000C07BF02188437030D249C873FF220A2195
:108290000020FBF767F9FF2213210020FBF762F9AA
:1082A000FF2211210020FBF75DF9FF22122100209F
:1082B000FBF758F9FF220E210020FBF753F9FF22AC
:1082C0000F210020FBF74EF9FF2210210020FBF7C1
:1082D00049F9F4E3FFE7039836283DD019DC082874
:1082E0007ED007DC801E030008F064FA0635A8FC87
:1082F000FBFAF97E102874D006DC092872D00D280C
:1083000071D00E2870D1FDE333286ED03428F9D116
:1083100070E13F286AD00FDC3738082864D2430068
:108320007B449B885B009F448A009702FF025F00AA
:108330005F006503CB0318004E287BD006DC402885
:1083400079D0412878D04D28DCD1BBE14F2874D0BA
:108350005028D7D14FE100BF00BF9E48407CF0219C
:1083600088439C4948740846807C00090001887451
:108370000846007D00090001C01D08750846007D03
:10838000F02188437030934908750846807CF021BD
:108390008843904988740846C07C00090001C01DCC
:1083A000C8740846C07CF02188438A49C8740846CE
:1083B000407C0009000148740846407D0009000126
:1083C00048750846407DF021884382494875084633
:1083D000007CF02188437F4908740846007C06E051
:1083E000A1E2FDE337E2D2E3FBE394E028E00009F9
:1083F000000108740846C07BF02188437549C873A2
:10840000FF220A210020FBF7ADF8FF2213210020F4
:10841000FBF7A8F800220E211046FBF7A3F8002274
:108420000F211046FBF79EF8002210211046FBF7A3
:1084300099F877E2ABE110E2DDE26DE000BF00BF4A
:108440006448407CF0218843624948740846807C37
:108450000009000188740846007D00090001C01D64
:1084600008750846007DF021884370305949087529
:108470000846807CF0218843564988740846C07CB1
:1084800000090001C8740846C07CF02188435149A6
:10849000C8740846407C0009000148740846407DC5
:1084A00000090001C01D48750846407DF021884341
:1084B000484948750846007CF021884345490874BE
:1084C0000846007C0009000108740846C07BF021C2
:1084D00088434049C873FF220A21002003E055E188
:1084E000EFE086E016E0FBF73DF8FF2213210020C5
:1084F000FBF738F800220E211046FBF733F8002274
:108500000F211046FBF72EF8002210211046FBF732
:1085100029F88EE700BF00BF2E48407CF021884339
:108520002C4948740846807C00090001C01D8874ED
:108530000846007D00090001C01D08750846007D41
:10854000F02188437030234908750846807CF0216B
:10855000884370301F4988740846C07C00090001B8
:10856000C8740846C07CF02188431A49C87408467C
:10857000407C0009000148740846407D0009000164
:1085800048750846407DF0218843124948750846E1
:10859000007CF02188430F4908740846007C0009DC
:1085A000000108740846C07BF02188430949C8735C
:1085B000FF220A210020FAF7D5FFFF221321002015
:1085C000FAF7D0FF00220E21104605E0E10000205E
:1085D000B80B000088260020FAF7C4FF00220F2104
:1085E0001046FAF7BFFF002210211046FAF7BAFF33
:1085F0001FE700BF00BFFE48407CF0218843FC49D4
:1086000048740846807C00090001C01D8874084633
:10861000007D00090001C01D08750846007DF0219D
:1086200088437030F24908750846807CF021884301
:10863000EF4988740846C07C00090001C8740846E8
:10864000C07CF0218843EA49C8740846407C000990
:108650000001C01D48740846407D000900014875AE
:108660000846407DF0218843E14948750846007C72
:10867000F0218843DE4908740846007C00090001A7
:1086800008740846C07BF0218843D949C873FF228B
:108690000A210020FAF766FFFF2213210020FAF7D3
:1086A00061FF00220E211046FAF75CFF00220F2125
:1086B0001046FAF757FF002210211046FAF752FF32
:1086C000F6E300BFCA48407CF0218843C84948749B
:1086D0000846807C0009000188740846007D000976
:1086E000000108750846007DF02188437030C049BC
:1086F00008750846807CF0218843BD498874084687
:10870000C07C00090001C8740846C07CF021884381
:108710007030B749C8740846407C000900014874AD
:108720000846407D0009000148750846407DF0215B
:108730008843AF4948750846007CF0218843AC491E
:1087400008740846007C0009000108740846C07BD4
:10875000F0218843A649C873FF220A210020FAF7B6
:1087600001FFFF2213210020FAF7FCFE00220E2158
:108770001046FAF7F7FE00220F211046FAF7F2FE34
:10878000002210211046FAF7EDFE91E300BF984851
:10879000407CF0218843964948740846807C000953
:1087A000000188740846007D00090001087508462C
:1087B000007DF021884370308D4908750846807C23
:1087C000F02188438A4988740846C07C000900016A
:1087D000C8740846C07CF02188438549C87408469F
:1087E000407C0009000148740846407D00090001F2
:1087F00048750846407DF021884370307C494875B3
:108800000846007CF0218843794908740846007CBA
:108810000009000108740846C07BF02188437449B0
:10882000C873FF220A210020FAF79CFEFF221321C1
:108830000020FAF797FE00220E211046FAF792FE6A
:1088400000220F211046FAF78DFE0022102110465B
:10885000FAF788FE2CE300BF00BF6548407CF0219A
:1088600088437030624948740846807C00090001E2
:10887000C01D88740846007D00090001C01D0875F0
:108880000846007DF0218843703059490875084634
:10889000807CF0218843564988740846C07C0009D2
:1088A0000001C8740846C07CF02188435049C87450
:1088B0000846407C0009000148740846407D0009D4
:1088C000000148750846407DF021884348494875B5
:1088D0000846007CF0218843454908740846007C1E
:1088E0000009000108740846C07BF0218843404914
:1088F000C873FF220A210020FAF734FEFF22132159
:108900000020FAF72FFE00220E211046FAF72AFE69
:1089100000220F211046FAF725FE002210211046F2
:10892000FAF720FEC4E200BF3148407CF0218843C2
:108930002F4948740846807C000900018874084665
:10894000007D0009000108750846007DF02188437C
:108950007030274908750846807CF02188432449F7
:1089600088740846C07C00090001C8740846C07CB1
:10897000F021884370301E49C8740846407C0009C5
:10898000000148740846407D00090001487508460A
:10899000407DF0218843164948750846007CF02147
:1089A0008843134908740846007C000900010874D4
:1089B0000846C07BF02188430D49C873FF220A2175
:1089C0000020FAF7CFFDFF2213210020FAF7CAFD9D
:1089D00000220E211046FAF7C5FD00220F21104695
:1089E000FAF7C0FD002210211046FAF7BBFD5FE246
:1089F0008826002000BFFC48407CF0218843FA49CB
:108A000048740846807C0009000188740846007D8F
:108A10000009000108750846007DF0218843703088
:108A2000F14908750846807CF0218843EE49887436
:108A30000846C07C00090001C8740846C07CF021CB
:108A40008843E949C8740846407C0009000148741D
:108A50000846407D0009000148750846407DF02128
:108A600088437030E04948750846007CF02188430F
:108A7000DD4908740846007C0009000108740846B6
:108A8000C07BF0218843D849C873FF220A21002007
:108A9000FAF768FDFF2213210020FAF763FD002298
:108AA0000E211046FAF75EFD00220F211046FAF75C
:108AB00059FD002210211046FAF754FDF8E1F8E1C3
:108AC000C948407CF02188437030C7494874084643
:108AD000807C00090001C01D88740846007D0009E3
:108AE0000001C01D08750846007DF0218843BE497D
:108AF00008750846807CF0218843BB498874084685
:108B0000C07C00E0A9E000090001C8740846C07CF0
:108B1000F0218843B449C8740846407C000900012C
:108B200048740846407D0009000148750846407DAC
:108B3000F0218843AC4948750846007CF021884301
:108B4000A94908740846007C000900010874084619
:108B5000C07BF0218843A449C873FF220A2100206A
:108B6000FAF700FDFF2213210020FAF7FBFC002298
:108B70000E211046FAF7F6FC00220F211046FAF7F4
:108B8000F1FC002210211046FAF7ECFC90E1964827
:108B9000407CF0218843944948740846807C000951
:108BA000000188740846007D000900010875084628
:108BB000007DF02188438C4908750846807CF021AF
:108BC0008843894988740846C07C00090001C8743C
:108BD0000846C07CF02188438349C874084601E0F8
:108BE0009EE003E1407C0009000148740846407D96
:108BF0000009000148750846407DF02188437A4904
:108C000048750846007CF021884377490874084677
:108C1000007C0009000108740846C07BF0218843ED
:108C200070307149C87300220A211046FAF79AFC85
:108C3000002213211046FAF795FCFF220E21002096
:108C4000FAF790FC00220F211046FAF78BFC002265
:108C500010211046FAF786FC2AE16348407CF02197
:108C60008843614948740846807C00090001887483
:108C70000846007D0009000108750846007DF021C6
:108C80008843594908750846807CF0218843564935
:108C900088740846C07C00090001C8740846C07C7E
:108CA000F02188435049C8740846407C00090001FF
:108CB00048740846407D0009000148750846407D1B
:108CC000F0218843484948750846007CF0218843D4
:108CD000454908740846007C00090001C01D08745D
:108CE0000846C07BF02188433F49C87300220A210F
:108CF0001046FAF737FC002213211046FAF732FC2F
:108D000000220E211046FAF72DFCFF220F21002031
:108D1000FAF728FC002210211046FAF723FCC7E0DE
:108D20003148407CF02188432F4948740846807CB4
:108D30000009000188740846007D000900010875DB
:108D40000846007DF0218843274908750846807C45
:108D5000F0218843244988740846C07C000900013A
:108D6000C8740846C07CF02188431F49C87408466F
:108D7000407C0009000148740846407D000900015C
:108D800048750846407DF0218843174948750846D4
:108D9000007CF02188437030134908740846007C39
:108DA0000009000108740846C07BF02188430E4981
:108DB000C87300220A211046FAF7D4FB00221321BF
:108DC0001046FAF7CFFB00220E211046FAF7CAFB35
:108DD00000220F211046FAF7C5FBFF2210210020C8
:108DE000FAF7C0FB64E0000088260020FD48407CC4
:108DF000F0218843FB4948740846807C0009000143
:108E000088740846007D0009000108750846007D49
:108E1000F0218843F34908750846807CF021884397
:108E2000F04988740846C07C00090001C8740846EF
:108E3000C07CF0218843EB49C8740846407C000997
:108E4000000148740846407D000900014875084645
:108E5000407DF0218843E34948750846007CF021B5
:108E60008843E04908740846007C00090001087442
:108E70000846C07BF0218843DA49C87300220A21E2
:108E80001046FAF76FFB002213211046FAF76AFB2F
:108E900000220E211046FAF765FB00220F21104632
:108EA000FAF760FB002210211046FAF75BFB00BFC7
:108EB00000BF002F03D0CC48007A002808D1F3F778
:108EC000A7FDCA49884203D3C9480078012872D156
:108ED000FF2211210020FAF745FBFF22122100207A
:108EE000FAF740FBC2480078012804D0F3F790FD60
:108EF000BE49884216D2BF48807BF021884370303B
:108F0000BC498873084640300078F02188437030AF
:108F1000B849403108700846007800090001C01DBA
:108F200008702DE07D20C000854214D2B148807BBE
:108F3000F0218843AF498873084640300078F0211B
:108F400088437030AB49403108700846007800090A
:108F50000001087014E0A748807BF021884370303E
:108F6000A4498873084640300078F0218843A1491D
:108F7000403108700846007800090001C01D0870E3
:108F80007D20C000854205D201462846EFF7D8F87B
:108F9000064604E098492846EFF7D2F8064694487A
:108FA0000078012804D0F3F733FD9049884203D2BA
:108FB0009248845D02E0A0E29148845DE007C00F22
:108FC000002809D08B484030C07800090001C01D3E
:108FD00088494031C87007E086484030C0780009B1
:108FE000000184494031C87002202040002807D089
:108FF0008048C07900090001C01D7E49C87105E0A4
:109000007C48C079000900017A49C87104202040D9
:10901000002807D07748807900090001C01D7549F4
:10902000887105E0734880790009000171498871F1
:1090300008202040002807D06E484079F02188435E
:1090400070306C49487105E06A484079F0218843E6
:109050006849487110202040002807D065484079B1
:1090600000090001C01D6349487105E0614840796D
:10907000000900015F49487120202040002807D0E6
:109080005C480079F021884370305A49087105E046
:1090900058480079F0218843564908714020204003
:1090A000002807D053488079F02188437030514917
:1090B000887105E04F488079F02188434D498871D7
:1090C0007D20C000854213D264212846EFF738F88E
:1090D000064647480078012804D0F3F799FC434935
:1090E000884202D24548845D23E04548845D20E003
:1090F000642128463230EFF723F87D21C900009023
:10910000EFF71EF8019164210198EFF719F8064670
:109110003C48854208D236480078012804D0F3F74D
:1091200077FC3249884202D23448845D01E03448F9
:10913000845DE007C00F002809D02E4840308078B9
:10914000F021884370302B494031887007E029486E
:1091500040308078F02188432649403188700220D1
:109160002040002807D02348807A00090001C01D54
:109170002049887205E01F48807A000900011D49D6
:10918000887204202040002807D01A48407A00093D
:109190000001C01D1749487205E01648407A0009D1
:1091A00000011449487208202040002807D01148C7
:1091B000007AF021884370300E49087205E00D48AE
:1091C000007AF02188430B490872102020400028C3
:1091D0001AD00848007A00090001C01D054908722C
:1091E00018E0000088260020580A0020B80B000074
:1091F000E1000020FC260020A0860100E816020005
:10920000FB16020010270000FE48007A000900014A
:10921000FC49087220202040002807D0F948C07976
:10922000F02188437030F749C87105E0F548C079EE
:10923000F0218843F349C87140202040002807D01E
:10924000F048407AF02188437030EE49487205E0DA
:10925000EC48407AF0218843EA4948727D20C000FA
:10926000854219D20A212846EEF76AFF0A210190A9
:10927000EEF766FF0E460A2D08D2E3480078012873
:1092800004D0F3F7C5FBE149884202D2E048845D8F
:1092900012E0E048845D0FE0642128463230EEF7AA
:1092A0004FFF0A210090EEF74BFF0A210190EEF7E5
:1092B00047FF0E46D6498C5DE007C00F002809D055
:1092C000D0484030807800090001C01DCD494031B0
:1092D000887007E0CB484030807800090001C94918
:1092E0004031887002202040002807D0C548807B8C
:1092F00000090001C01DC349887305E0C148807B97
:1093000000090001BF49887304202040002807D0CD
:10931000BC48407B00090001C01DBA49487305E004
:10932000B848407B00090001B64948730820204036
:10933000002807D0B348007BF02188437030B14942
:10934000087305E0AF48007BF0218843AD490873FE
:1093500010202040002807D0AA48C07A0009000148
:10936000C01DA849C87205E0A648C07A00090001DE
:10937000A449C87220202040002807D0A148807A44
:10938000F021884370309F49887205E09D48807ABB
:10939000F02188439B49887240202040002807D054
:1093A0009848407BF021884370309649487305E027
:1093B0009448407BF0218843924948737D20C00047
:1093C000854207D20A212846EEF7BAFE0E4690489B
:1093D000845D0BE0642128463230EEF7B1FE0A21AD
:1093E0000190EEF7ADFE0E4689498C5DE007C00F97
:1093F000002809D0834840304078F02188437030FD
:1094000080494031487007E07E4840304078F02184
:1094100088437C494031487002202040002809D010
:1094200078484030407800090001C01D754940313E
:10943000487007E0734840304078000900017149E6
:109440004031487004202040002807D06D48007C3F
:10945000F021884370306B49087405E06948007C4E
:10946000F02188436749087408202040002807D06D
:109470006448007C00090001C01D6249087405E0D1
:109480006048007C000900015E49087410202040FB
:10949000002807D05B48C07BF021884370305949D1
:1094A000C87305E05748C07BF02188435549C8730D
:1094B00020202040002807D05248C07B000900012E
:1094C000C01D5049C87305E04E48C07B000900012B
:1094D0004C49C87340202040002807D04948407CB0
:1094E00000090001C01D47494874ECE04548407C34
:1094F0000009000143494874E5E000220A211046B2
:10950000FAF730F8002213211046FAF72BF8002260
:1095100011211046FAF726F8002212211046FAF718
:1095200021F800220E211046FAF71CF800220F2124
:109530001046FAF717F8002210211046FAF712F831
:1095400030484030C078000900012E494031C870D1
:109550002C48C079000900014039C871084680795B
:1095600000090001887108464079F02188432549A7
:1095700048710846407900090001487108460079A1
:10958000F02188431F49087108468079F0218843FB
:109590001C498871084640308078F0218843194979
:1095A000403188701748807A00090001403988727C
:1095B0000846407A0009000148720846007AF02106
:1095C0008843104908720846007A000900010872B1
:1095D0000846C079F02188430A49C8710846407A94
:1095E000F0218843074948720846403080780009D6
:1095F0000001403188700348807B00090001403938
:10960000887309E0FC260020E1000020B80B000070
:10961000E8160200FB1602000846407B0009000124
:1096200048730846007BF0218843284908730846A0
:10963000C07A00090001C8720846807AF021884388
:10964000224988720846407BF02188431F494873AD
:10965000084640304078F02188431C49403148702A
:10966000084640780009000148701848007CF02145
:109670008843164908740846007C000900010874F4
:109680000846C07BF02188431049C8730846C07B58
:1096900000090001C8730846407C000900014874B5
:1096A0000846807BF021884308498873084640308B
:1096B0000078F02188430549403108700846007859
:1096C00000090001087005B0F0BD0000FC26002074
:1096D000F7B582B007460E460121FF200830FBF7A0
:1096E00099FF0121FC48FBF795FFFC480078012811
:1096F0007ED0F3F78DF9FA49884279D3F7F722FA49
:10970000032843D1F7F718FA002803D0F7F714FA23
:1097100001283BD1002F1CD1F7F712FB00280CD0F9
:10972000F048407CF0218843EE4948740846807C2C
:1097300000090001C01D8874EEE0EA48407CF02179
:109740008843E84948740846807C00090001887411
:10975000E2E0F7F7F5FA00280CD0E248407CF0216F
:1097600088437030DF4948740846807C0009000156
:109770008874D1E0DB48407CF0218843D9494874A3
:109780000846807C000900018874C5E0F7F7D4F929
:10979000002803D0F7F7D0F9012865D1002F0CD1AC
:1097A000D048407CF0218843CE4948740846807CEC
:1097B00000090001C01D88740BE0CA48407CF021FC
:1097C00088437030C74948740846807C000900010E
:1097D0008874F7F7B1F9002821D1C2482030C07849
:1097E000F02188437030BF492031C870BD4800E087
:1097F00064E0807D00090001203988750846807D7D
:10980000F0218843B7498875FF2223210020F9F70A
:10981000A9FE002222211046F9F7A4FE7CE0F7F70A
:109820008BF9012878D1AF482030C078F0218843E7
:10983000AC492031C870AB48807D00090001C01DD3
:10984000203988750846807DF02188437030A5490D
:109850008875002223211046F9F784FEFF22222179
:109860000020F9F77FFE57E09E48407CF0218843B6
:109870009C4948740846807C0009000188740846A9
:109880002030C078F021884396492031C87095482F
:10989000807D00090001203988750846807DF0210F
:1098A000884390498875002223211046F9F75AFE13
:1098B000002222211046F9F755FE2DE08948407C10
:1098C000F02188437030874948740846807C00093D
:1098D0000001C01D887408462030C078F0218843FC
:1098E000703080492031C8707E48807D00090001B9
:1098F000C01D203988750846807DF021884370306E
:1099000078498875FF2223210020F9F72BFEFF22DA
:1099100022210020F9F726FEF7F70EF9002808D0DB
:109920006E480078012804D0F3F772F86C49884239
:1099300076D26D48864209D96A4820304079F021B4
:109940008843703067492031487107E0654820300E
:109950004079F0218843634920314871634930469A
:10996000EEF7EEFB0A210190EEF7EAFB0D465E48AA
:10997000401C864202D35E48445D01E05D48445D80
:10998000E007C00F002809D056482030C0780009F1
:109990000001C01D53492031C87007E051482030F4
:1099A000C078000900014F492031C87002202040D2
:1099B000002809D04B4820308078F021884370304F
:1099C00048492031887007E0464820308078F021EF
:1099D000884344492031887004202040002809D061
:1099E000404820304078F021884370303D49203194
:1099F000487007E03B4820304078F02188433949DF
:109A0000203148700820204000280AD035482030F6
:109A1000407900090001C01D32492031487108E039
:109A2000A1E2304820304079000900012D49203161
:109A3000487110202040002809D02A4820300079A1
:109A4000F0218843703027492031087107E025480C
:109A500020300079F02188432249203108712020EC
:109A60002040002809D01F4820300079000900015B
:109A7000C01D1C492031087107E01A4820300079C8
:109A800000090001174920310871402020400028BA
:109A900009D014482030807800090001C01D114908
:109AA0002031887007E00F482030807800090001DD
:109AB0000C49203188707D21C9003046EEF740FB0B
:109AC0000A210190EEF73CFB0D460848864213D36D
:109AD0000748445D12E0000005050000E100002099
:109AE000B80B0000FC2600209F8601001027000014
:109AF000E8160200FB160200F948445DE007C00FBB
:109B0000002807D0F748C07FF02188437030F5491E
:109B1000C87705E0F348C07FF0218843F149C87752
:109B200002202040002807D0EE48C07F0009000135
:109B3000C01DEC49C87705E0EA48C07F0009000174
:109B4000E849C87704202040002807D0E548807FF6
:109B500000090001C01DE349887705E0E148807FE6
:109B600000090001DF49887708202040002809D03B
:109B7000DC482030407800090001C01DD94920315F
:109B8000487007E0D7482030407800090001D549E7
